:10000000B81E02200D02010815020108170201089E
:10001000190201081B0201081D020108000000006E
:100020000000000000000000000000001F020108A6
:100030002102010800000000230201086184030876
:10004000CB2D040827020108270201082702010816
:100050002702010827020108270201084B36010880
:1000600027020108270201082702010827020108C8
:1000700027020108270201082702010827020108B8
:1000800027020108270201082702010827020108A8
:100090002702010827020108270201082702010898
:1000A0002702010827020108270201082702010888
:1000B000D18403082702010827020108693A0208CF
:1000C000613A0208270201082702010827020108F5
:1000D0002702010839A003082702010827020108A6
:1000E0002702010827020108270201082702010848
:1000F0002702010827020108270201082702010838
:100100002702010827020108270201082702010827
:10011000270201086D990308270201082702010838
:10012000752001087D200108270201082702010827
:1001300027020108270201082702010827020108F7
:1001400027020108270201082702010827020108E7
:10015000852001082702010827020108270201085B
:1001600027020108270201082702010827020108C7
:1001700027020108659F02086D20010800000000A9
:1001800027020108270201087599030827020108C0
:100190002702010827020108270201082702010897
:1001A0009D640208956402082702010827020108DD
:1001B0002702010827020108270201082702010877
:1001C00027020108270201086B2101082702010804
:1001D00027020108270201082702010871560308B7
:1001E0002702010827020108270201082702010847
:1001F0009364020827020108DFF80CD000F058FAD7
:1002000000480047C55F0408B81E02200648804722
:1002100006480047FEE7FEE7FEE7FEE7FEE7FEE7EB
:10022000FEE7FEE7FEE7FEE76D840308F90101083B
:1002300040EA01039B0703D009E008C9121F08C068
:10024000042AFAD203E011F8013B00F8013B521EE8
:10025000F9D27047D2B201E000F8012B491EFBD25F
:1002600070470022F6E710B513460A4604461946C1
:10027000FFF7F0FF204610BD10B5044604E00B78F0
:1002800000F8013B03B1491C521EF8D2204610BDB4
:10029000421C10F8011B0029FBD1801A704703464D
:1002A00011F8012B00F8012B002AF9D118467047EC
:1002B00030B50B46014600202022012409E021FA36
:1002C00002F59D4205D303FA02F5491B04FA02F533
:1002D0002844151EA2F10102F1DC30BD2DE9F05FCA
:1002E0000546002092469B468846064681464024A5
:1002F0001BE0284641464746224600F0FAF953469D
:100300005A46C01A914110D311461846224600F0B1
:10031000E1F92D1A67EB01084F4622460120002122
:1003200000F0D8F917EB00094E41201EA4F101049A
:10033000DFDC484631462A464346BDE8F09F2DE9BA
:10034000FE4F804681EA0300C00F0C46009021F06A
:10035000004123F00045B8EB0200A94105D2404618
:10036000214690461C460B46024623F000401043AF
:1003700047D0270DC7F30A00C3F30A510290401A71
:10038000019040286BDAC3F3130040F4801B0098FF
:10039000924620B10023D2EB030A63EB0B0B0198CA
:1003A0005946C0F14002504600F094F906460D4609
:1003B00050465946019A00F0ACF910EB0800614133
:1003C000002487EA115284EAE7731A4340D0009A66
:1003D00062B3019A012A4FEA075215DC001B61EB58
:1003E00002014FF0004202EA0752CDE90042001C30
:1003F00041F5801132462B4600F0ACF903B0BDE860
:10040000F08F40462146F9E7001B61EB0201001C1A
:1004100041F5801300185B412018A2F5001747EB47
:10042000030140EAD570B6196D4111E06D084FEA3D
:10043000360645EAC0754FEA0752001B61EB020120
:10044000001C41F5801149084FEA30000019514164
:1004500032462B4603B0BDE8F04F00F06CB900986F
:10046000012240000023D0EB020263EBE07300980E
:1004700021464FEAE074B8EB000061EB0401E9E7C4
:1004800083F000435BE781F0004158E72DE9FE4F20
:1004900081EA030404F0004421F0004100944FF08D
:1004A000000B23F0004350EA01045ED052EA03043B
:1004B0005BD0C3F30A54C1F30A552C44A4F2F334BD
:1004C0000194A0FB0254C1F3130141F48011C3F362
:1004D000130343F4801301FB024400FB034E840A20
:1004E000970A44EA815447EA8357A4FB07680295B8
:1004F0008D0A05FB07854FEA932C04FB0C54270556
:10050000029D4FEA065847EA1637B5EB08056EEB31
:10051000070C870E920E47EA811742EA8312A7FB67
:100520000201B6EB0B0164EB00042B0D43EA0C3324
:100530005E1844EB1C50DA465146E7FB0201C5F356
:1005400013044FEA0B3343EA14534FEA0432019C7D
:1005500043EA0603A4F10C040294009CCDE900B424
:1005600000F0F8F803B0BDE8F08F00200146F9E78D
:100570002DE9F04D81EA030404F0004B21F0004521
:1005800014464FF0000A23F0004150EA050220D043
:1005900054EA01021DD0C5F30A570246C5F31303FE
:1005A000C1F31300C1F30A5640F4801543F48013DD
:1005B000A7EB0608101BD64608F2FD3873EB0500C2
:1005C00002D308F1010801E092185B41B8F1000F75
:1005D00003DA00200146BDE8F08D00204FF48011C1
:1005E000064684460EE0171B73EB050705D3121B66
:1005F00063EB050306434CEA010C49084FEA30005F
:1006000092185B4150EA0107EDD152EA030012D083
:1006100082EA040083EA0501084305D0101BAB41C0
:1006200006D20122002306E000224FF0004302E040
:100630006FF0010253101AEB06004CEB085110EB5F
:100640000A0041EB0B01BDE8F04D00F074B8C1F3B6
:100650000A52C1F3130140F2FF3341F480119A4270
:1006600002DA00200146704740F233439A42A2F278
:10067000334202DC524200F03CB800F02BB80000DC
:1006800030B5041E71F1000404DB4FF00044404219
:1006900064EB0101141E73F1000405DB1C464FF0EE
:1006A0000043524263EB0403994208BF904230BDBD
:1006B000064C074D06E0E06840F0010394E80700AF
:1006C00098471034AC42F6D3FFF79AFDA89B0D086B
:1006D000C89B0D08202A04DB203A00FA02F1002012
:1006E00070479140C2F1200320FA03F31943904070
:1006F0007047202A04DB203A21FA02F000217047DB
:1007000021FA02F3D040C2F1200291400843194679
:100710007047202A06DBCB17203A41FA02F043EA61
:10072000E07306E041FA02F3D040C2F120029140AA
:1007300008431946704710B5141E73F1000408DA17
:10074000401C41F1000192185B411A4301D120F095
:10075000010010BD2DE9F04D92469B4611B1B1FA52
:1007600081F202E0B0FA80F220329046FFF7B2FF49
:1007700004460F4640EA0A0041EA0B0153465A4636
:10078000084313D0114653EA010019D0C8F14002C2
:100790005046FFF7AEFF05460E46504659464246C4
:1007A000FFF798FF084305D0012004E020463946B2
:1007B000BDE8F08D0020054346EAE0762C43374340
:1007C0000A986305E40AA0EB08000022FD0A44EA47
:1007D00047540A3002D500200146E9E70105101907
:1007E0006941DDE9084500196941BDE8F04DA2E71E
:1007F00070B58C1810F8015B15F0070301D110F8E3
:10080000013B2A1106D110F8012B03E010F8016B0F
:1008100001F8016B5B1EF9D12B0705D40023521E92
:100820000DD401F8013BFAE710F8013BCB1A921CFA
:1008300003E013F8015B01F8015B521EF9D5A142F8
:10084000D8D3002070BD0000014800887047000028
:100850001400002010B51648164908604FF44030C7
:100860004860002113488160016181610162416239
:10087000C1628162C1600121C161002101634161E6
:100880000DF0BCFC10B16FF0010010BD11200A4941
:1008900008600120486000208860C86005480DF0AD
:1008A000EBFB10B14FF0FF30EFE70020EDE7000069
:1008B000002001403C260020CC26002000B5064840
:1008C0000DF008FD28B10320044908600420044904
:1008D0000870002000BD00003C260020680E0020AB
:1008E0005D0E0020014800887047000016000020BF
:1008F00010B51648164908604FF440304860002192
:10090000134881600161816101624162C16281625B
:10091000C1600121C1610021016341610DF06EFCE4
:1009200010B16FF0010010BD08200A4908600120D5
:10093000486000208860C86005480DF09DFB10B13C
:100940004FF0FF30EFE70020EDE70000002201400C
:1009500084260020CC26002000B505480DF0BAFC06
:1009600020B104200349086003490870002000BD3D
:1009700084260020680E00205D0E002008B5694620
:10098000002011F0C3FE40B1BDF90010002901DACA
:1009900000210091BDF9000008BD0C48006842F23A
:1009A0001071484340F6FF71B0FBF1F00849096847
:1009B00048434FF47A71B0FBF1F040F654314843AC
:1009C00042F21071B0FBF1F0E6E70000600E00208B
:1009D000580E002008B56946012011F097FE40B17D
:1009E000BDF90010002901DA00210091BDF90000D5
:1009F00008BD0C48006842F21071484340F6FF7190
:100A0000B0FBF1F00849096848434FF47A71B0FB34
:100A1000F1F040F65431484342F21071B0FBF1F06E
:100A2000E6E70000640E0020580E002043490968E4
:100A300021F44031424AC2F804131146D1F804139C
:100A4000426811433D4A11600168496821F4807190
:100A50000268516001684A68016942EA012102683E
:100A600051600168496821F0407102685160016875
:100A7000496882681143026851600168896821F4FD
:100A800000610268916001688968C2681143026868
:100A900091600168896821F0706102689160016865
:100AA0008968826A1143026891600168896821F04F
:100AB00040510268916001688968C26A1143026806
:100AC00091600168896821F0020102689160016803
:100AD0008A68816942EA4101026891600168496857
:100AE00021F40061026851600168C96A21F4700153
:100AF0000268D1620168CA6A818B491E42EA0151CB
:100B00000268D1620168896821F40071026891600D
:100B100001688A68016B42EA4121026891600168BC
:100B2000896821F480610268916001688A6841697E
:100B300042EA81210268916070470000042301406D
:100B40000020014010B5084821F0E2FF04460748A4
:100B5000604340F6FF71B0FBF1F00549B1FBF0F0E6
:100B60000449086010BD000098090020A08601001B
:100B7000000E2707580E002010B54E4800780128B7
:100B800007D14D480068806840F080404A490968B4
:100B9000886048480078032807D148480068806882
:100BA00040F08040454909688860424800784449DF
:100BB00008700846007804287AD2DFE800F00209BD
:100BC000303701203B49087064203E4908806FE0BF
:100BD0003C480088002805DD3A480088401E394915
:100BE000088005E001203849086004203149087078
:100BF00031480068006800F0020002280ED16FF052
:100C000012002D49096808602B480068C06C2F4904
:100C10000880FFF797FF02202649087048E003206C
:100C20002449087064202749088041E0254800884D
:100C3000002805DD23480088401E2249088005E081
:100C400002202149086004201A4908701B480068E6
:100C5000006800F00200022829D16FF01200174945
:100C60000968086015480068C06C194908802CF0B4
:100C7000B3FB2CF01BFC00200E490870052011F07E
:100C800067FDA0B15B2029F033FBFFF7A3FE04B2A0
:100C9000204629F071FB2C2029F02AFBFFF76EFE7D
:100CA00004B2204629F068FB5D2029F021FB00BF3B
:100CB00000BF10BD5D0E00203C26002084260020D1
:100CC0005C0E00205E0E0020680E00201400002044
:100CD000160000207CB505460C4601208DF800006A
:100CE0000020ADF802000848446034F0DFFF0648F9
:100CF0004068001B019000208DF80000DDE9000134
:100D0000C5E900017CBD0000DC2600207CB505465D
:100D10000E46144601208DF800000020ADF80200B8
:100D200008484460084A314634F086FF0548406868
:100D3000001B019000208DF80000DDE90001C5E9ED
:100D400000017CBDDC2600200053070070B586B092
:100D500005460E46144601208DF810000020ADF81F
:100D600012000F210CA24FF4C873CDE90206CDE9A1
:100D700000211A4621460A4834F0A6FF00208DF8CB
:100D8000100007484068001B0590DDE90401C5E933
:100D9000000106B070BD000000000000000000006F
:100DA000DC2600200A6810700A68521C0A6070472E
:100DB00070B505460C462DB904F10801C8B201F022
:100DC00039FA70BD04F11701C8B201F033FAF8E73F
:100DD0001CB5002007490871088048800846016852
:100DE00000918088ADF80400DDE9000102F0CAFD41
:100DF0001CBD00007E1700202DE9FC4106460F4671
:100E000015461C46B4F5C87F01DD002402E0C4F598
:100E1000C87084B2012008490871084605804480E2
:100E2000016800918088ADF80400DDE9000102F05E
:100E3000A9FDBDE8FC8100007E1700200FB410B5AD
:100E4000829C2046E31704EBD363C3F34F11E317EF
:100E500004EBD3635B11A4EB43139AB205A850F8DB
:100E6000210001239340184018B1012010BC5DF807
:100E700014FB0020FAE730B50C46CD1701EBD56521
:100E8000C5F34F12CD1701EBD5656D11A1EB4515DB
:100E9000ABB200F10C0454F8224001259D402C40D7
:100EA0005CB100F10C0454F8225001249C402D1B2D
:100EB00000F10C0444F822500AE000F10C0454F84C
:100EC000225001249C40254400F10C0444F8225097
:100ED00030BD000010B50648007838B118F04CFC61
:100EE000FF2001F080F900200149087010BD0000CA
:100EF000C91600202DE9F04704460D4616461F4648
:100F0000DDE9099ADDF8208026806780A4F8048056
:100F1000A4F806902846FFF7BBF9608732222946DD
:100F200004F10800FFF7A8F901213D200155002038
:100F300084F83C00A08FE087C4F840A0BDE8F087AB
:100F40002DE9F0410446884615461E46069FB8F135
:100F5000000F2AD00020B4F90010A94212DCB4F925
:100F60000010B4F904201144A9420BDBB4F90210BB
:100F7000B14207DCB4F90210B4F906201144B142C1
:100F800000DB012038B194F83C1069B9012184F8E4
:100F90003E10397008E094F83C10012904D100217A
:100FA00084F83E10012139700CE094F83C000128CF
:100FB00008D1002084F83E0001203870206C08B170
:100FC000206C8047BDE8F0812DE9F0410446884659
:100FD00015463F20015D3D20005D814201D001208A
:100FE000287094F83E103D20005D814201D0012020
:100FF0002870E08FA0873D20005D002850D094F835
:101000003C00022806D150231A461946FF200BF057
:101010004BFE10E094F83C00012806D1FF231A464D
:10102000194618460BF040FE05E096231A4619466D
:10103000FF200BF039FEB4F806C01FFA8CF3B4F8A9
:1010400004C01FFA8CF2B4F802C01FFA8CF1B4F895
:1010500000C01FFA8CF00BF033FDB4F9040000EB74
:10106000D071228802EB6101628F02EB4202A1EB98
:1010700042010EB2B4F9060000EBD071628802EBB7
:101080006101C91F0FB200231A461946FF200BF059
:101090000BFEB9B2B0B204F1080207F0A7FF00BF1F
:1010A000BDE8F08102463F208154012070470000D6
:1010B0000148006870470000700E00200748007863
:1010C000012803D005480078022804D100200349F4
:1010D0000870012070470020FCE70000740E00201B
:1010E00005480078022804D1002003490870012037
:1010F00070470020FCE70000740E00202DE9FE433D
:101100000E48006840F001000C490860084600687D
:1011100000F0010900240025032601274FF00008F4
:101120002B462246012106488DE8C0010BF008FF3E
:1011300004481FF057F9BDE8FE8300003038024034
:1011400000000240780E002002200149087070471C
:10115000740E00207047000010B5064800681FF0AC
:1011600009F90446642C04D902481FF03BF900F049
:1011700015FF10BD780E002010B52DED048B0E4824
:1011800000681FF0F7F808EE100AB8EE480BB0EE52
:10119000409B9FED0A0B89EE001BB0EE419B094876
:1011A00090ED000B30EE090B80ED000B02481FF0B4
:1011B00019F9BDEC048B10BD7C1500200000000067
:1011C0000088C3408015002000B513F063FB0028A1
:1011D00006DC00200C49088002200C49087012E04F
:1011E0000B4814F005F830B968200749088003203F
:1011F0000649087007E00020034908800549088077
:1012000001200249087000BDC2140020BE14002055
:10121000C0140020C414002010B518481FF0E2F8D4
:10122000002426E016480078012820D115480088BF
:10123000B0F57A7F06DB6920134908800320104946
:10124000087010BD1148008811490E4A128821F813
:1012500012000E4814F096F828B10A480088401C85
:101260000849088003E0022005490870E9E7601C8E
:1012700084B2C82CD6DB00BFE3E70000C81400200E
:10128000BE140020C4140020C2140020C01400208A
:10129000DC51012010B5012026F0AAFE10BD00008F
:1012A0000148007870470000E00E00200148006807
:1012B00070470000800E0020014800687047000061
:1012C000940E002001480068704700008C0E00203A
:1012D0000148006870470000880E0020014800683F
:1012E00070470000840E002001480068704700002D
:1012F000980E00200148006870470000900E002002
:1013000001480068704700009C0E002001480068FA
:1013100070470000A80E00200148006870470000D8
:10132000A40E00200148006870470000AC0E0020A9
:101330000148006870470000B00E002001480068B6
:1013400070470000A00E00200148006870470000B0
:10135000B40E00200148008870470000D40E002021
:101360000148006870470000CC0E0020014800785A
:1013700070470000B80E00202DE9FE4300F078FF12
:101380007C49086000F078FF7B4908604FF4C87022
:101390007A49086008460068C821484377490860D0
:1013A0000846006800EB40000860084600688008B6
:1013B00008607348006840F0010071490860084601
:1013C000006800F001006F4908606D48001F006868
:1013D00040F480006A49091F08600846006800F46C
:1013E0008000684908606648001F006840F00100FE
:1013F0006349091F08600846006800F00100614960
:1014000008605F48001F006840F002005C49091F47
:1014100008600846006800F002005A490860584811
:10142000001F006840F004005549091F0860084685
:10143000006800F00400534908605148001F00682C
:1014400040F008004E49091F08600846006800F097
:1014500008004C4908604A48001F006840F010002E
:101460004749091F08600846006800F01000454918
:10147000086002274FF00008032400250D2643468C
:101480003A46502140488DE870000BF059FD434624
:101490003A4680213D488DE870000BF051FD4346EF
:1014A0003A464FF43C613A488DE870000BF048FD35
:1014B00043463A46482137488DE870000BF040FD1E
:1014C00043463A46602134488DE870000BF038FD01
:1014D000E02132480170780331490860E02130484A
:1014E000083880F8391338064FF0E021C1F80401BC
:1014F0002C48006820F001002A49086004E02A48CE
:101500000068401C284908602648006800F0010077
:101510000028F4D1254823490860202021491431AE
:10152000086040201F49203908604FF4706008604F
:10153000E0201F4908600846C06840F01000C860FD
:101540000846C06840F00800C8600846C06840F01F
:101550000400C8600846C06840F00200C860084641
:10156000C06840F00100C860002012490870BDE862
:10157000FE830000BC0E0020C00E0020C40E002020
:1015800034380240DC0E002000000240000402401B
:1015900000080240000C0240001002404EE400E04F
:1015A00008E100E0286402407C0E0020005406029E
:1015B00000000550B80E0020014800787047000078
:1015C000E50E00200021304A1069304A1268521C92
:1015D0002E4B1A6000F00402042A0ED12C4A126825
:1015E000521C2B4B1A6001210422274B5A61294AB5
:1015F000126822F00102274B1A6000F00202022A50
:101600000ED10121244A1268521C234B1A60022277
:101610001D4B5A611F4A126822F001021D4B1A60CD
:1016200000F01002102A08D11C4A1268521C1B4BF1
:101630001A6001211022144B5A6100F00802082A96
:101640000CD1114A926A164B1A60164A1268521C43
:10165000144B1A60012108220B4B5A6100F0010261
:1016600052B1114A1268521C0F4B1A60012101221B
:101670000E4B1A70044B5A6121B90D4A1268521C64
:101680000B4B1A607047000000000550800E0020D0
:10169000840E002028640240880E00208C0E00205A
:1016A000F40E0020900E0020940E0020B90E0020B1
:1016B000980E00200021454A1268521C434B1A60C4
:1016C000434A106800F40072BAB1414A28321268E5
:1016D00002F004028AB13E4A2832126822F0040263
:1016E0003B4B28331A605A15394B08331A600121D5
:1016F000384A1268521C374B1A6000F040027AB127
:10170000334A3C32126802F080024AB14022304B28
:1017100008331A60304A1268521C2F4B1A6001219C
:1017200000F4807282B12A4A2832126802F0020262
:1017300052B14FF48072264B08331A60274A126860
:10174000521C264B1A60012100F480621AB3204A11
:101750002832126802F00802EAB1214A1268521CCB
:101760001F4B1A6001218A02194B08331A60184A6C
:101770002832126802F480226AB9154A28321268A7
:1017800002F480723AB9124A2832126822F0080232
:101790000F4B28331A6000F400627AB10C4A2832E9
:1017A000126802F010024AB10E4A1268521C0D4B28
:1017B0001A600121CA02064B08331A6021B90A4A8D
:1017C0001268521C084B1A60704700009C0E0020E3
:1017D00000640240A00E0020A40E0020A80E0020ED
:1017E000AC0E0020B00E0020B40E00200748007898
:1017F000022809D106480088401C054908800420B9
:1018000002490870012070470020FCE7E00E00202C
:10181000D40E00200348006840F001000149086030
:10182000704700000000055008B51448007818B152
:101830001248007802281ED111480068401C104947
:1018400008604FF4FA700F49088001200B490870B6
:1018500000200D49087026F0CBFB0C481EF0C2FD9D
:10186000002003460246009004480178082002F058
:1018700011FA012008BD0020FCE70000B80E00208E
:10188000D00E0020C80E0020B90E0020D80E002077
:101890000348006820F0010001490860704700001B
:1018A0000000055010B518F0A1FC10BD08B514F0EB
:1018B00031FE1A48007801282FD11948007880B1EC
:1018C00000201749087014F0EDFD0020134908703E
:1018D00003460246009008460178082002F0DAF933
:1018E0001BE0104800681EF045FDB0F5FA6F14D9F2
:1018F0000D480068401C0C49086002200749087028
:10190000FFF7C6FF14F0D4FD002003460246009006
:1019100002480178082002F0BDF908BDB80E002089
:10192000B90E0020D80E0020CC0E00200748007809
:10193000022803D103200549087006E00348007817
:10194000012802D10020014908707047E00E0020F4
:101950000748007818B901200549087006E00448D6
:101960000078032802D10220014908707047000066
:10197000E00E002030B587B004461EF063F985B252
:1019800001A9284613F0A4FBC8B19DF8060010B9C0
:101990000B20207015E09DF80A0010B10A2020707D
:1019A0000FE0BDF812004FF6FF71884202D1072008
:1019B000207006E000202070012007B030BD082014
:1019C00020700020F9E70000002004E00021034A15
:1019D0001154411C88B20228F8DB7047041400201F
:1019E000002004E00021034A1154411C88B20B2856
:1019F000F8DB7047CC27012038B504460020009062
:101A00008DF801406B460222502111F0FBFA402074
:101A10000149086038BD00001804024010B54FF4B9
:101A200000720448016801F500710348FEF700FCEC
:101A300010BD00009C1400207C61012010B54FF403
:101A4000007204490448006800F50070FEF7F0FBDE
:101A500010BD00007C6101209C1400202DE9F04F96
:101A60000E46DDE909450021DDF82CB0BBF1000F81
:101A700009D0BBF1010F08D0BBF1020F07D0BBF1B9
:101A8000040F08D105E0042107E0032105E002214D
:101A900003E0022101E0BDE8F08F00BF0027D0F88D
:101AA00004B00BF4704BC0F804B0D0F808B00BF4DD
:101AB000704BC0F808B004F10B0B1FFA8BFC934479
:101AC000ABF1010B1FFA8BF805F10B0B1FFA8BF929
:101AD0009B44ABF1010B1FFA8BFA4CEA084BC0F8A0
:101AE00004B049EA0A4BC0F808B0D0F810B02BF0A7
:101AF000070BC0F810B0DDF82CB0C0F810B0BB4632
:101B0000C0F818B0D0F814B02BF0FF0BC0F814B028
:101B10004FF0FF0BC0F814B0D0F81CB040F2077EB5
:101B20002BEA0E0BC0F81CB040F2076BC0F81CB0DB
:101B3000D0F828B0BB46C0F828B086620F46D0F86F
:101B40002CB00BF0E02BC0F82CB093460BFB07FB3E
:101B50000BF1030B02FB07FE4BEA0E4BC0F82CB057
:101B6000D0F830B06FF30A0BC0F830B0036300BF99
:101B700091E700002DE9F34F83B00C4625462B2D4D
:101B80002DDA04EB4400174951F8306004EB4400AF
:101B900001EBC000078904EB440001EBC000B0F882
:101BA0000A8004EB440001EBC00080891FFA80F931
:101BB00004EB440001EBC000B0F812A004EB4400B9
:101BC00001EBC000B0F814B043463A463146CDE9C7
:101BD00000ABCDF808900398FFF740FF00BF05B0B9
:101BE000BDE8F08F040F00202DE9F84307460E46AC
:101BF00015469846DDF820902B4632460221C80152
:101C0000CDF8008002F046F800204B463A4602210B
:101C10000090C80102F03EF848488488002108304E
:101C200000EB441001704548083000EB4410478039
:101C30004248083000EB441006714048083000EB81
:101C40004410C580284627F0B8FB3C49083101EB19
:101C500044110881C8213948083000EB4410418103
:101C60002946304606F0E8FD01463448083000EBCE
:101C70004410017329463046FFF79AF82F4908317E
:101C800001EB44110861384613F000FA2B49083182
:101C900001EB441108752948083000EB4410007D21
:101CA000A0B1384612F02CFE00EE100AB8EE400B40
:101CB000234890ED001B20EE010BBCEEC00B1F482B
:101CC000083000EB441080ED060A05E000211B48B7
:101CD000083000EB4410816101211848083000EB06
:101CE0004410017715488088401C144988800220E0
:101CF000C6EB061101EB4101124A02EB810105EB33
:101D0000450201F82200C6EB061000EB40000D4929
:101D100001EB800005EB450100EB81004760C6EB5D
:101D2000061000EB4000074901EB800005EB450180
:101D300000EB8100C0F80880BDE8F8833C73012007
:101D4000681600206C780120F8B506460D46002084
:101D50002B463246032100904FF4807001F09AFF29
:101D60002F4884880121083000EB441001700021C5
:101D70002B48083000EB441041802948083000EB24
:101D8000441006712648083000EB4410C5802846F0
:101D900027F013FB2249083101EB44110881C821C7
:101DA0001F48083000EB4410418100211C480830D6
:101DB00000EB441001751A48083000EB44108161B3
:101DC0001748083000EB4410017715488088401C04
:101DD000134988800120C6EB061101EB4101114A2D
:101DE00002EB810105EB450201F822000020C6EB61
:101DF000061101EB41010B4A02EB810105EB4502A3
:101E000001EB82014860C6EB061101EB4101054A76
:101E100002EB810105EB450201EB82018860F8BD10
:101E20003C7301206C780120F8B506460D46002071
:101E30002B46324604210090880101F02BFF2F48E9
:101E400084880221083000EB4410017000212B48E7
:101E5000083000EB441041802848083000EB441063
:101E600006712648083000EB4410C580284627F04C
:101E7000A4FA2249083101EB44110881C8211F4806
:101E8000083000EB4410418100211C48083000EB71
:101E9000441001751948083000EB4410816117485F
:101EA000083000EB4410017714488088401C134927
:101EB00088800020C6EB061101EB4101104A02EBBD
:101EC000810105EB450201F82200C6EB061101EB8A
:101ED00041010B4A02EB810105EB450201EB820156
:101EE0004860C6EB061101EB4101054A02EB810196
:101EF00005EB450201EB82018860F8BD3C730120CF
:101F00006C78012070B506460D4620488488002173
:101F1000083000EB441001701C48083000EB4410FE
:101F2000468002211948083000EB4410017100215D
:101F30001648083000EB4410C1801448083000EB0C
:101F4000441001811148083000EB441041810F48D2
:101F5000083000EB441001730C48083000EB4410CB
:101F60000561304613F092F801460848083000EB4E
:101F70004410017500210548083000EB441001773A
:101F800002488088401C0149888070BD3C73012054
:101F900000200149888070473C7301202F48007859
:101FA00020B1012825D0022856D142E02C480069F2
:101FB00000F0010028B92B480088401C29490880FE
:101FC00002E00020274908802648008803280FDD0A
:101FD0002548007818B124480078032802D1012050
:101FE0002149087000201F49088001201B49087002
:101FF00032E01B48006900F0010028B11948008850
:10200000401C1849088002E0002016490880154845
:10201000008803280CDD002012490880124800784F
:10202000012802D102201049087002200B490870D3
:1020300012E00C480088401C0A49088008460088C5
:102040001E2808DD0648006900F0010018B10020D4
:1020500008800249087000BF00BF70476E0E002064
:10206000000002406C0E0020740E002010B5FFF737
:10207000A9FA10BD10B521F02DF910BD10B5FFF76C
:1020800019FB10BD10B521F0DBF910BD0146087831
:1020900010381823B0FBF3F20848805CC865032AA7
:1020A00005D908686FF30900001D886503E008681A
:1020B0006FF309008865886D70470000F86E0408AA
:1020C000014600208A6A8B69CBB932B1012A0DD052
:1020D000022A03D0032A10D10EE000BFCB6A03F01E
:1020E0008073B3F1807F00D1012007E0CB6AB3F1A8
:1020F000C07F00D1012001E000E000BF34E08B6927
:10210000B3F5005F1AD132B1012A07D0022A03D0F9
:10211000032A11D10AE000BF01200EE0CB6A03F0D0
:102120008073B3F1807F00D1012006E0CB6AB3F168
:10213000C07F00D1012000E000BF15E032B1012ACC
:1021400005D0022A04D0032A0CD103E000BF00BF4F
:10215000012008E0CB6A03F08073B3F1807F00D1E7
:10216000012000E000BF00BF704710B500F0AAFCDE
:1021700010BD0146002205E0002301F51F7040F864
:102180002230521C0F2AF7D3002204E0002301F171
:102190001C008354521CB2F5007FF7D30020087056
:1021A0004870012088700020C1F8B80201230B7626
:1021B00040238B7100234B7681F81C32012381F878
:1021C0001D32704710B50548007828B9002000F08E
:1021D0000AF801200149087010BD0000C91600204E
:1021E00010B50A9C10BD10B5044623465122152196
:1021F000002034F0D1F910BD0348406820F00800F9
:102200000149486070470000007001400348406881
:1022100040F008000149486070470000007001402C
:1022200000487047C084AFC1014840687047000053
:10223000040F002001460A462B2A06DA01EB410072
:10224000034B03EBC000406870470020FCE7000030
:10225000040F00200148D0F894037047040F0020B9
:1022600000487047C084AFC100487047C0D7B6C1AE
:102270004FF04040704700000048704780A903C0FD
:102280000148008870470000FA0E002001480088CD
:1022900070470000FE0E00200148008870470000D3
:1022A000FC0E00200148008870470000000F00204D
:1022B00070B505460C4626462B2E09DA04EB440081
:1022C000074A02EBC00118222846FDF7B1FF70BD96
:1022D000182204492846FDF7ABFF00BFF7E70000CE
:1022E000040F0020DC270020014800687047000030
:1022F0001068014001480068704700000C68014008
:1023000001480068704700001868014001480068F3
:1023100070470000086801400148006870470000ED
:10232000146801400148006870470000AC68014033
:102330000148006870470000846801400148006857
:102340007047000094680140014800687047000031
:102350008868014001480068704700008C680140AF
:1023600001480068704700002C690140014800687E
:102370007047000004690140014800687047000090
:102380001469014001480068704700000869014075
:1023900001480068704700000C690140014800785E
:1023A000704700000D1300200148007870470000BE
:1023B000020F0020FEB5FE48006840F00100FC4915
:1023C00008600846006800F00107FA48006820F439
:1023D0004030F84908600846006840F480300860E2
:1023E0000846806820F4403088600846806840F4E1
:1023F000003088600846406820F4807048600846D5
:10240000C06820F44030C860E948006840F480604B
:10241000E74908600846006800F48067E6480068FD
:1024200020F44040E44908600846006840F48040D9
:102430000860E1480830006840F44040DE49083157
:102440000860081F006820F08000091F0860DA4853
:102450000C30006820F44040D7490C310860084631
:10246000006840F480400860D3481830006840F4A9
:102470000000D14918310860142034F021F8CE480A
:102480001830006840F08000CB49183108601420F3
:1024900034F016F8C6481430006840F08060C44933
:1024A000143108600846006800F08067C0480C38A6
:1024B000006840F08060BE490C390860084600683A
:1024C00020F080600860BA48006840F40000B84915
:1024D00008600846006800F40007B5482038006826
:1024E00040F40000B249203908600846006820F432
:1024F00000000860AE481430006840F00060AC494D
:10250000143108600846006800F00067A8480C38DD
:10251000006840F00060A6490C3908600846006871
:1025200020F000600860F021A44801704FF0807036
:10253000A3490860F021A248083880F85A134FF0E8
:1025400080604FF0E021C1F80801F0219B480A307B
:10255000017004204FF0E021C1F80C01944830389C
:10256000006820F08050924930390860002400E073
:10257000641C8F4830380068C0F340700028F7D1E1
:1025800090488B4958310860081D006800F44030BD
:10259000091D086086483038006840F08050844942
:1025A0003039086000E0641C814830380068C0F3AE
:1025B00040700028F7D08448406820F00800824925
:1025C00048608248006820F00100804908607F4828
:1025D0009C30006820F006007C499C3108607A48F5
:1025E000006B20F00100784908630846006B20F07A
:1025F000807008630846006B40F08070086300E05C
:10260000641C7148C06800F480500028F8D06E48FF
:10261000006B6F4908406C4908630846006B42F63E
:1026200090110843684908630846006B40F00100B8
:10263000086300E0641C6448C06800F480700028EF
:10264000F8D062489C30006840F006005F499C3139
:1026500008605E489030006820F003005B499031CC
:1026600008600846006840F0010008605748A03044
:10267000006820F003005549A03108600846006852
:1026800008605248001D006820F0FF004F49091DF6
:1026900008600846006840F00400086005254D48C1
:1026A00068434D49B0FBF1F64748806920F03F0090
:1026B0004549886108468069304388610020434964
:1026C000C031086000214148C43001603F483030CB
:1026D000006840F001003D49303108603A48006828
:1026E00020F00100384908600846006840F0010009
:1026F000086036480830006820F00300334908318C
:10270000086008460068086030481030006820F013
:1027100007002E4910310860084600680860081F4D
:10272000006820F00F00091F08600846006840F0AC
:10273000050008602448006820F00E002249086067
:102740000846006840F00A000860204860300068D1
:102750006FF30F001D49603108600846006840F4BF
:10276000C87008601848006820F0F000164908603A
:1027700008460068086015486430006820F00100D1
:102780001249643108600846006840F001000860A2
:102790000D48806840F001000B4988600846806859
:1027A00040F0020088600948643000680B4917E077
:1027B00030380240000002400028024058E400E0A7
:1027C00008E100E00060035300700140046C014028
:1027D0000386FCFF00093D00A0252600FF80F0FED7
:1027E0000840AD49086008460068AC490843AA495A
:1027F00008600846006820F002000860084600688B
:102800000860A748006820F07040A54908600846A5
:1028100000680860A24810380068A2490840A04932
:10282000103908600846006840F005100860081D6F
:1028300000689C4908409A490C39086008460068BD
:1028400040F00A100860081D006896490840944945
:1028500008390860084600689349084390490839D8
:102860000860081D00688F4908408D49091F0860ED
:10287000084600688D4908438949091F086088484F
:102880001430006800F07F40854914310860002052
:10289000086083481C30006840F0040080491C3107
:1028A00008600846006840F0020008607C48006844
:1028B00040F001007A49086077486438006840F0C9
:1028C00001007549643908607948406840F00800A3
:1028D000774948600A2033F0F3FD0523FE221521D5
:1028E000002033F059FE002305221521184633F04D
:1028F00053FE0723FE221521002033F04DFE4F2307
:1029000007221521002033F047FE0A23FE2215215D
:10291000002033F041FE1B231C221521002033F040
:102920003BFE0023FE221521184633F035FE00231E
:1029300035221521184633F02FFE002311220521E0
:10294000184633F029FE0020034602462921009054
:1029500033F0C4FD40F2311033F0B2FD00232922E0
:102960000521184633F018FE002033F0A9FD0020A1
:102970008DF808008DF8090001208DF80A008F20DD
:102980008DF80B0000208DF804008DF80500012063
:102990008DF806008F208DF8070046483623012267
:1029A00039210090002033F099FD02A82A23042247
:1029B00039210090002033F091FD01A82B2304223F
:1029C00039210090002033F089FD3B483A23012251
:1029D00039210090002033F081FD962033F070FD06
:1029E0002D480068354908402B49086008460068B2
:1029F00008600846006820F0020008600846006889
:102A0000086025483C38006820F01F0022493C3906
:102A100008600846006840F00400086024484068E8
:102A200040F0040022494860002000F0E9F81C480A
:102A30006C30006840F0010019496C3108600120D9
:102A400000F0EEF81648EC30006840F00100144940
:102A5000EC310860012012490C310860000218496D
:102A60008861012033F02CFD012012E04FF08071CD
:102A7000134A9161002100E0491CA629FCDB4FF4B8
:102A800080710F4A9161002100E0491CA629FCDBFE
:102A9000401C1628EADBFEBD686C0140007F0F0079
:102AA0001868014000F800F09A019A019F019F0107
:102AB00000700140F80E0020F90E0020FF80F0FEAB
:102AC000000002403CB53948C468002538480088F9
:102AD000401C3749088004F00100A0B13548008847
:102AE000401C344908800125012030490861002339
:102AF00034221521184633F04FFD2C48406840F031
:102B000004002A49486004F00200002847D02A48FF
:102B10000088401C284908800125022023490861BB
:102B20000846406820F0080048602448007800EB20
:102B30004000234901EBC000406822490860224858
:102B4000007800EB40001E4901EBC00040681D49C1
:102B5000803108601B488838006840F0010019493E
:102B6000883908601148406840F008000F49486003
:102B700000208DF804008DF8050001208DF8060076
:102B80008F208DF8070001A82A2304223921009004
:102B9000002033F0A3FC01200C49087000BF25B9C8
:102BA0000B480088401C0A4908803CBD0070014069
:102BB000FA0E0020FC0E0020FE0E00200C13002058
:102BC000040F0020AC6801400D130020030F00200B
:102BD000000F0020704770470348006840F0010074
:102BE00001490860704700002468014003480068FC
:102BF00040F001000149086070470000246801406E
:102C000030B5044625462B2D05DA034804702146CD
:102C10000248FEF7AFFF30BD0C130020846801406E
:102C200030B5044625462B2D05DA034804702146AD
:102C30000248FEF79FFF30BD0D13002004690140DC
:102C400070B50B4600EB4004104D55F8341000EB06
:102C5000400405EBC4042489544300EB40050B4EAB
:102C600006EBC5052D7C04FB051100EB4004354641
:102C700005EBC404247C03FB041100EB400405EBCA
:102C8000C4046160024C216070BD0000040F00208C
:102C9000AC68014010B500EB40020B4B03EBC202E5
:102CA000138900EB4002084C04EBC202127C534330
:102CB00000EB400204EBC202127C4A43D21C42EAFF
:102CC0000342024B1A6010BD040F0020B06801409F
:102CD0002DE9F04100F10B0C1FFA8CF49444ACF197
:102CE000010C1FFA8CF501F10B0C1FFA8CF69C44B9
:102CF000ACF1010C1FFA8CF744EA054CDFF81480A4
:102D0000C8F800C046EA074C08F10408C8F800C03B
:102D1000BDE8F0818868014070B50B4600EB4004C7
:102D2000104D55F8341000EB400405EBC404248921
:102D3000544300EB40050B4E06EBC5052D7C04FB10
:102D4000051100EB4004354605EBC404247C03FB6D
:102D5000041100EB400405EBC4046160024C2160E7
:102D600070BD0000040F00202C69014010B500EB7D
:102D700040020B4B03EBC202138900EB4002084CEC
:102D800004EBC202127C534300EB400204EBC2028C
:102D9000127C4A43D21C42EA0342024B1A6010BD25
:102DA000040F0020306901402DE9F04100F10B0CC7
:102DB0001FFA8CF49444ACF1010C1FFA8CF501F16C
:102DC0000B0C1FFA8CF69C44ACF1010C1FFA8CF72B
:102DD00044EA054CDFF81480C8F800C046EA074C06
:102DE00008F10408C8F800C0BDE8F0810869014096
:102DF0000948007868B90120074908700020074990
:102E000008700748406840F0040005494860012008
:102E100070470020FCE70000020F0020030F002095
:102E20000070014005480078012805D10448007869
:102E300010B100200149087070470000020F002007
:102E4000030F00207FB542233C223121FF2009F0EF
:102E50002BFF09F01DFF054600EBD5704410B82389
:102E60001A4640F22B2120B209F0AEFD01A811F064
:102E7000DDF840F28110B623009001A807C807F0E2
:102E800039F97FBD1FB5022009F030FF01A811F00C
:102E9000CDF84FF4C370B623009001A807C807F01F
:102EA00029F91FBD7FB542233C223121FF2009F0C3
:102EB000FBFE09F0EDFE054600EBD5704410B8238B
:102EC0001A4640F22B2120B209F07EFD01A811F034
:102ED000ADF840F28110B623009001A807C807F0B2
:102EE00009F97FBD70B504460D4616463246B7EE69
:102EF000000B2946204600F001F870BD2DE9F74F80
:102F00002DED020B8FB005468A46B0EE403BB7EE82
:102F1000004BB4EEC43BF1EE10FA0BDBFE48007838
:102F2000FF2807DB1FFA8AF1A8B209F00BFF14B0E3
:102F3000BDE8F08FF948008800287DD1F848046882
:102F4000F8480068800000FB0A4404EB85041398ED
:102F500010B1012871D118E0F34890F800B0F3489F
:102F600000780E90F24800780D90EB4800780C90B5
:102F70009DED0C4AB8EE444B24EE034BBCEEC44B23
:102F800014EE100AC0B20C90AAE0E678A77894F884
:102F9000018094F80090E048007804EE100AB8EE42
:102FA000444BB0EE441B21EE034BB0EE441B04EE49
:102FB000106AB8EE444B81EE045BB0EE451BDA4874
:102FC000007804EE100AB8EE444BB0EE440B20EE4D
:102FD000014BB0EE440B04EE107AB8EE444BB0EE69
:102FE000442BB7EE004B34EE414B24EE024BB0EED7
:102FF000442B30EE024BBCEEC44B14EE100A00F032
:10300000FF0BCA48007804EE100AB8EE444BB0EE4D
:10301000440B20EE014BB0EE440B04EE108AB8EEE8
:10302000444BB0EE442BB7EE004B34EE414B24EE54
:10303000024BB0EE442B01E05CE050E030EE024B7E
:10304000BCEEC44B14EE100AC0B20E90B848007823
:1030500004EE100AB8EE444BB0EE440B20EE014BE8
:10306000B0EE440B04EE109AB8EE444BB0EE442B95
:10307000B7EE004B34EE414B24EE024BB0EE442B46
:1030800030EE024BBCEEC44B14EE100AC0B20D90F1
:10309000A148007804EE100AB8EE444BB0EE440BA1
:1030A00020EE034BB0EE440BB7EE004B34EE404B3A
:1030B000B0EE440BC6F1010004EE100AB8EEC44BAA
:1030C000B0EE442BB7EE004B00EE424BB0EE440B9B
:1030D000BCEEC04B14EE100AC0B20C9027E726E7F6
:1030E00000BF0C98E07084F802B00E9860700D98E4
:1030F0002070EEE18948008801287CD18848046866
:103100008848006800EB400000FB0A4405EB4500DE
:103110000444139810B1012809D109E082480078CD
:10312000A07082480078607081480078207088E044
:10313000A77894F8018094F80090FF2676480078EC
:1031400004EE100AB8EE444BB0EE441B21EE034BE4
:10315000B0EE441B04EE106AB8EE444B81EE045B03
:10316000B0EE451B7048007804EE100AB8EE444BF0
:10317000B0EE440B20EE014BB0EE440B04EE107A9F
:10318000B8EE444BB0EE442BB7EE004B34EE414B5F
:1031900024EE024BB0EE442B30EE024BBCEEC44B9F
:1031A00014EE100A00F0FF0B6048007804EE100ADD
:1031B000B8EE444BB0EE440B20EE014BB0EE440BA6
:1031C00004EE108AB8EE444BB0EE442BB7EE004B41
:1031D00034EE414B24EE024BB0EE442B30EE024B6A
:1031E000BCEEC44B14EE100AC0B20E9050480078EA
:1031F00004EE100A00E025E0B8EE444BB0EE440BBC
:1032000020EE014BB0EE440B04EE109AB8EE444BA6
:10321000B0EE442BB7EE004B34EE414B24EE024BA4
:10322000B0EE442B30EE024BBCEEC44B14EE100A51
:10323000C0B20D9084F802B00E9860700D982070A6
:1032400000BF46E1354800880428FAD1DFF8D0C035
:10325000DCF80040DFF8CCC0DCF800C04FEA4C0CD2
:103260000CFB0A4404EB4504DDF84CC0BCF1000F34
:1032700003D0BCF1010F7CD123E0DFF8B8C09CF88B
:1032800000C04FEA2C10DFF8ACC09CF800C00CF076
:103290000F0104EE100AB8EE444B24EE034BBCEED3
:1032A000C44B14EE10CA0CF0FF0001EB001C0CF034
:1032B000FF036370DFF880C09CF800C084F800C092
:1032C00005E194F801C0CDF824C094F800C0CDF811
:1032D00020C0DDF824C04FEA2C12DDF824C00CF029
:1032E0000F0CCDF81CC0DDF820C04FEA2C1CCDF827
:1032F00018C0DDF820C00CF00F0CCDF814C0DFF8BA
:1033000034C09CF800C04FEA2C10DFF828C09CF8AD
:1033100000C00CF00F0111E0EA130020E8130020B8
:10332000DC130020E0130020EB130020EC1300203E
:10333000ED130020EE130020EF130020DFF898C1FA
:103340009CF800C04FEA2C1CCDF82CC0DFF888C1D7
:103350009CF800C00CF00F0CCDF828C004EE100A49
:10336000B8EE444BB0EE441B21EE034BB0EE441BD1
:1033700000E0ABE004EE102AB8EE444B81EE045BB3
:10338000B0EE451B04EE101AB8EE444BB0EE440B01
:1033900020EE014BB0EE440B9DED074AB8EE444BD6
:1033A000B0EE442BB7EE004B34EE414B24EE024B13
:1033B000B0EE442B30EE024BBCEEC44B14EE10CA00
:1033C0000CF0FF0CCDF80CC09DED0B4AB8EE444B51
:1033D000B0EE440B20EE014BB0EE440B9DED064ADF
:1033E000B8EE444BB0EE442BB7EE004B34EE414BFD
:1033F00024EE024BB0EE442B30EE024BBCEEC44B3D
:1034000014EE10CA0CF0FF0ECDF808E09DED0A4A4C
:10341000B8EE444BB0EE440B20EE014BB0EE440B43
:103420009DED054AB8EE444BB0EE442BB7EE004B91
:1034300034EE414B24EE024BB0EE442B30EE024B07
:10344000BCEEC44B14EE10CA0CF0FF0CCDF804C057
:1034500004EE100AB8EE444BB0EE440B20EE034BE2
:10346000B0EE440BB7EE004B34EE404BB0EE440BE5
:10347000C2F1010C04EE10CAB8EEC44BB0EE442BFE
:10348000B7EE004B00EE424BB0EE440B9FED134BFA
:1034900020EE044BBCEEC44B14EE10CA0CF0FF0E31
:1034A000CDF810E0DDE903CE0CEB0E1C0CF0FF03B1
:1034B000DDE901CE0CEB0E1C0CF0FF0CCDF800C0CA
:1034C0006370DDF800C084F800C000E02FE500BFA5
:1034D00000BF00BF2BE50000EF130020000000003C
:1034E00000E06F402DE9F04104460D4616460A2CD7
:1034F0006AD2DFE804F0050F19232D37414B555FE1
:103500000AF00CFD074600233A463146284608F0EB
:1035100079FB59E00AF006FD074600233A4631469A
:10352000284608F06FFB4FE00AF000FD0746002335
:103530003A463146284608F065FB45E00AF0FAFCB9
:10354000074600233A463146284608F05BFB3BE03D
:103550000AF0F4FC074600233A463146284608F0B4
:1035600051FB31E00AF0EEFC074600233A463146B3
:10357000284608F047FB27E00AF0E8FC074600234E
:103580003A463146284608F03DFB1DE00AF0E2FCD1
:10359000074600233A463146284608F033FB13E03D
:1035A0000AF0DCFC074600233A463146284608F07C
:1035B00029FB09E00AF0D6FC074600233A463146CB
:1035C000284608F01FFB00BF00BFBDE8F0817FB5B3
:1035D00042233C223121FF2009F066FB09F058FB11
:1035E000054600EBD5704410B8231A466FF09A01D7
:1035F00020B209F0E9F901A810F018FD0F20B62358
:10360000009001A807C806F075FD7FBD7FB5422375
:103610003C223121FF2009F047FB09F039FB054628
:1036200000EBD5704410B8231A466FF09A0120B20F
:1036300009F0CAF901A810F0F9FC0F20B623009098
:1036400001A807C806F056FD7FBD10B525F068FE3D
:1036500010BD000010B500241FE011480078A04202
:1036600019DD1048007820B90F4850F824100020C8
:1036700088470C480078012804D10B4850F82410E2
:103680000120884707480078022804D1064850F8EE
:10369000241002208847601C84B20A2CDDDB10BD98
:1036A000AA170020A8170020F008022070B50546D0
:1036B0000E4600240BE007480078A04205DD0648CE
:1036C00050F82420314628469047601C84B2032CD1
:1036D000F1DB70BDD21400207C63012070B505467B
:1036E00000240AE006480078A04204DD054850F8AE
:1036F000241028468847601C84B2032CF2DB70BD7E
:1037000054180020B00B022070B5054600240AE0D2
:1037100006480078A04204DD054850F824102846E9
:103720008847601C84B2032CF2DB70BDBA1C0020F9
:10373000BC0B022070B5054600240AE0064800785C
:10374000A04204DD054850F8241028468847601C34
:1037500084B2032CF2DB70BDC51C0020C80C022013
:1037600070B5054600240AE006480078A04204DD52
:10377000054850F8241028468847601C84B2032C62
:10378000F2DB70BD121D0020FC0C022070B5054656
:1037900000240AE006480078A04204DD054850F8FD
:1037A000241028468847601C84B2032CF2DB70BDCD
:1037B000881D00206C0D022070B5054600240AE02B
:1037C00006480078A04204DD054850F82410284639
:1037D0008847601C84B2032CF2DB70BDAD1D002055
:1037E000900D022070B5054600240AE006480078D6
:1037F000A04204DD054850F8241028468847601C84
:1038000084B2032CF2DB70BDB91D00209C0D022098
:1038100070B5054600240AE006480078A04204DDA1
:10382000054850F8241028468847601C84B2032CB1
:10383000F2DB70BDBF1D0020440E022070B50546AE
:1038400000240AE006480078A04204DD054850F84C
:10385000241028468847601C84B2032CF2DB70BD1C
:10386000D51D0020700E022070B5054600240AE028
:1038700006480078A04204DD054850F82410284688
:103880008847601C84B2032CF2DB70BDD91D002078
:10389000A00E02207FB500240BE007480078A0426C
:1038A00005DD064850F824509DE80F00A847601C2D
:1038B00084B2032CF1DB7FBDD1130020482301200B
:1038C0002DE9FC47044604EB4410294901EB0010A4
:1038D000B0F9009004EB441001EB0010468804EBB3
:1038E000441001EB001090F80C7204EB441001EB53
:1038F0000010B0F80E8204EB441001EB00100079C8
:10390000012820D100251BE01A480078A84215DDC7
:1039100004EB4410DFF858A00AEB001000F58473A4
:1039200004EB44100AEB0010CDE90078B0F80A224D
:10393000B1B2114850F825C04846E047681C85B22E
:10394000032DE1DB11E000250DE00C480078A842D2
:1039500007DDB1B20A4850F825C043463A4648460A
:10396000E047681C85B2032DEFDBBDE8FC87000053
:103970008428012039140020D0510120381400205F
:10398000C451012013B582B000200090BDF80A3068
:10399000BDF808209DF80C104FF4805000F07AF923
:1039A00000240BE007480078A04205DD064850F8E7
:1039B0002420DDE902019047601C84B2032CF1DB76
:1039C0001FBD000097170020707F012070B50546CD
:1039D0000E4600240BE007480078A04205DD0648AB
:1039E00050F82420314628469047601C84B2032CAE
:1039F000F1DB70BD0B170020F47C012070B505468B
:103A00000E4600240BE007480078A04205DD06487A
:103A100050F82420314628469047601C84B2032C7D
:103A2000F1DB70BD0A170020E87C01202DE9F0478A
:103A300011F022FB054629F019F8012800D100E019
:103A40000020074610F02EFB044610F017FF8246B8
:103A500010F080FF824501DA012000E0002081465D
:103A600010F018FF002801DD012000E000200646CC
:103A700015F07CFD032801D0012000E000208046E5
:103A8000B8F1000F04D0022017494873887314E07E
:103A900027B901201449887348730EE025B9012025
:103AA00011498873487308E000200F4988730CB1EE
:103AB000487302E001200C4948736DB186F00100A3
:103AC0000949887486F00100C87384F00100087405
:103AD00084F00100487405E0012003498874C8732C
:103AE00008744874BDE8F087D40C022010B5002398
:103AF0001A461946184609F0D7F81E23C8224FF473
:103B0000B971642008F0DCFF10BD70B504460D46A5
:103B100000231A461946184609F0C6F8B3EE0C2BD6
:103B200005F10E0000EE100AB8EEC01B04F10E0005
:103B300000EE100AB8EEC00B07F02CF970BD10B5FE
:103B4000022009F0D3F842233C223121FF2009F062
:103B5000ABF80A2332224FF4C371B62008F0B0FF4D
:103B600010BD10B500231A461946184609F09CF8F6
:103B70002823C822B421642008F0A2FF10BD10B58C
:103B800000231A461946184609F08EF81E23C8224B
:103B90004FF4B971642008F093FF10BD10B50023F5
:103BA0001A461946184609F07FF81E23C82200213C
:103BB000642008F085FF10BD10B500231A46194691
:103BC000184609F071F81E23C8220021642008F06D
:103BD00077FF10BD70B506460C461546304609F015
:103BE00085F800231A461946184609F05DF8642343
:103BF0008C222946204608F063FF70BD10B50320D3
:103C000009F074F800231A461946184609F04CF8D2
:103C100078231A468C21084608F052FF10BD10B5D3
:103C2000022009F063F842233C223121FF2009F0F1
:103C30003BF82D234FF48272FF21502008F040FF03
:103C400010BD70B56C24204604EBD0714910C1F151
:103C5000C805022009F04AF842233C223121FF2006
:103C600009F022F804F10C02A91F88B20E2340F2D9
:103C7000611108F025FF70BD10B500231A461946E2
:103C8000184609F011F846231A46A521084608F0FF
:103C900017FF10BD2DE9F04104460D4616461F469C
:103CA000DDF818802A480068204000284ED02948B6
:103CB000007800284AD0284800681CF05BFB2749A0
:103CC000098801EB4101264A42F831002348008867
:103CD00000EB4000114601EBC00044601F48008823
:103CE00000EB400001EBC00085601C48008800EB41
:103CF000400001EBC000C6601848008800EB40009F
:103D000001EBC00007611548008800EB400001EBA3
:103D1000C000C0F8148013480068401C11490860B6
:103D20000E480088401C0D49088008460088B0F500
:103D30007A7F01DB002008800B480088B0F57A7F8D
:103D400004DA09480088401C07490880BDE8F08172
:103D50001C1300202413002020130020181300201F
:103D6000F4270020141300201013002000207047B7
:103D700010B505481CF036FB0020044908800449B2
:103D800008600449088010BD201300201013002093
:103D9000141300201813002010B5044602481CF02C
:103DA00021FB0248047010BD2013002024130020C2
:103DB0002DE9F043D3B028F059FE012803D00120AB
:103DC00053B0BDE8F08300270026002477E03020C0
:103DD0008DF818013A208DF819016C208DF81A0120
:103DE0006F208DF81B0167208DF81C01B4F5803F12
:103DF00001DA302009E020140F2190FBF1F201FBE1
:103E0000120085B2284604F0BDFC8DF81D01B4F502
:103E1000805F01DA302009E020130F2190FBF1F2DE
:103E200001FB120085B2284604F0ACFC8DF81E019F
:103E3000FF2C01DC302009E020120F2190FBF1F271
:103E400001FB120085B2284604F09CFC8DF81F018E
:103E50000F2C01DC302009E020110F2190FBF1F242
:103E600001FB120085B2284604F08CFC8DF820017D
:103E70000F2094FBF0F100FB114085B2284604F0BE
:103E800081FC8DF821012E208DF8220174208DF8FF
:103E9000230178208DF8240174208DF8250100205D
:103EA0008DF8260146A828F0FDFC38B1641C701C72
:103EB00086B2B6F5803F02DB022081E70127002FA2
:103EC00085D046A828F07CFD8046314800683149FD
:103ED0000968CDE90010304803883048028830A1D5
:103EE00006A82FF06FF806A8FCF7D2F90546294678
:103EF00006A828F081FD002536E005EB450036498F
:103F000001EBC000406905EB4501334A02EBC101FA
:103F1000096905EB4502304B03EBC202D26805EBA1
:103F20004503DFF8B4C00CEBC3039B68CDE9013255
:103F3000CDE9031005EB4500614601EBC000406888
:103F4000009005EB450051F830302A4623A106A821
:103F50002FF038F806A8FCF79BF98146494606A8D9
:103F600028F04AFD681C85B20C4800888542C4DBF5
:103F700022A106A82FF026F806A8FCF789F9054625
:103F8000294606A828F038FD28F006FD002017E78E
:103F90001C130020141300201813002010130020FD
:103FA0004576656E74204C6F672028636F756E745C
:103FB0003D25642C2077726964783D25642C207738
:103FC00072697465733D25642C2066696C74657232
:103FD0003D2564290A000000F427002025642C20D8
:103FE00025642C2025642C2025642C2025642C207D
:103FF00025642C202564200A00000000456E642002
:104000006F66206C6F670A0010B50248008800F0E8
:104010000FF810BD1013002010B5642000F008F850
:1040200010BD10B54FF4FA7000F002F810BD00009A
:1040300010B504462848007800284AD1274800884F
:10404000A04218DC2548008800B225490880234892
:10405000008800B22349088020480088B0F57A7FA4
:1040600005DB2148008800B2204908801CE00020C0
:104070001E49088018E020B21949088020B2194969
:1040800008801948008816490988401A00B2174963
:1040900008800846B0F90000002805DA08460088C4
:1040A00000F57A7000B20880114800781149087054
:1040B00000F0C4F80120084908700A48B0F900204F
:1040C0000DA112482EF07EFF104826F057FA01206D
:1040D00010BD0020FCE70000251300201013002075
:1040E0002A1300202C13002018130020281300206E
:1040F00024130020261300205B4C6F6744756D70FD
:104100005374617274696E6725645D00B485002024
:1041100010B50948007860B10020074908700748C9
:10412000007808B100F084F805A026F027FA0120F5
:1041300010BD0020FCE700002513002026130020FE
:104140005B4C6F6744756D70436F6D706C65746523
:104150005D00000000B58DB025480078012845D1EC
:104160002448B0F90000002802DCFFF7D1FF3DE051
:104170002148B0F9000000EB4000204A02EBC001EA
:10418000182207A8FCF754F8DDE90923DDE90B1034
:10419000CDE90223CDE90410DDE90701CDE90001F5
:1041A0001748B0F900001349B1F90010421A144839
:1041B000B0F9003013A11A482EF004FF184826F079
:1041C000DDF90D480088401C00B20B490880084604
:1041D000B0F90000B0F57A7F01DB002008800548C7
:1041E0000088401E00B20349088000BF0DB000BD2A
:1041F000251300202C13002028130020F427002072
:104200002A1300205B25642C25642C25642C25644E
:104210002C25642C25642C25642C25645D0000006D
:10422000B485002001490860704700001C1300207D
:104230000120014908707047241300200020014923
:10424000087070472413002010B5FFF783FF10BDDE
:104250000F490978353903EE101AB8EEC33BB0EEBA
:10426000430B9FED0C3B80EE034BB0EE441B9FEDE8
:104270000B3B31EE033BB0EE432BB6EE003B32EE90
:10428000033BBCEEC33B13EE101A88B2704700002C
:104290005C13002033333333333303C0000000009A
:1042A00000405A4001480068704700005813002041
:1042B00001480068704700005413002000B5002238
:1042C00000BF1E48006840F002001C490860084614
:1042D000006800F002021A48006820F440501849B3
:1042E00008600846006840F480500860081D0068B7
:1042F00020F04000091D0860081D006820F44050AF
:10430000091D08600846006840F400500860081D58
:10431000006820F44050091D08600846006840F419
:104320008050086006482030006820F07060044922
:104330002031086000F066F800BD0000303802400F
:104340000004024070B52DED068B0446A4F169000F
:1043500000EE100AB8EEC00BB0EE409B9FED180BBC
:1043600029EE000BB0EE40AB9FED170B3AEE000BC1
:10437000B0EE408BB3EE040BB4EEC08BF1EE10FA4E
:1043800003D2B3EE040BB0EE408B9FED110BB4EEF5
:10439000C08BF1EE10FA03DD9FED0D0BB0EE408BFC
:1043A000B6EE000B38EE000BBCEEC00B10EE100AA0
:1043B00085B2E8B200F010F8BDEC068B70BD0000CD
:1043C00033333333333303C00000000000804A40EE
:1043D0000000000000206B4010B50446142C00DAE9
:1043E0001424D92C00DDD924044804700448007832
:1043F00018B102480078FDF7FFFA10BD5C130020E9
:10440000501300204FF48000024908600020024948
:1044100008707047180402405013002010B504487B
:104420000078FDF7E9FA01200249087010BD00008C
:104430005C130020501300202DE9F84F82460C46F3
:1044400016461F461648007808F050FC4FF0010849
:104450004FF00009E019801E05B21AE0721C91B2FB
:10446000A8B26A4608F0A8FB9DF80000FF280CD10E
:104470009DF80100E62808D19DF80200E62804D145
:104480009DF80300E62800D1C1444FEA4808681EA1
:1044900005B2601C8542E1DA4846BDE8F88F0000AD
:1044A00050170020014800787047000026180020AF
:1044B0001CB5FE480078012806D0FD480068019030
:1044C000BDF8041008461CBDFA480068002879D0E1
:1044D000002003460090F74804210268C801FFF756
:1044E000D9FBF5480068B0F80802C0F308000028BE
:1044F00069D1F1480068D0F8000290F80202401E2D
:10450000ED490968D1F8081200EA5120EB4908701A
:104510000846007800287DD1E7480068D0F80802F6
:1045200090B9E5480068D0F81002E54908600846EF
:10453000006828BBE0490968D1F8000200212FF08B
:10454000F9FFDF4908601BE0DB480068D0F824026F
:1045500050B1D9480068D0F80812D74800682FF049
:10456000B1FFD74908600BE0D34A1268D2F81412A1
:10457000D14A1268D2F800022FF0DCFFD04908605F
:10458000CF48006838B90020CA4908600090BDF8DB
:104590000010084697E7CA480068012814D1022095
:1045A000C549096881F807020120C6490880022030
:1045B000BE490870BE48001D00680090BDF800109C
:1045C000084680E7AEE148E1BD480068401C88B974
:1045D0000120B949096881F807020220B949088019
:1045E000B2490870B248083000680090BDF8001069
:1045F000084668E7B2480068AF490968C1F8140284
:10460000AD480068D0F8100220B9AD480068AA494A
:10461000096800E001E0C1F81002A748006890F8BE
:10462000060200F0400070B3002003460246052158
:1046300000904FF40070FFF72DFB9F490968D1F8F7
:1046400018229D490968D1F8001291F8010201234E
:104650009949096830F0F6FA0446ACB10120964950
:10466000096881F8070203209649088002208F49D3
:1046700008708F480C30006800908DF80140BDF83C
:10468000001008461FE70AE08B48006890F8060211
:1046900020F040008849096881F8060200BF864A78
:1046A0001268D2F81412844A1268D2F800022FF06D
:1046B00031FF854908600846006890B902207E49AC
:1046C000096881F8070203207E49088002207749A3
:1046D00008707748103000680090BDF80010084658
:1046E000F1E6794800687549097808447649086018
:1046F00070480068400A754908600846006800284C
:1047000071D06E480078096808446B490968D1F88F
:10471000001291F8021288420AD967480068D0F85E
:10472000000290F8020265490978401A674908605A
:10473000002003460246062100904FF40070FFF768
:10474000A9FA5D490968D1F8001291F801025F49A0
:104750000B685D490A685E49096830F073FA0446DF
:10476000A4B101205449096881F807020320554982
:10477000088002204D4908704D48143000680090B0
:104780008DF80140BDF8001008469CE64A480068D4
:10479000D0F818024C490968401A4C490968884207
:1047A0001AD245480068D0F81802474A1268801AA1
:1047B000474A126802EB40214FF400723E480068FD
:1047C00031F04BFE3C48006890F8060220F04000B3
:1047D0003949096881F806023C48006840023D49B1
:1047E000086080E0FFE734480068D0F818023649D6
:1047F000096888422BD030480068D0F808022E495A
:104800000968D1F80C12884220D22B490968D1F8E6
:10481000001291F8010201232B490A682649096810
:1048200030F0ACF990B101202349096881F8070202
:1048300003202449088002201C4908701C481830B5
:1048400000680090BDF8001008463CE600BF1E4816
:10485000006819490968C1F8180217480068B0F8DB
:104860000802C0F30800C0F500701A490860084645
:10487000006810490968884203D90E480068154944
:1048800008600D490968B1F80812C1F308010A4A25
:10489000126888180F490A680D49096831F0DDFD72
:1048A0000548006890F8060216E00000261800206F
:1048B000906F04082C1800203018002034180020B5
:1048C00038180020281800203C1800204418002028
:1048D000481800204018002040F04000284909688E
:1048E00081F8060200BF2748006827490968084484
:1048F0002449086022480068D0F808022249096863
:1049000008441F490968C1F80802204800681E4988
:104910000968401A1D49086000200190BDF8041084
:104920000846D0E516480068D0F80802144909681E
:10493000D1F80C12884207D911480068D0F8080253
:104940000F490968C1F80C020D48006890F806028A
:1049500040F020000A49096881F806020020034659
:104960000246032100904FF40070FFF793F90020F6
:10497000074908700190BDF804100846A3E500003F
:104980003018002048180020401800202C18002063
:10499000261800202DE9FC4104460D4616461F4608
:1049A0003648007838B1364800680190BDF80410E8
:1049B0000846BDE8FC8133480460334806600020A7
:1049C000034600903048002102684FF40070FFF762
:1049D00061F92E4805602E48076000202C490968BF
:1049E00008602848006831F0B2FF8046B8F1000F37
:1049F00009D02348001D006800908DF80180BDF8A3
:104A000000100846D5E71F48006890F8070268B113
:104A10001B480830006800901A48006890F80702A8
:104A20008DF80100BDF800100846C2E7154800687F
:104A300090F8060200F0020038B911480C30006806
:104A40000090BDF800100846B3E70E480068D0F8A3
:104A500008020D49096808440A490968D1F8081292
:104A6000884202D2002008490860012003490870EA
:104A700000200190BDF8041008469AE7261800208F
:104A8000806F0408301800202C18002048180020DF
:104A90004C18002010B50A48007880B10948006819
:104AA000382803D900200649087008E0054908782D
:104AB00000F082FA03480068401C0249086010BDFB
:104AC0003C13002038130020014800887047000084
:104AD0004013002001480088704700004213002066
:104AE00001480088704700003E13002001480088FC
:104AF00070470000441300202DE9FE43484B494A0B
:104B00004FF40051484821F063FC484B484A4FF4A9
:104B10000051484821F04AFC4FF00009464800681F
:104B200040F02000444908600846006800F0200971
:104B300041486030006820F400503F49603108600F
:104B40000846006840F4805008603B481030006818
:104B500040F080403849103108600846006800F095
:104B6000804902240025032600274FF008082B4621
:104B70002246C02131488DE8C00108F0E1F9600407
:104B80002F4908602F48006820F001002D49086077
:104B90004FF4D9602C4908602B480838006820F48D
:104BA00080402949083908600846006820F4006000
:104BB0000860081D006820F02000091D08600846F4
:104BC000006820F0080008600846006820F0020035
:104BD00008601D480C38006840F001001A490C3983
:104BE00008600846006840F00C000860084600684D
:104BF00040F0400008600846006840F0200008606F
:104C00000846006840F4807008600F48001F006884
:104C100040F001000C49091F0860BDE8FE83000058
:104C2000D4A60020D4860020B4860020D4E600203C
:104C3000D4C60020C4860020303802400014024050
:104C400008E100E0005000400C7800407047000090
:104C500038B52D480088401C2B4908802B48046833
:104C600004F0010040B101202849091D08602848CE
:104C70000088401C2649088004F0020040B1022050
:104C80002249091D086023480088401C21490880EA
:104C900004F0040040B104201C49091D08601E48AE
:104CA0000088401C1C49088004F0080040B108201E
:104CB0001649091D086019480088401C17490880DA
:104CC00004F0200040B1114808300068C5B2294600
:104CD000134821F0DBFB00BF04F0400090B14020FE
:104CE0000A49091D086069460E4821F09DFB28B15C
:104CF0009DF8000005490C31086002E000200A49D7
:104D0000087000BF38BD0000361300201C7800403A
:104D100046130020481300204A1300204C130020A3
:104D2000B4860020C48600203413002030B585B03E
:104D3000044622460BA168462EF044F96846FBF76C
:104D4000A7FA0546A9B2684624F02EFE7B2025F07E
:104D5000CFFAA9B2684625F0E1FA7D2025F0C8FA1D
:104D600005B030BD5220253032780D0001200349B6
:104D70000870002002490860704700003C130020C2
:104D8000381300203EB506A168462EF01BF9684690
:104D9000FBF77EFA0446A1B2684624F005FE3EBD4C
:104DA000572046462033310D000000003EB506A1D5
:104DB00068462EF007F96846FBF76AFA0446A1B286
:104DC000684624F0F1FD3EBD522030300D00000059
:104DD0003EB506A168462EF0F5F86846FBF758FA8E
:104DE0000446A1B2684624F0DFFD3EBD57203037AF
:104DF0002032360D0000000070B586B004460D4626
:104E00002B46224606A101A82EF0DCF801A8FBF7EC
:104E10003FFA0646B1B201A824F0C6FD06B070BD47
:104E200057202530326420253032640D0000000008
:104E300070B586B004460D462B4622460BA101A84C
:104E40002EF0C0F801A8FBF723FA0646B1B201A87C
:104E500024F0AAFD7B2025F04BFAB1B201A825F081
:104E60005DFA7D2025F044FA06B070BD572025304C
:104E7000327820253032780D000000002DE9FE4305
:104E80001348006840F001001149086008460068B6
:104E900000F0010901240025032601274FF0000836
:104EA0002B46224606210B488DE8C00108F048F841
:104EB00000F028F800F030F807481BF093FA0020C3
:104EC00006490870012006490870BDE8FE8300000D
:104ED0003038024000000240641300206C130020B0
:104EE0006013002001200149087070476C130020F6
:104EF0000348406940F002000149486170470000E2
:104F0000000002400348406920F002000149486166
:104F100070470000000002400348406940F0040070
:104F200001494861704700000000024003484069A1
:104F300020F0040001494861704700000000024071
:104F400010B51948007805282BD2DFE800F00304DB
:104F50000B1B290025E01548007810B102201249EA
:104F600008701EE0124800681BF004FAB0F57A7F62
:104F700007D9FFF7BDFF0F481BF034FA03200A4999
:104F800008700EE00B4800681BF0F4F940F6B831E9
:104F9000884204D9FFF7EAFE04200349087000E0C4
:104FA00000BF00BF10BD0000601300206C13002084
:104FB000641300206813002010B50446392C6ED20B
:104FC000DFE804F01D22272C31363B40454A4F5480
:104FD000595E63686E73787D82878C91969BA0A5DD
:104FE000AAAFB4B9BEC3C8CDD2D7DCF3F8FDEFEE9B
:104FF000EDECEBEAE9E8E7E6E5E4E3E2E1003121A4
:105000000020FFF7F9FE2BE150210220FFF7F4FE0C
:1050100026E160210D20FFF7EFFE21E161210F2045
:10502000FFF7EAFE1CE162213220FFF7E5FE17E1FF
:1050300063217D20FFF7E0FE12E164210846FFF7BF
:10504000DBFE0DE165217D20FFF7D6FE08E166213C
:10505000E620FFF7D1FE03E167210220FFF7CCFE37
:10506000FEE070210120FFF7C7FEF9E07121012069
:10507000FFF7C2FEF4E072210220FFF7BDFEEFE071
:1050800073212320FFF7B8FEEAE000210846FFF76E
:10509000B3FEE5E001213220FFF7AEFEE0E0DEE006
:1050A00002210720FFF7A8FEDAE00321D020FFF756
:1050B000A3FED5E004210520FFF79EFED0E00521E8
:1050C000DC20FFF799FECBE006210520FFF794FED8
:1050D000C6E00721DC20FFF78FFEC1E00821052094
:1050E000FFF78AFEBCE00921DC20FFF785FEB7E070
:1050F0000A210020FFF780FEB2E00B210420FFF719
:105100007BFEADE00C210020FFF776FEA8E00D212C
:105110000020FFF771FEA3E00E210020FFF76CFED8
:105120009EE00F210020FFF767FE99E0102100208C
:10513000FFF762FE94E011210020FFF75DFE8FE093
:1051400012210020FFF758FE8AE013210020FFF70C
:1051500053FE85E014210020FFF74EFE80E015216C
:105160000020FFF749FE7BE016210020FFF744FEF8
:1051700076E017210020FFF73FFE71E018210020A4
:10518000FFF73AFE6CE065E05FE059E053E04DE088
:1051900047E041E03BE035E02FE029E023E01DE07F
:1051A00017E011E00BE005E0FFE719210020FFF711
:1051B00023FE55E01A210420FFF71EFE50E01B21BC
:1051C0000020FFF719FE4BE01C210020FFF714FE22
:1051D00046E01D210020FFF70FFE41E01E210020C8
:1051E000FFF70AFE3CE01F210020FFF705FE37E035
:1051F00020210420FFF700FE32E021210020FFF7EC
:10520000FBFD2DE022210020FFF7F6FD28E0232101
:105210000020FFF7F1FD23E024210020FFF7ECFD43
:105220001EE025210120FFF7E7FD19E026210520DA
:10523000FFF7E2FD14E027210020FFF7DDFD0FE07E
:1052400028210020FFF7D8FD0AE0FE214820FFF7C3
:10525000D3FD05E0FF210020FFF7CEFD00E000BFF9
:1052600000BF10BD10B52A2001F022FB10BD10B503
:105270002C2001F01DFB10BD10B52B2001F018FBF8
:1052800010BD10B5252001F013FB10BD10B5262070
:1052900001F00EFB10BD10B5282001F009FB10BD78
:1052A00010B5044602480480292001F001FB10BD1E
:1052B000B413002010B5272001F0FAFA10BD000049
:1052C0002DE9F0412DED028B8EB005460C462CB930
:1052D000F7482946026800200DF04EFA44B9002034
:1052E00003460090F248294602680120FEF7D2FCEE
:1052F000032C0AD1EF48006840F28A21884204D288
:10530000EC480068401CEB490860284611F0B2F8F0
:10531000B8BB0FF059FB34280CD10FF0B5FA0B21B4
:1053200001EB0020E249086038200EB0BDEC028B92
:10533000BDE8F08116F0B0FF2E2808D116F0A6FFC8
:105340000C2101EB0020DA4908603820EDE71AF063
:105350009FFC332808D11AF069FC0D2101EB0020D5
:10536000D34908603820E0E718F010F9192809D16E
:1053700018F0F4F80E2101EB0020CD490860382028
:10538000D3E7FFE73C2D81F0E681DFE815F03C0034
:1053900042007B009C00DA000B012D0148015F01F7
:1053A000CC01E00111029202D70269037B039A0348
:1053B000F50300041804EA0136046B047404850440
:1053C000B504BF04E604EF04000530053F057B0586
:1053D0006F059B051D060D070E079207B2071608FD
:1053E000000863087E089308A808C308C408FF08DB
:1053F000420985092F0630064506640601079C0907
:105400009D099E09D509042C01D101208DE728466C
:105410008BE75CB9012024F06FFD022016F058FFE5
:1054200014F0C2F8A4481AF0DDFF29E0032C27D1BC
:10543000A14800681AF09EFF41F28831884201D9E4
:10544000012000E00020074614F090F8012801D068
:10545000012000E0002006460EB1FFF743FD17B122
:105460000EB1022061E7944800681AF083FF934967
:10547000884204D90F208E490860382055E700BFC4
:10548000284652E78CB924F09CFA8D481AF0AAFFFE
:1054900000201EF06BFA064636B1102000EB062005
:1054A00083490860382040E70BE0032C09D1844889
:1054B00000681AF05FFF40F6C411884201D903204A
:1054C00033E7284631E764B910F07CF90646012E2F
:1054D00006D0112000EB062075490860382024E72B
:1054E0002DE0032C2BD10FF06FFA06460C2E01D1C4
:1054F00004201AE70B2E08D10FF0C6F96C4908609A
:1055000001207049087004200FE7342E08D10FF0F5
:10551000BBF9122101EB002065490860382004E73F
:10552000654800681AF026FF6749884206D91320AB
:1055300000EB06205E4908603820F6E600BF2846EA
:10554000F3E654B900206149087027F041FEFEF7E8
:1055500065FF64205E49087022E0032C20D15C487E
:105560000078401E5A49087014F000F8022801D053
:10557000012000E0002006465548007800280EDC97
:105580002DF028FC0120534908701EB952490870BB
:1055900013F0E6FF0120514908700620C5E600BF60
:1055A0002846C2E61CB94E481AF01CFF1AE0032C2C
:1055B00018D14CF250361AF095FB08B90620B4E623
:1055C000474800681AF0D6FE4CF25031884208D99C
:1055D0001AF05EFB142101EB0020354908603820E9
:1055E000A3E600BF2846A0E6BCB1032C15D1324883
:1055F00000681AF0BFFE46F2A81188420DD9FCF7E8
:10560000A7F93048007808B107208EE60FF05AFD60
:1056100008B1092089E60A2087E6284685E624B9EC
:105620002348006824F09FFC0EE00E2C08D120488F
:105630000068152101EB00201D490860382074E640
:105640000D2C01D1082070E628466EE6D4B9254815
:105650001AF0C8FE10F008F90646022E08D10FF025
:10566000B3F9162101EB00201149086038205CE6EF
:10567000012E06D0172000EB06200D4908603820C7
:1056800053E64EE0032C4CD10FF09EF906460C2E4B
:1056900003D118F044F90A2047E6342E24D10FF044
:1056A000F3F8182101EB00200149086038203CE69E
:1056B00074130020801300208C130020A0860100AA
:1056C00098130020A4130020400D0300A513002010
:1056D000A0130020A2130020A3130020A113002078
:1056E000A8130020881300200B2E08D10FF0CCF84F
:1056F000192101EB0020F7490860382015E6F6482B
:1057000000681AF037FE4CF25031884208D90FF089
:105710005BF91A2101EB0020EE490860382004E60D
:1057200000BF284601E62CB9ECA2F0A1F2A024F0BB
:1057300009FC0AE00F2C01D10A20F6E5032C04D164
:10574000FBF7CEFC08B10A20EFE52846EDE534B9B9
:10575000EB48007808B11320E7E50B20E5E5284683
:10576000E3E574B927F034FD0020E6490870DA4813
:105770001AF038FE032024F0BFFB022016F0A8FD2B
:1057800014E0032C12D1D44800681AF0F3FD064649
:1057900042F21070864208D9142D06D1DA480078FA
:1057A00008B10D20C1E50B20BFE500BF2846BCE5D0
:1057B00094B90020D4490870FEF730FE21F074FD42
:1057C0000EF0DEFC064628F01DFF032024F094FBBB
:1057D000042016F07DFD6AE0132C01D11520A4E50C
:1057E000142C04D10020C94908701A209DE5172CFB
:1057F00004D10120C44908700D2096E5262C04D15F
:105800000120C14908700D208FE5032C33D113F01E
:10581000ADFE052803D013F0A9FE062817D121F00C
:1058200051FD10B121F02CFD04E024F061FA08B123
:1058300024F0C5FB13F09AFE052802D0062804D1F7
:1058400001E0122071E513206FE500BF00BFFBF7F8
:1058500035FC60B321F036FD10B121F011FD26E0DA
:1058600024F046FA10B124F0AAFB20E0FBF7A4FED6
:10587000E8B90C2059E5272C01D10C2055E5122C54
:1058800001D1212051E5212C01D121204DE5242CED
:1058900001D13B2049E52B2C01D1252045E52C2CBD
:1058A00001D1242041E52D2C01D101203DE52846E0
:1058B0003BE574B921F0EEFC87481AF093FD022213
:1058C0004FF47A7141F2883024F0F7F816F0FAFCC0
:1058D00032E0032C30D141F270777F4800681AF033
:1058E00049FD06463846864225D916F0E5FC20B12A
:1058F0000120874908700B2017E516F0CDFC2E28F3
:1059000008D116F0C3FC1B2101EB0020714908608F
:1059100038200AE5704800681AF02CFD4CF250312E
:10592000884208D916F0B8FC1C2101EB0020694917
:1059300008603820F9E400BF2846F6E4ACB900203E
:105940007449087001207049087021F0ADFCFEF721
:1059500065FD0EF015FC064628F054FE032024F0E9
:10596000CBFA042016F0B4FC78E0132C01D11520FA
:10597000DBE4142C04D10020644908701A20D4E41C
:10598000122C01D12120D0E4212C01D12120CCE402
:10599000172C04D100205C4908700B20C5E4252C8D
:1059A00004D10020584908700B20BEE4282C04D1F3
:1059B0000020594908700E20B7E4292C08D1012095
:1059C0005549087055480088554908800E20ACE4B8
:1059D0002B2C01D12520A8E42C2C01D12420A4E4D7
:1059E000242C01D13B20A0E42D2C01D101209CE4EA
:1059F000032C33D113F0BAFD052803D013F0B6FD04
:105A0000062817D121F05EFC10B121F039FC04E02A
:105A100024F06EF908B124F0D2FA13F0A7FD05289E
:105A200002D0062804D101E012207EE413207CE499
:105A300000BF00BFFBF742FB80B121F043FC10B177
:105A400021F01EFC0AE024F053F910B124F0B7FA5B
:105A500004E0FBF7B1FD08B9102066E4284664E4D1
:105A600074B921F017FC032016F032FC032024F057
:105A700043FA0FF001FB08B1102056E40F2054E464
:105A8000284652E41CB927481AF0ACFC17E0032C56
:105A900015D10FF0F1FA08B1102046E42148006852
:105AA0001AF068FC41F28831884208D90EF08CFF68
:105AB0003C2101EB002007490860382035E42846E6
:105AC00033E41CB9052016F003FC53E02A2C2BD13B
:105AD00011202AE474130020881300205441502020
:105AE000544F20434F4E54494E554500302E3031CF
:105AF0002E3039310000000056455253494F4E00B8
:105B0000A3130020A513002094130020AD13002040
:105B1000A1130020AC130020B8130020B413002000
:105B2000B6130020B0130020032C23D113F01EFD68
:105B3000052803D013F01AFD062801D1112005E431
:105B40000FF0B4FA08B111200DE4FC48007838B128
:105B50000EF00CFFFA490988884201DB11200FE49E
:105B6000FBF72AFD08B111200AE4FBF7A7FA08B1F8
:105B7000112005E4284649E43CB9042016F0A8FBAE
:105B80000120F04908700D2040E428463EE444B965
:105B9000FEF738FC032024F0AFF9012016F098FB43
:105BA0000BE0032C09D113F0E1FC062805D10020FD
:105BB00016F08EFB0020FCF716FB284626E444B9BD
:105BC000FEF720FC0020FCF70EFB002016F080FB07
:105BD00011E0032C0FD1DC48007801280BD113F021
:105BE000C5FC052807D127F0F3FA0020D649087034
:105BF000FF20FCF7F8FA284608E46CB921F04AFBCC
:105C00000EF0BEFA064629F0ABFD012016F060FB4F
:105C1000042024F071F923E0032C1DD113F0A6FC1D
:105C200003280AD013F0A2FC042806D114F018FEB1
:105C300018B924F0C4F9162014E424F063F808B16C
:105C400017200FE4FBF74CFA50B124F045F838B1B7
:105C500024F0B5F9162005E4192C01D117200DE424
:105C600028460BE4032C04D124F04CF808B117208B
:105C700004E4284605E46CB929F0E2F906460EF082
:105C80007FFAB04204D030460EF084FA18200AE4BD
:105C9000192008E4284606E49CB90EF081FA06466D
:105CA000012E0AD0002033461722092100904FF41C
:105CB0008030FDF7EFFF192004E4A4481AF092FBAE
:105CC00018E0032C16D10EF07FFE0C2801D119200C
:105CD00005E49E4800681AF04DFB44F620618842B6
:105CE00008D90EF071FE1D2101EB002098490860D3
:105CF000382009E4284607E434B99648007808B10A
:105D00000D200CE40B200AE4284608E474B921F0C5
:105D1000C1FA012016F0DCFA0EF026FA06463046EB
:105D20002AF010FA052024F0E7F814E0032C0ED135
:105D300023F0B6FF08B11C2030E4FBF7D1F950B1D5
:105D400023F0A2FF38B124F02EF91B2026E41A2CF0
:105D500001D11C2022E4284620E4032C04D123F0A6
:105D60009FFF08B11C2019E4284617E46CB929F0FC
:105D70007BFF06460EF0F8F9B04204D030460EF034
:105D8000F9F91D200AE41E2008E4284606E49CB91F
:105D90000EF006FA0646012E0AD0002033461722DE
:105DA000092100904FF48030FDF774FF1E2006E4B7
:105DB00066481AF017FB18E0032C16D10EF004FE0B
:105DC0000C2801D11E200BE4604800681AF0D2FABA
:105DD00044F62061884208D90EF0F6FD1E2101EB41
:105DE00000205B49086038200FE428460DE45CB9C8
:105DF0005948007830B95748007808B10D2004E4BC
:105E00000B2007E4202005E4284605E46CB921F0C6
:105E100041FA01204C49087027F0E0F9022016F001
:105E200057FA062024F068F81EE0032C0DD11F2D30
:105E30001AD113F09BFB052801D1122005E413F0C1
:105E400095FB062810D1132011E41B2C0CD13E48E1
:105E50000078012801D1142009E43E48007808B1F7
:105E60000D2004E40B200BE4284609E444B935482E
:105E7000007818B916F020FD17F04AFD20200BE439
:105E8000284609E4E4B92F48007830B100202D49B4
:105E9000087016F011FD17F042FDFEF7B3FA21F07D
:105EA00003FA072024F028F824F01EF80EF068F911
:105EB00006462CF099FE022016F00AFA22201DE474
:105EC00028461BE41CB925481AF08CFA7AE0152CF8
:105ED00001D1332012E4162C04D101201E49087090
:105EE0001A200BE4222C01D1342007E41D2C01D10F
:105EF000212014E4202C01D1232010E42B2C01D1EB
:105F000025200CE42C2C01D1242008E4032C59D1A9
:105F100027F0AEF888B112480078032822DA10483A
:105F20000078401C0E49087027F052F927F00EF84F
:105F300027F08EF927F052F92AE022E0B81300206A
:105F4000B6130020A1130020A5130020B0130020D9
:105F50007413002094130020AD1300208813002038
:105F6000B913002014F076FC0020FD49087027F0DA
:105F70002FF926F0EBFF27F06BF90020F9490870A4
:105F800006E026F073FD012802D10020F5490870D3
:105F900013F0ECFA052801D1122005E413F0E6FA1B
:105FA000062801D113201AE4FBF79AF820B121F05A
:105FB00089F910B121F064F904E023F08FFD08B9EC
:105FC00023200CE428460AE474B913F0E1FBE4480A
:105FD0000078012801D1142008E4E348007808B1D2
:105FE0000D200AE40B2008E4284606E400BF8CB923
:105FF000012016F06DF921F04DF923F0CCFF342D7E
:1060000001D123F0D8FF0FF037F808B1362019E49A
:10601000362017E4284615E41CB9D4481AF0E2F9F2
:1060200017E0032C15D10FF027F808B1362009E44A
:10603000CE4800681AF09EF94EF66021884208D9D1
:106040000EF0C2FC332101EB0020C9490860382062
:1060500010E428460EE4ECB3012C03D10020C5491E
:10606000087093E0232C03D123F0A1FF372005E42F
:10607000032C61D123F02CFE08B1202006E4FBF7AD
:106080002FF830B123F018FE18B123F090FF37201D
:1060900004E4B94800681AF06DF94CF250318842B6
:1060A00013D9AF48007880B9B248007868B913F0C6
:1060B0005DFA032809D123F0FFFD30B10120AD497D
:1060C0000870A749087027F089F826F0D1FFD0B1F1
:1060D000A44800E059E0007803280DDAA1480078D0
:1060E000401CA049087027F073F826F02FFF27F016
:1060F000AFF827F073F80DE023F0DEFD50B123F088
:1061000056FF372005E426F0B1FC012802D100201B
:106110009449087013F02AFA032837D013F026FAAE
:10612000042833D114F09CFB78BB23F0C5FD60B389
:1061300023F03DFF37201BE4062C01D1242017E477
:10614000052C01D1252013E4072C01D12E200FE4CA
:10615000082C01D12F200BE40A2C01D1302007E4B8
:10616000092C01D131200AE40C2C0FD01C2C0DD1AC
:106170007B480078012801D1142004E47A48007893
:1061800008B10D200AE40B2008E4FFE7284605E4E7
:10619000032C07D123F09CFD20B100207549087025
:1061A000202009E4284607E400BF44BB21F072F830
:1061B00021F00CF8242D05D10EF0CCFB064621F081
:1061C00049F804E00EF05AFB064621F043F820F0AF
:1061D000A5FF064620F09CFF0746314623F07CFED3
:1061E0009FED660B23F0C8FE012016F071F8242DF8
:1061F00002D120F0F5FF5AE021F004F857E0102C0E
:1062000003D121F031F828200FE4032C4FD113F0F3
:10621000ADF9042803D121F027F8282005E413F074
:10622000A5F9052803D121F01FF8122015E413F079
:106230009DF9062803D121F017F813200DE420F072
:10624000ABFF0646022E01D1262006E4032E01D123
:106250002A2004E4052E01D12C200EE4042E0BD1BB
:1062600020F050FF47490880084600888C2801D15B
:106270002B2004E42D2004E41F2E08D120F042FF3F
:10628000322101EB00203A490860382005E420F073
:106290004BFFB0EE408B23F06FFE20F03FFF074630
:1062A00020F036FF8046394623F016FE00BF284610
:1062B00004E484B9B7EE000B23F05EFE20F02EFF5D
:1062C000064620F025FF0746314623F005FE2A4802
:1062D0001AF088F80BE0032C09D1274800681AF05F
:1062E00049F842F21071884201D9272027E4284654
:1062F00025E47CB920481AF075F80DF0E9FE064651
:10630000012E06D0202000EB062019490860382015
:1063100015E43AE0032C38D10EF056FB06460C2E5D
:1063200001D129200BE4342E08D10EF0ADFA212141
:1063300001EB00200E490860382005E40E48006893
:106340001AF018F84EF6602188421DD90EF03CFB79
:10635000222101EB002006490860382004E40000F7
:10636000A5130020B913002094130020B0130020BF
:1063700074130020AC1300208813002000000000DC
:10638000000000009013002000BF284616E43CB92E
:10639000AFF6A002AFF6BC01F2A023F0D3FD0AE0F5
:1063A000032C04D1FAF79CFE28B1202006E40F2C20
:1063B00001D1202020E428461EE444B9ED481AF01B
:1063C00011F8EBA2EAA1ECA023F0BCFD40E0032C05
:1063D0003ED120F08BFE074617B1E6481AF002F8CE
:1063E00020F0DAFE0646022E01D0032E01D12A202B
:1063F00022E4052E01D12C201EE4042E0BD120F026
:1064000081FEE0490880084600888C2801D12B20B5
:1064100012E42D2010E41F2E08D120F073FE23215A
:1064200001EB0020D8490860382005E4D148006815
:1064300019F0A0FF49F64041884208D920F0ACFE8F
:10644000242101EB0020D0490860382007E400BF78
:10645000284604E464B913F089F8032801D026F033
:10646000B7FEC3A2AFF68C11C8A023F06BFD0AE003
:10647000032C04D1FAF734FE28B1202007E40F2CB6
:1064800001D1202005E4284605E434B9AFF6B41262
:10649000C2A1C5A023F056FD0AE0032C04D1FAF7EF
:1064A0001FFE28B1202007E40F2C01D120200FE48B
:1064B00028460DE434B9AEA2AFF6E011BCA023F03B
:1064C00041FD0AE0032C04D1FAF70AFE28B120208E
:1064D0000FE40F2C01D120200BE4284609E464B915
:1064E000A8480288B5A101A82CF06CFDA0A2AFF6C7
:1064F0001421B3A023F026FD0AE0032C04D1FAF7FF
:10650000EFFD28B1202017E40F2C01D1202013E447
:10651000284611E400BF74B923F0EAFCAB4819F037
:1065200061FF2E2D02D10DF0C7FD2DE02F2D2BD1B7
:106530000DF0CEFD28E0032C26D10EF045FA0646DC
:106540000C2E04D10120A2490870202004E4342E2E
:1065500008D10EF099F9252101EB00208A49086045
:1065600038200FE49948006819F004FF4EF66021C6
:10657000884208D90EF028FA262101EB0020824932
:106580000860382013E400BF284610E48CB923F0DB
:10659000AFFC8E4819F026FF0DF0A6FD0646012E31
:1065A00006D0272000EB06207749086038200AE44F
:1065B0002DE0032C2BD18548006819F0DBFE44F652
:1065C0002061884223D90EF0FFF906460C2E01D136
:1065D000322009E4342E08D10EF056F9282101EBBF
:1065E000002069490860382009E47848006819F0FB
:1065F000C1FE4EF66021884208D90EF0E5F9292146
:1066000001EB002060490860382017E400BF2846ED
:1066100014E48CB923F06CFC6C4819F0E3FE0DF027
:10662000DFFD0646012E06D02A2000EB0620564943
:106630000860382008E42DE0032C2BD16348006863
:1066400019F098FE44F62061884223D90EF0BCF977
:1066500006460C2E01D1322005E4342E08D10EF06E
:1066600013F92B2101EB002047490860382006E48C
:106670005648006819F07EFE4EF66021884208D91F
:106680000EF0A2F92C2101EB00203F4908603820D0
:1066900015E400BF284612E444B901204C490870B3
:1066A00033A233A14BA023F04DFC0AE0032C04D10C
:1066B000FAF716FD28B120200CE40F2C01D1202080
:1066C00008E4284606E400BF00BF64B9012043493E
:1066D000087026F083FD00204149088020F0E4FD89
:1066E000FDF7ACFD26E0032C23D13D48B0F90000B6
:1066F000002806DD3A480088401E00B2384908806C
:106700000EE0322036490880FDF77CFE012015F0AE
:10671000DFFD0D2023F0F0FB1B48006823F0D6FBC3
:10672000FAF7CCFC30B120F0CDFD18B120F0A8FD77
:1067300000E000BF284630E454B920F0ABFD012052
:1067400015F0C6FD0AA20AA126A023F0FBFB00E07B
:1067500000BF284621E4FE2000EB05200A4908601E
:1067600038201AE4494D414745532053415645448A
:10677000000000009C13002053544F5050494E47D6
:106780000000000090130020741300205341564570
:106790002043414E43454C4C45440000415641493D
:1067A0004C41424C45000000555342204E4F54008E
:1067B0005553422046554C4C000000002564000013
:1067C00053415645204641494C454400881300201A
:1067D000A11300205355434345535300A5130020F4
:1067E00092130020544553540000000001480068F3
:1067F00070470000741300200148007870470000C3
:10680000701300200148007870470000A213002098
:1068100010B5002005490870054823F0AFFA054877
:106820000EF084FF042000F043F810BD7013002028
:1068300085A30208C7A1020801480078704700003C
:10684000941300200C4800780E2801D101207047D5
:10685000094800780F2801D10120F8E706480078A0
:10686000102801D10120F2E703480078112801D156
:106870000120ECE70020EAE77013002010B521208A
:1068800000F016F810BD10B5242000F011F810BD6E
:1068900010B5232000F00CF810BD10B5202000F03A
:1068A00007F810BD10B5222000F002F810BD00005E
:1068B0002DE9F04780462048077841463846FEF7E4
:1068C000FFFC04464FF00009A74201D1012000E07F
:1068D0000020824629E009F101000FFA80F9B9F1A0
:1068E000C80F0BDD40F2E730144908603920124927
:1068F00008700021FEF7E4FCBDE8F087012138466E
:10690000FEF7DEFC0546BD4200D02C4600212046A5
:10691000FEF7D6FC0646A64202D14FF0010A03E07C
:10692000274634464FF0000A00BFBAF1000FD2D01C
:106930000148047000BFDFE77013002074130020CB
:1069400010B50120024908701D20FFF7B1FF10BDEE
:10695000A113002010B52D20FFF7AAFF10BD0000E5
:1069600010B504480068401C024908600320FFF786
:106970009FFF10BD7C13002070B5044616492046C9
:1069800026F0E4FD28B31548007805280BD1FBF765
:1069900067FC054610490888294619F0F9FA0420D1
:1069A0000E4908700AE0FBF75FFC05460A490888B3
:1069B000294619F0EDFA05200849087008480480B6
:1069C00000EE104AB8EE400B064880ED000B0120A7
:1069D00070BD0020FCE700008E6A012059150020E0
:1069E0005A150020601500200C490988491E0C4AE0
:1069F0001288914202DC042101700EE00121094A53
:106A0000117007490988491C00EE101AB8EEC00B36
:106A1000054981ED000B00210170704752150020DF
:106A20005415002068150020701500200B490988B6
:106A3000002902DC032101700EE00121084A1170D7
:106A400006490988491E00EE101AB8EEC00B054928
:106A500081ED000B002101707047000054150020EB
:106A6000681500207015002003B5ADF5097D8A98E2
:106A700048BB8998032811D0252819D1F748808868
:106A80000090F64840888790F44800888690024637
:106A90000420879B8999FDF7FDF813E00020034649
:106AA0000090EF48027804208999FDF7F3F809E097
:106AB000002003460090EB48026804208999FDF706
:106AC000E9F800BF00BF8998352881F0EB85DFE841
:106AD00010F0350044004E00A000BB00BC00D60002
:106AE0002501380178018F01AC0D0502050651051D
:106AF000CF0501074A085308A308B908CF0833098E
:106B00004A09700979092808020D210D800D960D9A
:106B10004107520774079807270528059D09A8090A
:106B2000100B240B490BBE0BD20BE90B030C760C9C
:106B30008A0CE80CAA04B5040405D50D8A9804282B
:106B400009D1C9481DF0A0FAC8481DF0B5FA0120C6
:106B50000DF50B7D00BD8998FAE78A98052804D1C8
:106B60000120C34908700220F2E78998F0E78A986B
:106B700068B90020879087AB40F259720021BD4868
:106B800000681DF02BFA1420BB4908803FE08A986A
:106B90000A281ED1B74800680068B849884210D159
:106BA0000020B7490870B348006890F8000418B195
:106BB0000020AB49087002E00120A94908700320B9
:106BC000C6E70120AE4908700220AE4908800420C3
:106BD000BEE78A980B2808D10DF056FE662101EB1E
:106BE0000020A04908600B20B2E78A9802280ED145
:106BF000A1480088002805DD9F480088401E9E4966
:106C0000088004E06720974908600B20A0E7899876
:106C10009EE78A98B0B9FAF701FF86A819F0FCFB45
:106C20009DF8180248B9BDF91A02BDF91C1200EB13
:106C300001208C4908600B208AE7012091490880D7
:106C40000C2085E7899883E700BF8A98A8B90DF0E2
:106C500021FE002801DD012000E000208A490870A3
:106C60008998052804D100201BF0FCFD08206FE75F
:106C700001201BF0F7FD06206AE7899868E78A98EB
:106C800010BB824819F0AEFB0020879087AB012231
:106C900011467848006800F500701DF015FB8690DD
:106CA0000020034600909DF81C2208214803FCF7B1
:106CB000F1FF869838B13C21869801EB00206949A4
:106CC0000860342044E727E08A98072800D13FE78E
:106CD0008A98082804D17820624908600B2037E799
:106CE0008A98092804D179205E4908600B202FE793
:106CF0008A98032810D16548006819F03BFB44F6D8
:106D00002061884208D90DF05FFE7A2101EB002056
:106D1000544908600B201BE7899819E78A9818B92D
:106D20005A4819F05FFB0AE08A98032807D15748B0
:106D3000006819F01FFB642801D9082008E789982A
:106D400006E78A98E0B932204B4908804FF4EB609F
:106D500087900020869086AB02214648879A00687B
:106D600000F580601DF0B0FA8590859838B17B21E0
:106D7000859801EB00203B4908600B20E8E61EE007
:106D80008A98072801D10920E2E68A98082804D1C8
:106D90007C20344908600B20DAE68A9802280ED15C
:106DA00035480088002805DD33480088401E3249F8
:106DB000088004E07D202B4908600B20C8E68998F4
:106DC000C6E68A9818B902202B4908800EE08A98F6
:106DD00002280BD128480088002805DD26480088B5
:106DE000401E2549088001E00A20B1E68998AFE6F7
:106DF0008A98B8B90020879087AB012200211D48EE
:106E000000681DF061FA8690869838B17E218698D8
:106E100001EB0020134908600B2099E63220164947
:106E2000088059E08A9807283CD10020184908803A
:106E30001849088018490880184908800021184816
:106E400001801148007830B100200F4908700021FE
:106E50000846FCF72BFC0C207AE60000AC59012018
:106E60003D140020701400204924020871240208F7
:106E7000761400209C14002074140020CDDBCDDBA0
:106E80003C140020781400204B140020941400209F
:106E90003E1400204014002044140020421400201E
:106EA000461400208A98082804D17F20F8490860F9
:106EB0000B204DE68A9802280ED1F648008800285B
:106EC00005DDF4480088401EF249088004E0802077
:106ED000EF4908600B203BE6899839E68A9800283C
:106EE00010D08A98212804D10120EB490870312064
:106EF0002EE68A981B282BD1E848007818B1042088
:106F0000E54908708DE2E64800884EF66021884227
:106F100003DB0520E049087083E206F0B5FC8790AA
:106F20009DF81C0202468490DD48018885A807F080
:106F30005DF8BDF81402C0F3801018B90620D649D8
:106F4000087004E00120D44908701A2000E668E2C5
:106F50008A981D280BD1D148007818B10420CE4959
:106F600008705EE20120CC4908702320F0E58A9881
:106F70001E280BD1C948007818B10420C6490870F2
:106F80004FE20120C44908702420E1E58A981C28BA
:106F900035D1C248007818B10420BF49087040E2DA
:106FA000BF4800884EF66021884203DB0520BA49BD
:106FB000087036E206F068FC87909DF81C020246D5
:106FC0008490B748018885A807F010F8BDF814022E
:106FD000C0F3801018B90620AF4908700EE0BDF864
:106FE0001A024FF6FF71884203D10720AA490870A0
:106FF00004E00120A84908701B20A9E511E28A9845
:107000000E280BD1A548007820B90120A2490870AC
:107010000E209DE50420A049087002E28A980F28FE
:1070200052D19E48007818B10E209B490870F8E1B3
:1070300001209A49087000209A4908809A480068FF
:1070400000F5C0609949097800EB412040894FF66E
:10705000FF71884228D19448006800F5C0609349C8
:10706000097800EB412000884EF6602188420FDA53
:107070008D48006800F5C0608C49097800EB41201C
:107080000088322101EB00208149086034205FE54F
:107090008548006800F5C0608449097800EB41200C
:1070A0004088834908800AE07F48006800F5C06096
:1070B0007E49097800EB412040897D490880012004
:1070C000754908700C2043E58A98102826D173482A
:1070D000007820B90820704908700C2038E5714804
:1070E000008841F29411884204DB0F206A4908703D
:1070F0000C202DE56E4800886E49088008460088FF
:107100004EF66021884204DB032061490860342088
:107110001EE50120604908700D2019E58A981128A4
:1071200019D15E48007890B15E48008838B90020D7
:107130005A4908700120584908700C2008E50020C1
:1071400056490870012054490870102000E50820B5
:107150005149087065E18A9812283BD14F48007860
:1071600018B104204C4908705BE10DF073FF18B1B1
:1071700003204949087054E106F086FB87909DF88A
:107180001C02024684904648018885A806F02EFF1E
:10719000BDF81402C0F3801018B906203E490870EB
:1071A00017E0BDF81402C0F3401018B90A203A499C
:1071B00008700EE0BDF81A024FF6FF71884203D046
:1071C0000C203549087004E0012033490870112073
:1071D000BEE426E18A98132834D13048007818B1EB
:1071E00004202D4908701CE106F04EFB87909DF8A5
:1071F0001C02024684902A48018885A806F0F6FE03
:10720000BDF81402C0F3801018B906202249087096
:1072100017E0BDF81402C0F3401018B90A201E4947
:1072200008700EE0BDF81A024FF6FF71884203D1D4
:107230000B201949087004E0012017490870182034
:1072400086E4EEE08A9814280FD10DF023FB002885
:1072500007DD00201149087001200F490870042043
:1072600076E401200C490870DBE08A98152823D1C8
:107270000DF010FB002807DD0020084908700120F0
:1072800005490870052063E4012003490870C8E03F
:107290007014002074140020761400208014002044
:1072A00064140020821400209C1400203D1400204F
:1072B000841400205C1400208A9816282BD1F848EA
:1072C000007818B10420F7490870AAE006F0DCFA4B
:1072D00087909DF81C0202468490F348018885A897
:1072E00006F084FEBDF81402C0F3801018B9062021
:1072F000EC4908700EE0BDF81402C0F3401020B94C
:107300000120E84908701F2022E40120E5490870A7
:1073100021201DE485E08A98172821D1E0480078D3
:1073200018B10420DF4908707BE006F0ADFA8790C1
:107330009DF81C0202468490DB48018885A806F06F
:1073400055FEBDF81402C0F3801018B90620D549C7
:10735000087004E00120D34908701F2004E460E0B5
:107360008A9818282AD1CE48007818B10420CD492F
:10737000087056E006F088FA87909DF81C020246D5
:107380008490C948018885A806F030FEBDF8140233
:10739000C0F3801018B90620C24908700DE0BDF88E
:1073A0001402C0F3401018B90A20BE49087004E066
:1073B0000120BC49087021200AE432E08A9819288B
:1073C00007D10120B74908700DF058FA48B32220C0
:1073D0000AE48A981A2801D11C2005E48A982028FA
:1073E00004D10120AF49087025200FE48A980628AF
:1073F00003D10120AB49087008E48A981F2810D1F6
:107400000120A8490870A9490870A9490870A9482D
:1074100012F04FFA0FF0A2FBA64811F081FD2520D3
:107420000AE4899808E48A9830B9FAF707FB0A2039
:10743000A1490880322004E4899804E48A9810BBAA
:107440009E4818F0CFFF0020879087AB012211469D
:107450009B48006800F500701CF036FF8690002005
:10746000034600909DF81C2208214803FCF712FCFB
:10747000869838B13C21869801EB00219148016043
:1074800034201FE427E08A98072805D10021032033
:10749000FCF70CF90C2015E48A98082805D1012185
:1074A0000420FCF703F90C200CE48A98092801D188
:1074B000332007E48A9803280DD18048006818F02B
:1074C00059FF44F62061884205D902210420FCF7C7
:1074D000EDF80C200BE4899809E48A9818B97A48E9
:1074E00018F080FF1AE08A98032817D176480068C0
:1074F00018F040FFB0F57A7F10D96F480088002857
:1075000006DD6D480088401E6B490880322004E487
:1075100003210420FCF7CAF80C200FE489980DE43D
:1075200000BF8A9820BB654818F05CFF614812F0E4
:1075300096F90FF013FB8998232801D1012000E070
:107540000020879001225B49879811F00BFD8690FF
:107550008698012807D03221869801EB00215948EE
:10756000016034200AE4534811F0DAFC252005E4D8
:10757000899809E48A9890BB3221544801800120FF
:1075800053490870494908704A4812F068F90FF0E9
:10759000E5FA0DF05FFD78B10121464810F08EFE4E
:1075A00088908898012807D00421889801EB002151
:1075B00044480160342018E40020879001223D49AE
:1075C00087A80FF09FF888908898012808D0052197
:1075D000889801EB00203B490860342005E422E054
:1075E000344811F09DFCBDF81C0240F2D51148430F
:1075F00040F2627101EB400086900020859085ABDF
:1076000040F2AA323348869900681CF05DFE8490EF
:10761000849838B10621849801EB0020294908603C
:10762000342019E422E08A98072801D10F2013E4BE
:107630008A98082804D107202249086034200BE4E6
:107640008A98022812D121480088002805DD1F48A9
:107650000088401E1D49088008E01BF0F5FC082149
:1076600001EB002017490860342022E4899820E4C7
:107670008A9818B9184818F0B5FE0EE08A980328C1
:107680000BD11548006818F075FE87908798B0F503
:107690007A7F01D925200CE400BF899809E4000015
:1076A0008014002076140020641400204A14002066
:1076B00049140020AC5901205414002094140020D7
:1076C0009C140020701400209814002074140020D2
:1076D00048140020581400207C1400208A98B8BB5D
:1076E000F848008840F2D511484340F2627101EB3E
:1076F000400087900020869086AB40F2AA32F24884
:10770000879900681CF0E0FD8590859808B3EF48E4
:107710000088401CED490880084600880F2808DDD5
:107720009DF81802092101EB0020E9490860342086
:107730000CE4E84985980880E7480088401CE64941
:107740000880E6480088401CE44908800C200DE4CD
:1077500006E00020DD4908803221E1480180B7E0E1
:107760008A9807287DD1DF480088401CDD490880C1
:1077700008460088012803D1D2480088DA490880E9
:10778000D0480088D9490880CE480088C117839026
:1077900000EB916080118790CA480088C1178390E0
:1077A00000EB916081118398A0EB811080B28690EC
:1077B0000020859087987C90CD48006800F5C060D7
:1077C000CC49097800EB412010304FF4F8720146A3
:1077D00083906846F8F72CFDC548006800F5C06046
:1077E000C449097800EB412083900FC8F9F726FBC4
:1077F00008B10120859040F2D51185984843BC49D5
:10780000096801F5206101EB8021879801EB402197
:10781000869801EBC000408884904FF6FF718498F1
:1078200088420BD1B248006800F5C060B1490978C0
:1078300000EB41204088B049088010E04EF66021FE
:107840008498884208DB0B21849801EB0021A04832
:10785000016034201BE404E0A749849808800C20D0
:1078600015E48A9809280BD19B480088401C9A4946
:1078700008809A480088401C984908800C2006E43B
:107880008A9808280BD194480088401C92490880A7
:1078900092480088401C914908800C2013E48A9883
:1078A000022815D18E480088002805DD8C48008804
:1078B000401E8B4908800BE087480088401C8649A1
:1078C000088086480088401C844908800C2005E414
:1078D00089980EE48A98A8BB0120884908708849D5
:1078E0000870884811F0BBFF0FF038F90DF032F83E
:1078F000B0F57A7F0FDB0121824810F0DFFC889021
:107900008898012807D00E21889801EB0021704843
:107910000160342012E475480088009072480388A2
:10792000012278496F4800880EF0CCFF8890889833
:10793000012808D00F21889801EB002164480160DC
:10794000342045E404E06F4811F0EAFA25203FE4D2
:1079500089983DE48A9860B90120684908700CF064
:1079600099FF012803D168490870042030E42020E1
:107970002EE489982CE48A98F0B9012063490870B4
:10798000604811F06CFF0FF0E9F801225D49604892
:1079900000880FF063FD87908798012807D0102199
:1079A000879801EB00204A490860342010E45548CC
:1079B00011F0B6FA25200BE400BF8A9800BB012025
:1079C0004E490870514908704E4811F048FF0FF0B9
:1079D000C5F801224B494E48008810F0E1FC879021
:1079E0008798012807D01121879801EB002038499A
:1079F0000860342024E4434811F092FA25201FE463
:107A000000BF8A9808BB434818F0ECFC01203B49B2
:107A100008703E4908703B4811F021FF00200346E2
:107A200014220A2100904FF48030FCF733F90FF054
:107A300095F80020034615220A2100904FF480306B
:107A4000FCF728F90FF0F4FC69E08A98032866D166
:107A500001212C480FF03CFC8790879824280ED1F8
:107A60002C48006818F086FC2B49884256D94B21D7
:107A7000879801EB002116480160342044E4879880
:107A8000012816D10020034616220A2100904FF447
:107A90008030FCF7FFF81B4811F042FA0020034643
:107AA00017220A2100904FF48030FCF7F3F82520CC
:107AB0002AE41221879801EB002005490860342050
:107AC00022E42CE05C140020581400205214002002
:107AD00070140020501400204C1400204E1400207C
:107AE0007414002082140020681400206A140020FE
:107AF0009C1400203D140020841400204A1400200F
:107B000048140020AC5901207614002049140020AC
:107B10006414002094140020A086010000BF8998FE
:107B20001CE48A98E8B9FE4811F099FE0FF016F8A7
:107B30000123FB4AFB480178FB48008811F022FB37
:107B400087908798012807D01321879801EB0020A0
:107B5000F649086034202FE4F14811F0E1F92520BE
:107B60002AE4899828E48A9820B90120F04908700D
:107B7000122021E489981FE48A9810BBEA48008803
:107B800040F2D511484340F2627101EB400087900A
:107B90000020869086AB40F2AA32E64887990068BA
:107BA0001CF01CFA8590859838B11421859801EB5A
:107BB0000020DE49086034200AE43220DE490880D3
:107BC00028E08A980A2801D1142006E48A980B2814
:107BD00004D11520D5490860342006E48A980C2881
:107BE00001D1132008E48A980D2801D1132017E44D
:107BF0008A9802280ED1D0480088002805DDCE489A
:107C00000088401ECC49088004E01620C74908605F
:107C1000342005E4899805E48A9818B9C74818F013
:107C2000E1FB0DE08A9803280AD1C448006818F0E7
:107C3000A1FB87908798C82801D9122021E400BFB2
:107C400089981EE48A9818B9BC4818F0CBFB0DE05F
:107C50008A9803280AD1B948006818F08BFB8790EE
:107C60008798C82801D915200BE400BF899808E43B
:107C70008A98D8BBB248006800F5C060B14909785D
:107C800000EB41204089B0490880084600884EF644
:107C90006021884208DBAC480088172101EB0020F6
:107CA000A2490860342004E40120A8490870A648CD
:107CB000008840F2D511484340F2627101EB400068
:107CC00087900020869086AB40F2AA329948879927
:107CD00000681CF0F9FA8590859840B118218598C4
:107CE00001EB002091490860342010E403E03220C9
:107CF000914908801EE08A98072801D1162006E4E1
:107D00008A98082804D1192088490860342004E49E
:107D10008A9802280ED188480088002805DD864808
:107D20000088401E8449088004E01A207F490860CA
:107D3000342017E4899815E48A9818B97F4818F018
:107D400051FB0EE08A9803280BD17C48006818F09C
:107D500011FB87908798B0F57A7F01D9172006E448
:107D600000BF899805E48A9808BB0120784908700B
:107D700008706B4811F073FD0EF0F0FE0123684AA5
:107D800071480188684800880EF04CFF87908798FA
:107D9000012807D01B21879801EB00206349086068
:107DA000342008E45E4811F0BBF8252016E48998D9
:107DB00014E48A9820B901205D49087019200DE467
:107DC00089980BE48A98F8B9012061490870087015
:107DD000534811F044FD0EF0C1FE012250495248B3
:107DE00000880FF043FF87908798012807D01C2157
:107DF000879801EB00204D490860342011E4484881
:107E000011F08EF825200CE489980AE48A9830B99C
:107E100000205049088050490880262007E48998AE
:107E200005E48A98C8BB3E48801C4A49098830F856
:107E30001100879001214948018000208690879891
:107E40007C903F48006800F5C0603E49097800EB2F
:107E5000412010304FF4F872014680906846F8F7E0
:107E6000E7F93748006800F5C0603649097800EB4B
:107E7000412080900FC8F8F7E1FF08B101208690FB
:107E80008698C0F10100C0B28590879884903148EF
:107E90000088401C80B2809084E0EAE000207F905F
:107EA0001F48801C809930F811007E908498401CF7
:107EB0007E99814267D18698012821D17E987C9055
:107EC0001F48006800F5C0601E49097800EB41209A
:107ED00010304FF4F87201467D906846F8F7A8F923
:107EE0001748006800F5C0601649097800EB41208A
:107EF0007D900FC8F8F7A2FF90B301207F9042E079
:107F00007E987C900E48006800F5C0600D490978A5
:107F100000EB412010304FF4F87201467D9020E0D4
:107F2000AC59012066140020641400207014002055
:107F30004A14002058140020741400207C140020DF
:107F40009C1400203D1400205C14002048140020E4
:107F500049140020A414002086140020A614002038
:107F600011E06846F8F764F9F848006800F5C06069
:107F7000F749097800EB41207D900FC8F8F75EFFC4
:107F800008B901207F907F9838B1F2480088401CE2
:107F9000F04908807E98849000E009E08098401CB9
:107FA00080B28090EC480188809881423FF776AF9C
:107FB00000BF8798401D83908598012803D183983E
:107FC00000F2AA3083908398009000214FF4803013
:107FD000879B859AFBF75EFE002003460090DD48F4
:107FE000028800214FF48030FBF754FE3220DB4939
:107FF00008800020829040F2D51185984843D349EB
:10800000096801F5206101EB8021879801EB402090
:1080100082AB8090CF480288839980981CF054F9F5
:108020008190819820B3CE48008803280FDACD498B
:1080300081980870CC480088401CCB490880C8480B
:108040000088401C81B2C6480180272008E4002037
:1080500000909DF8083201210804819AFBF71AFE6E
:108060001D21819801EB0020C0490860342006E4FE
:108070003DE08A98072801D128200FE48A98082833
:1080800004D11E20B9490860342007E48A980928E1
:1080900017D1B348008803280EDA6320B14908706D
:1080A000B1480088401CB0490880AD480088401C99
:1080B000AB49088027200AE41D20AC490860342021
:1080C00005E48A98022812D1A4480088002805DD1A
:1080D000A2480088401EA149088008E01AF0B4FFB9
:1080E0001F2101EB0020A1490860342012E4899887
:1080F00010E48A9818B99E4818F074F90BE08A9831
:10810000032808D19A48006818F034F9B0F5FA6FDE
:1081100001D9262015E4899813E48A9818B995485E
:1081200018F060F91CE08A98032819D1914800687A
:1081300018F020F987908798B0F57A7F0FD98E488C
:1081400001888448008808448B4908808248008858
:108150000988884201DD262008E4292006E400BFC2
:10816000899805E48A98E8BB32207C4908807848E1
:108170000078F8B90020879087AB0122042173486A
:10818000006800F500601CF09FF886900020034610
:1081900000909DF81C220221C803FBF77BFD869806
:1081A00038B12021869801EB00217048016034200D
:1081B00020E44AE00020879087AB01220321634836
:1081C000006800F5C0601CF07FF886900020034630
:1081D00000909DF81C2203214FF48030FBF75AFDDC
:1081E000869800E009E038B12121869801EB002053
:1081F0005E490860342041E427E08A98072801D1CD
:108200002B203BE48A98082804D122205749086093
:10821000342033E48A98092801D12A202EE48A9850
:10822000022812D14D480088002805DD4B480088FF
:10823000401E4A49088008E01AF006FF232101EB9E
:1082400000204A490860342018E4899816E48A9886
:1082500018B94A4818F0C6F80BE08A98032808D1E4
:108260004648006818F086F8B0F5FA6F01D9292061
:1082700004E489981CE48A9818B93E4818F0B2F8CA
:108280000EE08A9803280BD13A48006818F072F87B
:1082900087908798B0F57A7F01D92C2008E400BF39
:1082A000899805E48A98A8B92948007840B900203F
:1082B0002649096881F8000401202549087007E073
:1082C00001202249096881F8000400202049087033
:1082D0002D2025E4899823E48A9838BB32201F4951
:1082E00008800020879087AB012202211748006890
:1082F00000F580601BF0E8FF869000200090134896
:10830000006890F8000485909DF81C320246042114
:108310008803FBF7BFFC869838B12421869801EBCF
:10832000002012490860342015E446E08A980728A6
:1083300004D10020124908802F200CE48A980828D4
:1083400020D1252009490860342004E49C14002031
:108350003D140020A6140020AC5901207414002004
:10836000861400208A140020881400207014002035
:108370008C1400207C140020A414002094140020ED
:10838000821400208A98092801D12E2014E48A98AA
:10839000022812D1C7480088002805DDC54800889A
:1083A000401EC449088008E01AF04EFE262101EB69
:1083B0000020C1490860342007E4899805E48A98C0
:1083C00018B9BE4818F00EF80BE08A98032808D1B7
:1083D000BA48006817F0CEFFB0F5FA6F01D92D202A
:1083E00005E4899815E48A98C0B9B54817F0FAFFF2
:1083F000B44817F0F7FFB448007870B3F8F7E4FE1C
:10840000B248007803284AD1B148B0F900002D21C4
:1084100001EB0020A849086034200FE48A98032863
:108420003DD1A948007840B9A548006817F0A2FFDF
:10843000B0F57A7F33D9302016E4F8F7EDFEA34883
:10844000007803280AD1A248B0F90000272101EBE7
:10845000002099490860342006E420E09B48007819
:1084600002280BD19648006817F084FFB0F57A7F98
:1084700015D9002094490870302014E49148006810
:1084800017F078FF4EF66021884208D98F480078AF
:10849000282101EB002088490860342025E48998D0
:1084A00023E48A98A8B98B48007830B10020894924
:1084B000087000210120FBF7F9F88748007830B1F7
:1084C00000208549087000210220FBF7EFF80C20FE
:1084D0000BE4899809E48A98D0B9804811F0BFF973
:1084E0000EF03CFB7D497E48008810F04FFF8790DE
:1084F0008798012807D02921879801EB00206E4931
:108500000860342015E4754810F00AFD252010E4B9
:1085100089980EE48A9868BB7248008840F2D511A9
:10852000484340F2627101EB400087900020869042
:1085300086AB40F2AA326C48879900681BF04EFD6A
:108540008590859830B932205A49088001206749C2
:1085500008700EE0002000909DF818320B214FF4B7
:108560008030859AFBF796FB2920604908700C2023
:1085700017E42CE08A980A2801D11E2011E48A9879
:108580000B2804D12B204C490860342009E48A9838
:108590000C2801D11D2004E48A980D2801D11D204A
:1085A00004E48A98022812D142480088002805DD98
:1085B00040480088401E3F49088008E01AF044FD0A
:1085C0002C2101EB00203C490860342016E48998F6
:1085D00014E48A9818B93A4817F004FF0DE08A9815
:1085E00003280AD13648006817F0C4FE87908798A0
:1085F000C82801D91C2006E400BF899805E48A98A0
:1086000018B92F4817F0EEFE0DE08A9803280AD11A
:108610002B48006817F0AEFE87908798C82801D9CC
:108620000C2013E500BF899810E58A9820B38A983A
:1086300005280BD100202E490870264908702649CC
:1086400008700120294908700220FFE48A98062852
:1086500003D1012025490870F8E48A9814280BD129
:108660000020234908701B4908701B49087001202D
:108670001E4908700420E9E48998E7E48A9878B1F3
:108680008A9814280BD100201949087011490870E4
:10869000114908700120154908700420D6E400BF74
:1086A0008998D3E4FE21899801EB002002490860F3
:1086B0003420CBE4741400207014002094140020A3
:1086C0007C140020901400204A140020BE140020C6
:1086D000C21400204814002049140020AC59012085
:1086E000641400205E140020601400207614002022
:1086F000801400202DE9F047804620480778414645
:108700003846FEF7B1F904464FF00009A74201D1FF
:10871000012000E00020824629E009F101000FFA63
:1087200080F9B9F1640F0BDD40F2E73014490860BD
:108730003420124908700021FEF796F9BDE8F08751
:1087400001213846FEF790F90546BD4200D02C467F
:1087500000212046FEF788F90646A64202D14FF0D6
:10876000010A03E0274634464FF0000A00BFBAF181
:10877000000FD2D00148047000BFDFE76C14002066
:10878000701400200146092903DC01F13000C0B259
:1087900070470F2903DC01F13700C0B2F8E75F2012
:1087A000F6E70000B0F900100F4A128811440029C2
:1087B00004DA0D490988494209B20180B0F9001074
:1087C000094A12881144B1F5C87F05DD06490988B8
:1087D000C1F5C87109B201800188034A12881144A9
:1087E00009B2024A91807047DE1C0020D40C02209E
:1087F000B0F900100E4A12881144002904DA0C491D
:108800000988494209B20180B0F90010084A12886B
:108810001144002904DD06490988494209B2018052
:108820000188034A1288114409B2024A1181704733
:10883000A81D0020780D022002461AB901F1080097
:10884000C0B2704701F11700C0B2FAE7B5EEC00B35
:10885000F1EE10FA03D29FED0E1BB0EE410B0E4865
:10886000008801EE100AB8EE411BB4EEC10BF1EE28
:1088700010FA07DD0848008801EE100AB8EE411B27
:10888000B0EE410BBCEEC01B11EE100A80B2704777
:1088900000000000000000005215002010B5F8F79D
:1088A0005BFC10BD70B505460E461446A4F12000D1
:1088B0003A2822D2DFE800F0D1D2D2D2D2D2D2D21C
:1088C000D2D2D2C2D2C7BDCC1D22272C31363B40DA
:1088D000454AD2D2D2D2D2D2D24F54595E63686DB9
:1088E0007277D27C81868B9095D29A9FA4A9AEB3E1
:1088F000D2B83146284600F0F4F8AFE031462846B9
:1089000000F04BF9AAE03146284600F059F9A5E0FD
:108910003146284600F07EF9A0E03146284600F0B6
:10892000A6F99BE03146284600F0BBF996E03146B7
:10893000284600F0E0F991E03146284600F00DFAB3
:108940008CE03146284600F01BFA87E03146284685
:1089500000F051FA82E03146284600F0A2FB7DE0AB
:108960003146284600F0FAFB78E03146284600F010
:1089700071FC73E03146284600F0D2FC6EE03146CF
:10898000284600F02BFD69E03146284600F047FDFF
:1089900064E03146284600F05BFD5FE03146284642
:1089A00000F0E8FD5AE03146284600F0FDFD55E0B4
:1089B0003146284600F012FE50E03146284600F0CD
:1089C000B7FE4BE03146284600F0C4FE46E0314693
:1089D000284600F003FF41E03146284600F054FFEE
:1089E0003CE03146284600F0ABFF37E031462846F0
:1089F00000F0F1FF32E03146284601F061F82DE049
:108A00003146284601F0D8F828E03146284601F0E2
:108A1000E5F823E03146284601F0FAF81EE0314639
:108A2000284601F03AF919E03146284601F0C2F92A
:108A300014E03146284601F032FA0FE0314628466C
:108A400001F03AFA0AE03146284600F0F0FA05E073
:108A50003146284600F0F7FA00E000BF00BF70BDC5
:108A600070B505460E4614460A2C38D2DFE804F0ED
:108A7000050A0F14191E23282D323146284600F00E
:108A800030F870BD3146284600F087F8F9E73146E6
:108A9000284600F095F8F4E73146284600F0BAF889
:108AA000EFE73146284600F0E2F8EAE7314628468B
:108AB00000F0F7F8E5E73146284600F01CF9E0E75A
:108AC0003146284600F049F9DBE73146284600F0F8
:108AD00057F9D6E73146284600F08DF9D1E700BFB7
:108AE000CFE770B504460D46A9B2A21C90B203238D
:108AF000082203F0E5FF05F10C0291B2A21C90B22E
:108B00000323082203F0DCFFAA1C91B2A0B20B23BE
:108B1000032203F0D5FFAA1C91B204F1090290B21E
:108B20000B23032203F0CCFF6A1C91B2621C90B2AB
:108B300004F008F9EA1C91B2E21C90B204F002F9C8
:108B40006A1C91B204F10A0290B204F0FBF8EA1C2C
:108B500091B204F1080290B204F0F4F805F10D02AC
:108B600091B2621C90B204F0EDF805F10B0291B2E3
:108B7000E21C90B204F0E6F805F10B0291B204F1A8
:108B8000080290B204F0DEF805F10D0291B204F192
:108B90000A0290B204F0D6F870BD70B505460C46D6
:108BA000A1B2EA1C90B20323062203F089FFE21C63
:108BB00091B2AA1D90B20C23032203F081FF70BD75
:108BC00070B504460D46A9B2A0B203230C2203F0EF
:108BD00077FFAA1D91B2A0B203230C2203F070FF0D
:108BE00005F10C0291B2A0B203230C2203F068FF3E
:108BF000EA1C91B204F1090290B203231A4603F071
:108C00005FFF05F1090291B2A0B203231A4603F0F7
:108C100057FF70BD70B504460D46A9B2A0B203233C
:108C20000C2203F04DFFAA1D91B2E21C90B2032367
:108C3000092203F045FF05F10C0291B2A0B2032313
:108C40000C2203F03DFFEA1C91B204F1090290B23C
:108C500003231A4603F034FF05F1090291B204F12F
:108C6000090290B203231A4603F02AFF70BD70B5C3
:108C700005460C46A1B2A8B20923032203F020FF47
:108C8000A21D91B2EA1C90B20323062203F018FF42
:108C9000A1B205F1090290B20F23032203F010FFE5
:108CA00070BD70B504460D46A9B2A0B203230C22D4
:108CB00003F006FFAA1D91B2A0B203230C2203F019
:108CC000FFFE05F10C0291B2A0B203230C2203F0C7
:108CD000F7FEEA1C91B2A0B203231A4603F0F0FE9D
:108CE00005F1090291B204F1090290B203231A4678
:108CF00003F0E6FE70BD70B504460D46A9B2A0B201
:108D000003230C2203F0DCFEAA1D91B2A0B20323C0
:108D10000C2203F0D5FE05F10C0291B2A0B20323A0
:108D20000C2203F0CDFEEA1C91B2A0B203231A4636
:108D300003F0C6FE05F1090291B2A0B203231A4660
:108D400003F0BEFE05F1090291B204F1090290B2EE
:108D500003231A4603F0B4FE70BD70B504460D46F9
:108D6000A9B2A0B203230C2203F0AAFEEA1C91B21E
:108D700004F1090290B20C23032203F0A1FE70BD9E
:108D800070B504460D46A9B2A0B203230C2203F02D
:108D900097FEAA1D91B2A0B203230C2203F090FE0D
:108DA00005F10C0291B2A0B203230C2203F088FE5D
:108DB000EA1C91B2A0B203231A4603F081FE05F12A
:108DC000090291B2A0B203231A4603F079FEEA1C0D
:108DD00091B204F1090290B203231A4603F070FE27
:108DE00005F1090291B204F1090290B203231A4677
:108DF00003F066FE70BD70B504460D46A9B2A0B280
:108E00000323092203F05CFEAA1D91B2A0B2032342
:108E1000092203F055FEEA1C91B2A0B203231A46C0
:108E200003F04EFEA9B204F1090290B20F2303220F
:108E300003F046FE70BD00002DE9F04105460E46E8
:108E40001446002C07DA3146284600F0F0F8644258
:108E500005F10F0085B26048844210DD401C94FB90
:108E6000F0F00A2190FBF1F201FB1200C7B23A4682
:108E700031462846FFF7F4FD05F10F0085B257484B
:108E8000844210DD401C94FBF0F00A2190FBF1F2CB
:108E900001FB1200C7B23A4631462846FFF7E0FD13
:108EA00005F10F0085B24E48844210DD401C94FB52
:108EB000F0F00A2190FBF1F201FB1200C7B23A4632
:108EC00031462846FFF7CCFD05F10F0085B2454835
:108ED000844210DD401C94FBF0F00A2190FBF1F27B
:108EE00001FB1200C7B23A4631462846FFF7B8FDEB
:108EF00005F10F0085B23C48844210DD401C94FB14
:108F0000F0F00A2190FBF1F201FB1200C7B23A46E1
:108F100031462846FFF7A4FD05F10F0085B242F265
:108F20000F70844210DD401C94FBF0F00A2190FB8E
:108F3000F1F201FB1200C7B23A4631462846FFF76C
:108F40008FFD05F10F0085B2B4F57A7F11DB4FF488
:108F50007A7094FBF0F00A2190FBF1F201FB120011
:108F6000C7B23A4631462846FFF77AFD05F10F00B1
:108F700085B2632C10DD642094FBF0F00A2190FB95
:108F8000F1F201FB1200C7B23A4631462846FFF71C
:108F900067FD05F10F0085B2092C10DD0A2094FB56
:108FA000F0F00A2190FBF1F201FB1200C7B23A4641
:108FB00031462846FFF754FD05F10F0085B20A201F
:108FC00094FBF0F100FB1140C7B23A463146284607
:108FD000FFF746FDBDE8F081FFC99A3BFFE0F505CC
:108FE0007F9698003F420F009F8601002DE9F041D7
:108FF00006460F4614462046F7F74AF91FFA80F84E
:10900000002510E0625D39463046FFF74BFC605D9D
:10901000202803D106F10C0086B202E006F10E0012
:1090200086B2681C85B24545ECDBBDE8F08170B5C1
:1090300004460D46EA1D91B2A21C90B203230822F9
:1090400003F03EFD70BD70B505460C4604F10C0200
:1090500091B26A1C90B203231A4603F031FD04F169
:10906000090291B2EA1C90B203231A4603F028FDCC
:10907000A21D91B26A1D90B203231A4603F020FD8F
:10908000E21C91B2EA1D90B203231A4603F018FDC8
:10909000A1B205F1090290B203231A4603F010FDB4
:1090A00070BD70B505460C46221D91B2A8B20B23C7
:1090B000032203F005FD221D91B205F1090290B2D1
:1090C0000B23032203F0FCFC04F1090291B2EA1C19
:1090D00090B20323062203F0F3FC221D91B2EA1C96
:1090E00090B203F02FFE221D91B205F1080290B25A
:1090F00003F028FEE01C03B2281D02B2E01C01B2FE
:10910000681C00B201F020FDE01C03B205F10A006A
:1091100002B2E01C01B2E81D00B201F015FDA01C76
:1091200003B205F1090002B2A01C01B2A81C00B2F2
:1091300001F00AFD601C03B205F1080002B2601CD8
:1091400001B2E81C00B201F0FFFC23B2E81D02B23C
:1091500021B2281D00B201F0F7FC70BD70B50546C4
:109160000C46A1B2A8B20F23032203F0A9FCA1B2BE
:10917000EA1C90B20323062203F0A2FCA21D91B2C6
:10918000EA1C90B20323072203F09AFC04F10C02BC
:1091900091B2EA1C90B20323062203F091FCA21CB8
:1091A00091B205F1090290B20523022203F088FC76
:1091B00004F1080291B205F1090290B205230222DE
:1091C00003F07EFC601D03B205F10B0002B2E01C4F
:1091D00001B205F10B0000B201F0B6FC04F10B0086
:1091E00003B205F10B0002B204F1090001B205F16E
:1091F0000B0000B201F0A8FC621C91B205F109025B
:1092000090B203F09FFDE21C91B205F1080290B20A
:1092100003F098FD621D91B205F1080290B203F0CF
:1092200091FD04F1090291B205F1080290B203F038
:1092300089FD04F10B0291B205F1080290B203F02E
:1092400081FD04F10D0291B205F1090290B203F023
:1092500079FD70BD70B504460D46AA1C91B2A0B24E
:109260000B23032203F02CFCA9B2A21C90B203230F
:10927000082203F025FC05F10C0291B2A21C90B269
:109280000323082203F01CFCAA1C91B204F109027A
:1092900090B203231A4603F013FC05F10A0291B2BF
:1092A00004F1090290B203231A4603F009FC6A1C78
:1092B00091B2621C90B203F045FDEA1C91B2E21C2F
:1092C00090B203F03FFD05F10D0291B2621C90B225
:1092D00003F038FD05F10B0291B2E21C90B203F0ED
:1092E00031FDEA1C91B204F1080290B203F02AFDAC
:1092F0006A1C91B204F10A0290B203F023FD05F159
:109300000B0291B204F1080290B203F01BFD05F1CB
:109310000D0291B204F10A0290B203F013FD70BD88
:1093200070B504460D46EA1C91B2A0B2092303228F
:1093300003F0C6FBA9B2A0B20323092203F0C0FBCD
:1093400005F10C0291B2A0B20323092203F0B8FB8D
:10935000EA1C91B204F1090290B20923032203F03E
:10936000AFFB6A1C91B204F1090290B203F0EAFC6F
:10937000AA1C91B204F1090290B203F0E3FCAA1C0A
:1093800091B204F10A0290B203F0DCFCEA1C91B243
:1093900004F1080290B203F0D5FC05F10B0291B282
:1093A00004F1080290B203F0CDFC05F10D0291B278
:1093B00004F1090290B203F0C5FC05F10C0291B270
:1093C00004F1090290B203F0BDFC05F10C0291B268
:1093D00004F10A0290B203F0B5FC70BD70B504460A
:1093E0000D46A9B2A0B203230C2203F069FB05F1DC
:1093F0000C0291B2A0B203230C2203F061FBAA1D60
:1094000091B2E21C90B20323062203F059FBEA1C3E
:1094100091B2A0B20923032203F052FB70BD70B5D4
:1094200004460D46A9B2A0B203230C2203F048FB68
:10943000AA1D91B2E21C90B20323062203F040FB66
:10944000EA1C91B2A0B20C23032203F039FB70BDD9
:1094500070B504460D46EA1C91B2A0B2092303225E
:1094600003F02EFBEA1C91B2E21C90B203F06AFCFE
:10947000AA1C91B2621C90B203F064FC6A1C91B207
:10948000A21C90B203F05EFCAA1C91B2A21C90B286
:1094900003F058FCA9B2E21C90B20323062203F0A9
:1094A0000FFB6A1C91B204F1080290B203231A4622
:1094B00003F006FB05F10B0291B2E21C90B203F03F
:1094C00041FC05F10C0291B2621C90B203F03AFC2F
:1094D00005F10C0291B2A21C90B203F033FC05F12D
:1094E0000D0291B2A21C90B203F02CFC05F10C020B
:1094F00091B2E21C90B20323062203F0E1FA05F1D7
:109500000B0291B204F1080290B203F01BFC05F1CA
:109510000C0291B204F1090290B203F013FC05F1C0
:109520000C0291B204F1090290B203F00BFC05F1B8
:109530000C0291B204F10A0290B203F003FC05F1AF
:109540000D0291B204F1090290B203F0FBFB05F1A8
:109550000A0291B204F1090290B20223032203F03D
:10956000AFFAEA1D91B2A21D90B20323062203F0C6
:10957000A7FA70BD70B505460C46A1B2A8B20F237C
:10958000032203F09DFAA1B205F1090290B20F2364
:10959000032203F095FAA21D91B2EA1C90B20323B4
:1095A000062203F08DFA70BD70B504460D46A9B2CF
:1095B000A0B203230C2203F083FA05F10C0291B24E
:1095C000A0B203230C2203F07BFAEA1C91B2221D05
:1095D00090B20923042203F073FA70BD70B50546FA
:1095E0000C46A1B2A8B20F23032203F069FA621D50
:1095F00091B2EA1C90B20523032203F061FA221D06
:1096000091B26A1D90B203F09DFB04F10A0291B27F
:109610006A1D90B203F096FBA01D03B2A81D02B212
:10962000E01C01B2A81D00B201F08EFA601D03B269
:10963000E81D02B2A01C01B2E81D00B201F084FADC
:10964000201D03B205F1080002B2601C01B205F151
:10965000080000B201F078FAE01C03B205F109003D
:1096600002B221B200B201F06FFAA01C03B205F100
:109670000A0002B221B200B201F066FA601C03B225
:1096800005F10B0002B221B200B201F05DFA04F163
:109690000B0003B2A81D02B204F1080001B2A81D1C
:1096A00000B201F051FA04F10C0003B2E81D02B25D
:1096B00004F1090001B2E81D00B201F045FA04F11D
:1096C0000D0003B205F1080002B204F10A0001B274
:1096D00005F1080000B201F037FA04F10E0003B200
:1096E00005F1090002B204F10B0001B205F1090015
:1096F00000B201F029FA04F10E0003B205F10A00EC
:1097000002B204F10C0001B205F10A0000B201F04E
:109710001BFA04F10E0003B205F10B0002B204F1D2
:109720000D0001B205F10B0000B201F00DFA70BDA1
:1097300070B504460D46A9B2A0B20F23032203F070
:10974000BFF905F10C0291B2A0B203230C2203F081
:10975000B7F970BD70B505460C46A1B2A8B20F238B
:10976000032203F0ADF9A1B205F1090290B20F2373
:10977000032203F0A5F9601D03B2E81C02B2601CCD
:1097800001B2E81C00B201F0DFF9601D03B205F17F
:10979000080002B2601C01B205F1080000B201F03D
:1097A000D3F9A01D03B2281D02B2A01C01B2281DCE
:1097B00000B201F0C9F9A01D03B2E81D02B2A01C5D
:1097C00001B2E81D00B201F0BFF9E21C91B26A1DBE
:1097D00090B20523022203F073F970BD70B50546FF
:1097E0000C46A1B2A8B20F23032203F069F9A1B27B
:1097F00005F1090290B20F23032203F061F9601D05
:1098000003B2E81C02B2601C01B2E81C00B201F015
:109810009BF9A01D03B2281D02B2A01C01B2281D95
:1098200000B201F091F904F1080003B2681D02B220
:10983000201D01B2681D00B201F086F904F10A0092
:1098400003B2A81D02B2A01D01B2A81D00B201F012
:109850007BF904F10C0003B2E81D02B204F1080028
:1098600001B2E81D00B201F06FF904F10D0003B27E
:1098700005F1080002B204F1090001B205F1080087
:1098800000B201F061F970BD70B504460D46A9B291
:10989000A21C90B20323082203F012F905F10C0276
:1098A00091B2A21C90B20323082203F009F9AA1C6A
:1098B00091B2A0B20B23032203F002F9AA1C91B2C9
:1098C00004F1090290B20B23032203F0F9F86A1C99
:1098D00091B2621C90B203F035FAEA1C91B2E21C1C
:1098E00090B203F02FFA6A1C91B204F10A0290B20E
:1098F00003F028FAEA1C91B204F1080290B203F0D6
:1099000021FA05F10B0291B2E21C90B203F01AFAAF
:1099100005F10D0291B2621C90B203F013FA05F149
:109920000B0291B204F1080290B203F00BFA05F1B8
:109930000D0291B204F10A0290B203F003FA70BD75
:1099400070B505460C46A1B2A8B20F23032203F05E
:10995000B7F8A1B2EA1C90B20323062203F0B0F8D4
:10996000E21D91B2EA1C90B20323062203F0A8F88C
:10997000E21C91B205F1080290B203F0E3F9A21DD6
:1099800091B205F1080290B203F0DCF904F108008D
:1099900003B205F1090002B2601C01B205F1090031
:1099A00000B201F0D1F8A21C91B205F10A0290B206
:1099B00003F0C8F9E21D91B205F10A0290B203F07A
:1099C000C1F9E21C91B205F10A0290B2042302220D
:1099D00003F076F870BD70B505460C46A1B2A8B28A
:1099E0000F23032203F06CF8A1B2EA1C90B2032308
:1099F000062203F065F8E21D91B2EA1C90B203233F
:109A0000062203F05DF8E21C91B205F1080290B263
:109A100003F098F9A21D91B205F1080290B203F08B
:109A200091F904F1080003B205F1090002B2601CCB
:109A300001B205F1090000B201F086F8A21C91B252
:109A400005F10A0290B203F07DF9E21D91B205F131
:109A50000A0290B203F076F9E21C91B205F10A0213
:109A600090B20423022203F02BF804F10A0291B20F
:109A7000AA1D90B203F066F904F10A0291B2EA1D40
:109A800090B20223032203F01BF804F10C0291B2FE
:109A900005F1080290B203F055F904F10B0291B2FE
:109AA00005F10A0290B203F04DF904F10C0291B2F3
:109AB00005F1090290B203231A4603F001F870BDC4
:109AC00070B504460D46A9B2A21C90B20323082229
:109AD00002F0F6FF6A1C91B204F1080290B203236F
:109AE0001A4602F0EDFF6A1C91B2621C90B2032389
:109AF0001A4602F0E5FFAA1C91B204F10A0290B2E4
:109B00000323022202F0DCFFAA1C91B2A0B20423BC
:109B1000032202F0D5FF6A1D91B2621C90B20223AB
:109B2000032202F0CDFFAA1D91B2A21C90B2022323
:109B3000072202F0C5FFEA1D91B2E21C90B2022397
:109B4000072202F0BDFF05F1080291B204F10802FC
:109B500090B20223032202F0B3FF05F1090291B291
:109B600004F1090290B20423032202F0A9FF05F1D7
:109B70000B0291B204F1080290B203231A4602F0DC
:109B80009FFF05F10C0291B2A21C90B203230822A0
:109B900002F096FF05F10B0291B2621C90B2032312
:109BA0001A4602F08DFF05F10A0291B2A0B203231A
:109BB000022202F085FF70BD70B504460D46A9B2C1
:109BC000A0B203230C2202F07BFFEA1C91B2221DFB
:109BD00090B20C23032202F073FF70BD70B50446EF
:109BE0000D46A9B2A0B20F23032202F069FF05F1CE
:109BF0000C0291B2A0B203230C2202F061FFA9B2C1
:109C000004F1090290B20C23032202F059FF70BD47
:109C100070B505460C46A1B2A8B203231A4602F05D
:109C20004FFFA1B205F1090290B203231A4602F0D8
:109C300047FFE21C91B26A1C90B203231A4602F05D
:109C40003FFFE21C91B205F1080290B203231A46CD
:109C500002F036FFA21D91B2AA1C90B203231A464D
:109C600002F02EFFA21D91B2EA1D90B203231A4604
:109C700002F026FF04F1090291B2EA1C90B203231C
:109C8000062202F01DFF04F10C0291B22A1D90B2CF
:109C90000323042202F014FF70BD70B505460C4684
:109CA000A1B2A8B203231A4602F00AFFA1B205F13D
:109CB000090290B203231A4602F002FFE21C91B29D
:109CC0006A1C90B203231A4602F0FAFEE21C91B21B
:109CD00005F1080290B203231A4602F0F1FEA21D1C
:109CE00091B2AA1C90B203231A4602F0E9FEA21D0B
:109CF00091B2EA1D90B203231A4602F0E1FE04F18C
:109D0000090291B2EA1C90B20323062202F0D8FEA7
:109D100004F10C0291B22A1D90B20323042202F036
:109D2000CFFEA1B205F1090290B203231A4602F058
:109D3000C7FEA1B205F1120290B203231A4602F047
:109D4000BFFEE21C91B205F10A0290B203231A464B
:109D500002F0B6FEE21C91B205F1110290B20323AB
:109D60001A4602F0ADFEA21D91B205F10B0290B2AF
:109D700003231A4602F0A4FEA21D91B205F11002BF
:109D800090B203231A4602F09BFE04F1090291B23D
:109D900005F10C0290B20323062202F091FE04F1B9
:109DA0000C0291B205F10D0290B20323042202F0DD
:109DB00087FE70BD70B505460C4604F1090291B2EC
:109DC0002A1D90B20623042202F07AFEA21D91B24F
:109DD000EA1C90B20323062202F072FEA1B2A8B2DE
:109DE00003231A4602F06CFEA1B2A8B203231A465E
:109DF00002F066FEA1B205F1090290B203231A46F1
:109E000002F05EFEE21C91B26A1C90B202230322B1
:109E100002F056FEE21C91B205F1080290B2022354
:109E2000032202F04DFE601D03B2281D02B2601D28
:109E300001B2A81C00B200F087FE601D03B205F15C
:109E4000090002B2601D01B2E81D00B200F07CFE04
:109E5000A21C91B2EA1C90B202F074FFA21C91B253
:109E600005F1080290B202F06DFF221D91B22A1D89
:109E700090B202F067FF221D91B2EA1D90B202F08B
:109E800061FFA21D91B2AA1C90B202F05BFFA21D5D
:109E900091B205F1090290B202F054FF70BD70B5A5
:109EA00004460D4605F1090291B2E21C90B2062368
:109EB0001A4602F005FE70BD70B504460D46EA1D57
:109EC00091B2A21C90B20323082202F0F9FD2A1DD0
:109ED00091B2621D90B20823032202F0F1FD70BD21
:109EE0002DE9F04306460F4690460320A0EB4809B3
:109EF000002445463EE07A1B91B2321990B202F03E
:109F000021FF7A1B91B2321B90B202F01BFF3A1B69
:109F100091B2721990B202F015FF3A1B91B2721B06
:109F200090B202F00FFF7A1991B2321990B202F09A
:109F300009FF7A1991B2321B90B202F003FF3A196D
:109F400091B2721990B202F0FDFE3A1991B2721BF1
:109F500090B202F0F7FEB9F1000F04DA062000EB30
:109F60008400814405E0601B0A2101EB80008144EC
:109F70006D1E641CAC42BED9BDE8F0832DE9F04FE4
:109F800006460F46904699460024C9F100054FEA5F
:109F90004800C0F1020A9FED560AB0EE403A9FED2C
:109FA000540AF0EE403A9FED520AB0EE404A00EEFD
:109FB000108AB8EEC00AF0EE403A00EE109AB8EE01
:109FC000C00AB0EE404A84EE230AB0EE403A00BF29
:109FD00000EE104AB8EEC00AC0EE030ABCEEE00A7A
:109FE00010EE100A80B2301A00EE100AB8EEC00B64
:109FF000B0EE405B781900EE100AB8EEC00BB0EE80
:10A00000401BB0EE450B02F00BFF00EE104AB8EE1D
:10A01000C00AC0EE030ABCEEE00A10EE100A80B2DD
:10A02000304400EE100AB8EEC00BB0EE405B781979
:10A0300000EE100AB8EEC00BB0EE401BB0EE450BC0
:10A0400002F0EEFE00EE104AB8EEC00AC0EE030ABF
:10A05000BCEEE00A10EE100A80B2304400EE100AA6
:10A06000B8EEC00BB0EE405B781B00EE100AB8EE05
:10A07000C00BB0EE401BB0EE450B02F0D1FE00EE7F
:10A08000104AB8EEC00AC0EE030ABCEEE00A10EEB9
:10A09000100A80B2301A00EE100AB8EEC00BB0EE13
:10A0A000405B781B00EE100AB8EEC00BB0EE401B10
:10A0B000B0EE450B02F0B4FED346A3450BDC601CAA
:10A0C0000446012101EB40008244E54203D1AB4547
:10A0D00001DC4FF0000BAB4505DD681C0546012196
:10A0E00001EB40008244002D7FF772AFBDE8F08F96
:10A0F000000000002DE9FF4F82B00F9CBDF8080062
:10A10000BDF80A206C4909688B4202D306B0BDE84D
:10A11000F08F6A4909688C4200D3F7E71918664D39
:10A120002D68A94203D364490988C91A88B2A118C5
:10A13000624D2D68A94203D360490988091B8AB280
:10A140005F49098861BB002127E0002521E0DFF895
:10A1500074C1DCF8006004EB010CDFF85C81D8F816
:10A1600000800CFB08FC06EB8C0603EB050C06EBF1
:10A170008C0601FB00FC1FFA8CF707EB050C1FFA9D
:10A180008CF7DDF810C05CF827C0C6F800C06E1C64
:10A19000B5B28542DBDB4D1CA9B29142D5DB88E02C
:10A1A00047490988012938D1002533E000262DE0F0
:10A1B000DFF810B1DBF8001004EB050BDFF8F8E076
:10A1C000DEF800E00BFB0EFB0BEB4B0B594403EBF3
:10A1D000060B0BEB4B0B594405FB00FB1FFA8BFCEA
:10A1E0000CEB060B1FFA8BFCDDF810B05BF82C7043
:10A1F000C7F30748C7F3072907F0FF0A81F800A053
:10A2000081F8019081F80280711C8EB28642CFDB0A
:10A21000691C8DB29542C9DB4BE0294909880429A4
:10A2200047D1002543E000213DE0DFF898B0DBF89E
:10A23000006004EB050BDFF880E0DEF800E00BFBCC
:10A240000EFB06EB4B0603EB010B06EB4B0605FB87
:10A2500000FB1FFA8BFC0CEB010B1FFA8BFCDDF8EB
:10A2600010B05BF82C70C7F30748C7F3072A07F054
:10A27000FF094FF0F00B0BEB281B0BF0FF0BCDF899
:10A2800004B00AF0F00B0BEB291B0BF0FF0BCDF821
:10A2900000B0DDF800B086F800B0DDF804B086F854
:10A2A00001B04E1CB1B28142BFDB691C8DB2954238
:10A2B000B9DB00BF2AE70000E0130020E413002010
:10A2C000E8130020DC1300202DE9FF41BDF8005009
:10A2D000BDF8026028480068824201D3BDE8FF81D2
:10A2E00026480068834200D3F8E7501922490968DC
:10A2F000884203D320480088801A85B298191F49E4
:10A300000968884203D31D480088C01A86B21C48D9
:10A31000008804282DD1002029E0002123E0DFF867
:10A3200064C0DCF8004003EB000CDFF84C80D8F888
:10A3300000800CFB08FC04EB4C0402EB010C04EB6A
:10A340004C04BDF800C00CFB00FC1FFA8CF707EBB7
:10A35000010C1FFA8CF7DDF804C03CF817C0A4F814
:10A3600000C04C1CA1B2A942D9DB411C88B2B0424A
:10A37000D3DB00BFB2E70000E0130020E4130020AD
:10A38000E8130020DC1300202DE9FF4FDDE90E8EDD
:10A39000DDF834C0BDF80070BDF80290314C24687F
:10A3A000A24201D3BDE8FF8F2F4C2468A34200D303
:10A3B000F8E7D4192B4D2D68AC4203D3294C2488DF
:10A3C000A41AA7B203EB0904274D2D68AC4204D3AD
:10A3D000254C2488E41A1FFA84F9244C2488042C80
:10A3E0003DD1002439E0002533E002EB050B1FFAD4
:10A3F0008BF003EB040B1FFA8BF1604525DB7045F6
:10A4000023DC414521DBDDF840B059451DDCDFF898
:10A4100060B0DBF80060DFF84CB0DBF800B001FBA7
:10A420000BFB06EB4B0606EB4006BDF800B00BFB42
:10A4300004FB1FFA8BFA0AEB050B1FFA8BFADDF807
:10A4400004B03BF81AB0A6F800B005F1010B1FFAF2
:10A450008BF5BD42C9DB651CACB24C45C3DB00BF0C
:10A46000A0E70000E0130020E4130020E813002020
:10A47000DC1300202DE9FF41BDF80040BDF802606B
:10A4800029480068824201D3BDE8FF81274800685F
:10A49000834200D3F8E7101923490968884203D39F
:10A4A00021480088801A84B2981920490968884296
:10A4B00003D31E480088C01A86B21D4800880428AD
:10A4C00030D100202CE0002126E0DFF868C0DCF865
:10A4D000005003EB000CDFF85080D8F800800CFB34
:10A4E00008FC05EB4C0502EB010C05EB4C05BDF837
:10A4F00000C00CFB00FC1FFA8CF7A4EB010CACF1C4
:10A50000010CBC441FFA8CF7DDF804C03CF817C0FE
:10A51000A5F800C04D1CA9B2A142D6DB411C88B2EF
:10A52000B042D0DB00BFAFE7E0130020E41300200F
:10A53000E8130020DC1300202DE9FF4FDDE90E8E2B
:10A54000DDF834C0BDF80060BDF80290324C2468DC
:10A55000A24201D3BDE8FF8F304C2468A34200D350
:10A56000F8E794192C4D2D68AC4203D32A4C24886B
:10A57000A41AA6B203EB0904284D2D68AC4204D3FB
:10A58000264C2488E41A1FFA84F9254C2488042CCC
:10A5900040D100243CE0002536E002EB050B1FFA19
:10A5A0008BF003EB040B1FFA8BF1604528DB704541
:10A5B00026DC414524DBDDF840B0594520DCDFF8DE
:10A5C00064B0DBF80070DFF850B0DBF800B001FBDE
:10A5D0000BFB07EB4B0707EB4007BDF800B00BFB8D
:10A5E00004FB1FFA8BFAA6EB050BABF1010BD3446E
:10A5F0001FFA8BFADDF804B03BF81AB0A7F800B0E8
:10A6000005F1010B1FFA8BF5B542C6DB651CACB238
:10A610004C45C0DB00BF9DE7E0130020E4130020A1
:10A62000E8130020DC1300202DE9FF4F86B01D4603
:10A63000079E96F80080079E76780596934E3668BA
:10A64000B24202D30AB0BDE8F08F914E3668B542EF
:10A6500000D3F7E702EB08068C4F3F68BE4204D3F5
:10A660008A4E3688B61A1FFA86F8059E2E44884F01
:10A670003F68BE4204D3864E3688B61AB6B20596F7
:10A68000059E2E44761E36B2049602EB0806761E10
:10A6900034B2079E96F80290032606EB4900114655
:10A6A0002B46E6E0079E365CFF2E51D1BDF81870B0
:10A6B000861CB74249DD471CDDF81CC01CF807604A
:10A6C000871CDDF81CC01CF807A04FF0030C0CEB36
:10A6D000460C079F17F80C7003974FF0040C0CEB17
:10A6E000460C079F17F80C700297019101EB0A07BF
:10A6F0007F1E0FFA87FEA64500DDA646019F19E0E2
:10A70000DFF890B1DBF800C0DFF880B1DBF800B013
:10A710004FEA4B0B0BFB03CC0CEB470CDDF80CB0FA
:10A720008CF801B0DDF808B08CF800B007F1010C2E
:10A730000FFA8CF77745E3DD01EB0A0739B2A14246
:10A7400002DD11465F1C3BB200BFC61CB0B290E0F8
:10A75000079E365CFE2E50D1471CDDF81CC01CF84D
:10A760000760871CDDF81CC01CF807E04FF0030CE5
:10A770000CEB460C079F17F80C7003974FF0040C76
:10A780000CEB460C079F17F80C700297019303EB34
:10A790000E077F1E3FB20097019B9A4623E01746A3
:10A7A00019E0DFF8F0B0DBF800C0DFF8E0B0DBF86C
:10A7B00000B04FEA4B0B0BFB0ACC0CEB470CDDF85F
:10A7C0000CB08CF801B0DDF808B08CF800B007F1DF
:10A7D000010C0FFA8CF702EB080CBC45E1DC0AF126
:10A7E00001070FFA87FA009FBA45D8DD114603EB3F
:10A7F0000E073BB2C71CB8B23BE0DDF81CB01BF83B
:10A8000000604FF0030E0EEB460EDDF81CB01BF897
:10A810000EC04FF0040E0EEB460EDDF81CB01BF818
:10A820000EA00AEB0C2B1FFA8BFBCDF80CB0DFF857
:10A8300064B0DBF80070DFF854B0DBF800B003FB65
:10A840000BFB07EB4B0707EB4107DDF80CB0A7F854
:10A8500000B001F1010B0FFA8BF1A14204DD1146AA
:10A8600003F1010B0FFA8BF300F1010B1FFA8BF0D0
:10A8700000BFBDF81860864205DDA1427FF712AF28
:10A88000049EB342FADD00BFDCE60000E0130020C6
:10A89000E4130020DC1300202DE9FF4F89B014469B
:10A8A0001E46DDF858E00A9D95F800900A9D6D78E7
:10A8B0000895A24D2D68AC4202D30DB0BDE8F08FD3
:10A8C0009F4D2D68AE4200D3F7E704EB09059B4F7F
:10A8D0003F68BD4204D3994D2D882D1B1FFA85F981
:10A8E000089D3544964F3F68BD4204D3944D2D8852
:10A8F0002D1BADB20895089D35446D1E2DB20795F0
:10A9000004EB09056D1E2BB20A9D95F802A00325E4
:10A9100005EB4A01002506950A9D0595224630461D
:10A92000FFE00A9D6D5CFF2D63D1BDF824708D1C86
:10A93000AF425BDD4D1CDDF828C01CF805708D1C96
:10A94000DDF828C01CF805B04FF0030C0CEB470CE9
:10A950000A9D15F80C5004954FF0040C0CEB470CB5
:10A960000A9D15F80C500395029202EB0B056D1E23
:10A970002DB20195019D9D4200DD0193029D28E0CD
:10A98000754522DBDDF860C065451EDCDDF85CC086
:10A9900060451ADBDDF864C0604516DCDFF8A48191
:10A9A000D8F800C0DFF89481D8F800804FEA480852
:10A9B00008FB00CC0CEB450CDDF810808CF8018016
:10A9C000DDF80C808CF8008000BF05F1010C0FFA57
:10A9D0008CF5DDF804C06545D2DD02EB0B052AB22B
:10A9E0009A4202DD2246451C28B200BFCD1CA9B206
:10A9F00097E00A9D6D5CFE2D57D14D1C0A9F17F8FC
:10AA000005C08D1C0A9F7D5D0495032707EB4C074D
:10AA10000A9DED5D0395042707EB4C070A9DED5D4C
:10AA200002950190049D05446D1E2DB2009501987C
:10AA3000074630E0254628E0754522DBDDF86080DA
:10AA400045451EDCDDF85C8047451ADBDDF8648097
:10AA5000474516DCDFF8ECB0DBF80080DFF8DCB04F
:10AA6000DBF800B04FEA4B0B0BFB078808EB4508FF
:10AA7000DDF80CB088F801B0DDF808B088F800B057
:10AA800000BF05F101080FFA88F504EB0908A84595
:10AA9000D2DC7D1C2FB2009DAF42CBDD2246049D4F
:10AAA000054428B2CD1CA9B23BE00A9F7D5C4FF063
:10AAB000030808EB45080A9F17F808C04FF0040880
:10AAC00008EB45080A9F17F808B00BEB0C27BFB23C
:10AAD000049772451BDB189FBA4218DC179FB842D7
:10AAE00015DB199FB84212DCDFF85880D8F80070E7
:10AAF000DFF84880D8F8008000FB08F807EB48072B
:10AB000007EB4207DDF81080A7F8008000BF571C54
:10AB10003AB29A4202DD2246471C38B24F1CB9B203
:10AB200000BFBDF824508D4205DD9A427FF7F9AE93
:10AB3000079DA842FADD00BFBFE60000E013002039
:10AB4000E4130020DC1300202DE9F04F8AB0044606
:10AB50000D4691469A465A48007810B90AB0BDE8A9
:10AB6000F08FA14503DACDF82490A146099CAA45AF
:10AB700003DACDF824A0AA46099D55450ED15148C7
:10AB80000068854209D2264605E0A9B2B0B202F0BB
:10AB9000D9F8701C06B24E45F7DD8EE04C450ED15B
:10ABA000494800688442F8D2AEB205E0A0B231460E
:10ABB00002F0C8F8701C86B25645F7DD7DE000262D
:10ABC0000027B34600200890079006900590049057
:10ABD00080460390029001900090A9EB040006B219
:10ABE000002E01DA704206B2AAEB050007B2002F70
:10ABF00001DA784207B2A3460895A14503DB01209C
:10AC00000790069003E04FF0FF3007900690AA45AA
:10AC100003DB01200590049003E04FF0FF30059026
:10AC20000490BE420CDB002007900490B0463046F2
:10AC300006EBD071491009B20391029701960BE01F
:10AC4000002006900590B846384607EBD0714910B1
:10AC500009B20391029601970020009028E0089A1B
:10AC600091B21FFA8BF002F06DF8DDE90210084492
:10AC700000B20390039840450DDB0398A0EB080059
:10AC800000B20390079858440FFA80FB0599089882
:10AC9000084400B20890069858440FFA80FB0499C3
:10ACA0000898084400B208900098401C00B2009038
:10ACB000DDE900018842D2DD00BF00BF4EE70000A1
:10ACC000D8130020E4130020E01300202DE9F04306
:10ACD00004460D4616461F462B48007808B9BDE8C5
:10ACE000F083A019401E1FFA80F8E819401E1FFAD1
:10ACF00080F926480068804504D324480088401E17
:10AD00001FFA80F822480068814504D32048008853
:10AD1000401E1FFA80F906B9E1E707B9DFE71B48D3
:10AD20000068844200D3DAE719480068854200D3FE
:10AD3000D5E7A019401E02B22BB229B220B2FFF70C
:10AD400003FFE819401E03B222B229B220B2FFF776
:10AD5000FBFEE819401E03B2A019401E02B2E8191A
:10AD6000401E01B220B2FFF7EFFEE919491E0BB2F7
:10AD7000A119491E0AB2A119491E08B229B2FFF74A
:10AD8000E3FE00BF00BFAAE7D8130020E0130020B5
:10AD9000E41300202DE9F04F2DED108B87B0B0EEBD
:10ADA00040ABB0EE41BBB0EE429BC748007820B943
:10ADB00007B0BDEC108BBDE8F08FC44800880428B4
:10ADC0007ED13AEE490BBDEEC00B10EE100A07B271
:10ADD0003AEE090BB7EE001B30EE010BBDEEC00BD7
:10ADE00010EE100A0FFA80F83BEE490BBDEEC00BD7
:10ADF00010EE100A0FFA80F93BEE090BB7EE001BBC
:10AE000030EE010BBDEEC00B10EE100A0FFA80FA07
:10AE1000AF480068874200D3CAE7B8F1000F00DAF4
:10AE2000C6E7AC480068814500D3C1E7BAF1000F1E
:10AE300000DABDE7002F00DA0027A548006880454A
:10AE400004D3A3480088401E0FFA80F8B9F1000F20
:10AE500001DA4FF000099F480068824504D39D48FD
:10AE60000088401E0FFA80FA3D4627E14E4620E159
:10AE700000EE105AB8EEC00B30EE4AEB00EE106A4E
:10AE8000B8EEC00B30EE4BDB2EEE0E1B0DEE0D1BA5
:10AE9000B0EE410B28F078FBB0EE40CBB6EE000BE5
:10AEA00039EE000BB4EECC0BF1EE10FA7DD9B6EE14
:10AEB000000B39EE400BB4EECC0BF1EE10FA00E0D3
:10AEC00000E173D2B6EE003B39EE433B3CEE433B30
:10AED000B7EE004B34EE438BDFF8FCB1DBF80040FB
:10AEE000DFF8ECB1DBF800B04FEA4B0B0BFB06448C
:10AEF00004EB450494F801B0CDF818B094F800C004
:10AF0000DDF818B04FEA2B1B00EE10BADDF818B0D0
:10AF10000BF00F0B00EE90BA4FEA2C1B01EE10BAAB
:10AF20000CF00F0B01EE90BADFF8B0B19BF800B057
:10AF30004FEA2B1B02EE10BADFF8A0B19BF800B06D
:10AF40000BF00F0B02EE90BADFF894B19BF800B053
:10AF50004FEA2B1B06EE10BADFF884B19BF800B065
:10AF60000BF00F0B06EE90BAB8EE423B28EE033B17
:10AF7000B7EE004B34EE484BB8EE405B04EE053BB9
:10AF8000B0EE437BB8EE623B28EE033BB7EE004BDE
:10AF900034EE484BB8EE605B04EE053BB0EE43FB8D
:10AFA000B8EE463B28EE033B01E080E070E0B7EEF0
:10AFB000004B34EE484BB8EE415B04EE053B8DEDA3
:10AFC000043BB8EE663B28EE033BB7EE004B34EE95
:10AFD000484BB8EE615B04EE053B8DED023BB0EEF5
:10AFE000473BB6EE004B33EE043BBCEEC33B13EEE7
:10AFF00010BA0BF0FF00B0EE4F3BB6EE004B33EE55
:10B00000043BBCEEC33B13EE10BA0BF0FF019DED09
:10B01000043BB6EE004B33EE043BBCEEC33B13EEF9
:10B0200010BA0BF0FF029DED023BB6EE004B33EE83
:10B03000043BBCEEC33B13EE10BA0BF0FF03002839
:10B0400000DA00200F2800DD0F20002900DA00219F
:10B050000F2900DD0F21002A00DA00220F2A00DD6F
:10B060000F22002B00DA00230F2B00DD0F2301EB52
:10B07000001B0BF0FF0E03EB021B0BF0FF0BCDF8D8
:10B0800004B084F801E0DDF804B084F800B00EE00C
:10B09000114804680E480068400000FB064404EBB9
:10B0A00045040E48007860700D4800782070701CD0
:10B0B00006B256457FF7DCAE681C05B245457FF702
:10B0C000D5AE00BF00BF73E6D8130020E813002000
:10B0D000E0130020E4130020DC130020EE13002016
:10B0E000EF1300202DE9F04F2DED108B89B0B0EE5D
:10B0F00040BBB0EE41CBB0EE428BB0EE43DBD94863
:10B10000007820B909B0BDEC108BBDE8F08FD648AF
:10B11000008804287ED13BEE480BBDEEC00B10EE3C
:10B12000100A07B23BEE080BB7EE001B30EE010B26
:10B13000BDEEC00B10EE100A0FFA80F83CEE480B83
:10B14000BDEEC00B10EE100A0FFA80F93CEE080BB2
:10B15000B7EE001B30EE010BBDEEC00B10EE100A77
:10B160000FFA80FAC1480068874200D3CAE7B8F1F5
:10B17000000F00DAC6E7BE480068814500D3C1E78A
:10B18000BAF1000F00DABDE7002F00DA0027B74858
:10B190000068804504D3B5480088401E0FFA80F847
:10B1A000B9F1000F01DA4FF00009B148006882459B
:10B1B00004D3AF480088401E0FFA80FA3D464BE1A9
:10B1C0004E4644E100EE105AB8EEC00B30EE4BFB99
:10B1D00000EE106AB8EEC00B30EE4CEB2FEE0F1BFA
:10B1E0000EEE0E1BB0EE410B28F0CEF9B0EE40ABE8
:10B1F00000200890B6EE000B38EE000BB4EECA0B40
:10B20000F1EE10FA45D9B6EE000B38EE400BB4EE75
:10B21000CA0B00E024E1F1EE10FA0ED201200890F2
:10B22000B6EE000B38EE400B3AEE400BB7EE001BCB
:10B2300031EE400BB0EE409B2BE0B6EE000B3DEE46
:10B24000000BB4EECA0BF1EE10FA0FD8894804686F
:10B2500086480068400000FB064404EB450486482D
:10B260000078607085480078207012E0B6EE000B20
:10B270003DEE400BB4EECA0BF1EE10FA09D80120F6
:10B280000890B6EE000B3DEE400B3AEE400BB0EEF0
:10B29000409B089800287CD0DFF8D8B1DBF800404C
:10B2A000DFF8C8B1DBF800B04FEA4B0B0BFB0644EC
:10B2B00004EB450494F801C094F800E04FEA2C1B1D
:10B2C00000EE10BA0CF00F0B00EE90BA4FEA2E1BF6
:10B2D00002EE90BA0EF00F0B06EE10BADFF898B13E
:10B2E0009BF800B04FEA2B1B06EE90BADFF888B14E
:10B2F0009BF800B00BF00F0B01EE10BADFF87CB139
:10B300009BF800B04FEA2B1B01EE90BADFF86CB14E
:10B310009BF800B00BF00F0B02EE10BAB8EE663BD4
:10B3200029EE033BB7EE004B34EE494BB8EE405BE1
:10B3300004EE053BB0EE437BB8EE413B29EE033B08
:10B34000B7EE004B34EE494BB8EE605B04EE053BC4
:10B350008DED063BB8EE613B29EE033BB7EE004BAB
:10B3600034EE494BB8EE625B04EE053B8DED043BD9
:10B37000B8EE423B29EE033BB7EE004B34EE494BAF
:10B38000B8EE465B04EE053B8DED023BB0EE473B6D
:10B3900000E05AE0B6EE004B33EE043BBCEEC33B9C
:10B3A00013EE10BA0BF0FF009DED063BB6EE004B1E
:10B3B00033EE043BBCEEC33B13EE10BA0BF0FF01BF
:10B3C0009DED043BB6EE004B33EE043BBCEEC33BBD
:10B3D00013EE10BA0BF0FF029DED023BB6EE004BF0
:10B3E00033EE043BBCEEC33B13EE10BA0BF0FF038D
:10B3F000002800DA00200F2800DD0F20002900DAE5
:10B4000000210F2900DD0F21002A00DA00220F2A77
:10B4100000DD0F22002B00DA00230F2B00DD0F23AD
:10B4200001EB001B0BF0FF0BCDF804B003EB021B8C
:10B430000BF0FF0BCDF800B0DDF804B084F801B0DC
:10B44000DDF800B084F800B000BF701C06B25645AD
:10B450007FF7B8AE681C05B245457FF7B1AE00BFB7
:10B4600000BF4FE6D8130020E8130020E0130020AF
:10B47000E4130020DC130020EE130020EF13002063
:10B480002DE9F05F2DED0A0B2DED108BB8B0B0EE6D
:10B49000409BB0EE41ABB0EE43DBB0EE44EBF9487D
:10B4A000007828B938B0BDEC108B0AB0BDE8F09F29
:10B4B000F548008804287DD1B0EE000B8DEE001B0E
:10B4C0008DED361BB0EE000B8EEE001BB0EE41FB97
:10B4D0009DED361B21EE011B0FEE0F1BB0EE410B55
:10B4E00028F052F88DED340B9DED340B39EE400B06
:10B4F000BDEEC00B10EE100A07B29DED340B39EE15
:10B50000000BB7EE001B30EE010BBDEEC00B10EED2
:10B51000100A0FFA80F89DED340B3AEE400BBDEEA9
:10B52000C00B10EE100A0FFA80F99DED340B3AEEC5
:10B53000000BB7EE001B30EE010BBDEEC00B10EEA2
:10B54000100A0FFA80FAD1480068874200D3A9E7B1
:10B55000B8F1000F00DAA5E7CD480068814500D3B7
:10B56000A0E7BAF1000F00DA9CE7002F00DA00270D
:10B57000C6480068804504D3C4480088401E0FFABE
:10B5800080F8B9F1000F01DA4FF00009C0480068F7
:10B59000824504D3BE480088401E0FFA80FA9DED14
:10B5A0004C0B27F041FF8DED320B9DED4C0B27F03E
:10B5B00093FF00E01BE38DED300B9DED320B20EE91
:10B5C0000D1BB0EE002B81EE020B39EE40BB9DED62
:10B5D000300B20EE0D1BB0EE002B81EE020B3AEE8D
:10B5E000400B8DED2E0B9DED320B20EE0D1BB0EEC2
:10B5F000000B81EE002B32EE090B8DED2C0B9DED37
:10B60000300B20EE0D1BB0EE000B81EE002B32EE66
:10B610000A0B8DED2A0B9DED300B20EE0E0BB0EEDC
:10B62000001B80EE012B32EE09CB9DED320B20EE9C
:10B630000E1BB0EE000B81EE002B3AEE420B8DEDAF
:10B64000280B9DED300B20EE0E1BB0EE000B81EEB3
:10B65000002B39EE420B8DED260B9DED320B20EECB
:10B660000E0BB0EE001B80EE012B32EE0A0B8DEDBF
:10B67000240B9FED880B8DED220B9FED860B8DED3E
:10B68000200B3D46AFE24E46A8E2002015901490F4
:10B6900013900F900E900D9000EE105AB8EEC00B64
:10B6A0008DED1A0B00EE106AB8EEC00B8DED180B85
:10B6B0009DED2A0B9DED2E1B30EE411B9DED1A0BCF
:10B6C00021EE001B9DED2C0B30EE4B2B9DED180B4E
:10B6D00002EE401B9DED2C0B9DED2E2B00EE021B70
:10B6E0009DED2A0B00EE4B1B8DED1E1B9DED1E0BE1
:10B6F000B5EEC00BF1EE10FA05D29DED1E0BB1EECA
:10B70000400B8DED1E0B9DED2A1B9DED2E2B31EE7A
:10B71000421B21EE011B9DED2C2B32EE4B3B9DED90
:10B720002C2B32EE4B2B03EE021BB0EE410B27F01D
:10B730002BFF8DED1C0B9DED1E0B9DED1C1B80EE5C
:10B74000012B8DED222B9DED240B9DED281B30EE62
:10B75000411B9DED1A0B21EE000B9DED261B31EEDA
:10B760004C2B9DED181B02EE410B9DED261B9DED14
:10B77000282B01EE020B9DED241B01EE4C0B8DEDF1
:10B780001E0B9DED1E0BB5EEC00BF1EE10FA05D2AF
:10B790009DED1E0BB1EE400B8DED1E0B9DED241BA0
:10B7A0009DED282B31EE421B21EE011B9DED262B3A
:10B7B00032EE4C3B9DED262B32EE4C2B03EE021B62
:10B7C000B0EE410B27F0E0FE8DED1C0B9DED1E0B46
:10B7D0009DED1C1B80EE012B8DED202B9DED360B7E
:10B7E000B6EE001B30EE011B9DED200BB4EEC01B2E
:10B7F000F1EE10FA02D2012015905FE09DED360BBC
:10B80000B6EE001B30EE411B9DED200BB4EEC01BCD
:10B81000F1EE10FA02DD012014904FE001201390A8
:10B820009DED1A0B30EE4C2B9DED240B9DED281B4E
:10B8300030EE410B22EE000B9DED181B9DED282BE9
:10B8400031EE422B9DED261B31EE4C1B02EE410BDF
:10B850008DED160B9DED160BB5EEC00BF1EE10FA4B
:10B860001CD29DED200B9DED361B30EE410BB6EE4C
:10B87000001B30EE010BB7EE001B31EE400B8DEDDF
:10B88000100B1BE0D8130020E8130020E013002069
:10B89000E413002000000000000000009DED360BC6
:10B8A000B6EE001B30EE411B9DED200B30EE410B40
:10B8B000B7EE001B31EE400B8DED100B159810B15B
:10B8C00001200F9057E0B6EE000B3FEE001B9DED00
:10B8D000220BB4EEC01BF1EE10FA02D201200F9041
:10B8E00049E0B6EE000B3FEE401B9DED220BB4EE9F
:10B8F000C01BF1EE10FA02DD01200E903BE00120AA
:10B900000D909DED1A0B30EE4B2B9DED2A0B9DED0E
:10B910002E1B30EE410B22EE000B9DED181B9DED12
:10B920002E2B31EE422B9DED2C1B31EE4B1B02EEEC
:10B93000410B8DED160B9DED160BB5EEC00BF1EE28
:10B9400010FA0EDDB6EE000B3FEE401B9DED220B14
:10B9500030EE410BB7EE001B31EE400B8DED0A0BC4
:10B9600009E0B6EE000B3FEE401B9DED220B30EEE2
:10B97000410B8DED0A0B0020099083461FED3B8B98
:10B98000159840BB0F9830BB149868B10E9810B151
:10B99000012009901FE00D98E8B14FF0010B9DEDDB
:10B9A0000A0BB0EE408B16E01398A0B10E9830B1A0
:10B9B0004FF0010B9DED100BB0EE408B0BE00D989E
:10B9C00048B14FF0010B9DED100B9DED0A1B20EED1
:10B9D000010BB0EE408B099848B9BBF1000F16D0AF
:10B9E000B7EE000BB4EEC08BF1EE10FA0FDB81481E
:10B9F000046881480068400000FB064404EB4504ED
:10BA00007E48007860707E4800782070E4E0BBF1EA
:10BA1000000FFBD0B5EEC08BF1EE10FAF6DDDFF8CB
:10BA2000D4C1DCF80040DFF8D0C1DCF800C04FEA38
:10BA30004C0C0CFB064404EB450494F801E094F82C
:10BA400000C0CDF820C04FEA2E1C00EE10CA0EF048
:10BA50000F0C00EE90CADDF820C04FEA2C1C01EE5E
:10BA600010CADDF820C00CF00F0C01EE90CADFF810
:10BA70008CC19CF800C04FEA2C1C02EE10CADFF803
:10BA80007CC19CF800C00CF00F0C02EE90CADFF8ED
:10BA900070C19CF800C04FEA2C1C06EE10CADFF8FB
:10BAA00060C19CF800C00CF00F0C06EE90CAB8EE16
:10BAB000423B28EE033BB7EE004B34EE484BB8EE6A
:10BAC000405B04EE053BB0EE437BB8EE623B28EEF4
:10BAD000033BB7EE004B34EE484BB8EE605B04EE30
:10BAE000053B8DED063BB8EE463B28EE033BB7EE3B
:10BAF000004B34EE484BB8EE415B04EE053B8DED58
:10BB0000043BB8EE663B28EE033BB7EE004B34EE49
:10BB1000484BB8EE615B04EE053B8DED023BB0EEA9
:10BB2000473BB6EE004B33EE043BBCEEC33B13EE9B
:10BB300010CA0CF0FF009DED063BB6EE004B33EE55
:10BB4000043BBCEEC33B13EE10CA0CF0FF019DEDAD
:10BB5000043BB6EE004B33EE043BBCEEC33B13EEAE
:10BB600010CA0CF0FF029DED023BB6EE004B33EE27
:10BB7000043BBCEEC33B13EE10CA0CF0FF030028DD
:10BB800000DA00200F2800DD0F20002900DA002154
:10BB90000F2900DD0F21002A00DA00220F2A00DD24
:10BBA0000F22002B00DA00230F2B00DD0F2301EB07
:10BBB000001C0CF0FF0CCDF804C003EB021C0CF0D1
:10BBC000FF0CCDF800C0DDF804C084F801C0DDF83A
:10BBD00000C084F800C000BF701C06B256457FF755
:10BBE00054AD681C05B245457FF74DAD00BF00BFA1
:10BBF00058E40000DC130020E0130020EE130020C6
:10BC0000EF1300202DE9FF4F2DED028B8BB0834603
:10BC10000F46144694F8009094F801A0E178A078BB
:10BC200001EB002080B208906179207901EB0020BF
:10BC300080B20790E179A07901EB002080B20690F4
:10BC4000617A207A01EB002080B205900A2500205D
:10BC500002903EE00EF07CF9029805EB400014F8EB
:10BC60000080029805EB4000401C265CF21911B2DE
:10BC700008EB0B0210B2109AF7F734F9B9F1000F84
:10BC80000AD0C8EB4900401E584400B20490314627
:10BC9000109A0498F7F726F9BAF1000F0AD0C6EB0C
:10BCA0004A00401E384400B203904046109A03995F
:10BCB000F7F718F9B9F1000F07D0BAF1000F04D067
:10BCC000109ADDE90310F7F70DF90298401C80B2D5
:10BCD0000290089902988842BCDB0221089801FB77
:10BCE000005085B2002002905CE00EF031F902981D
:10BCF00000EB4000284414F80080029800EB40005C
:10BD00002844401C265C029800EB40002844801C1C
:10BD1000205C0A909DED0A0AB8EE400BB0EE408B15
:10BD20009FED960B88EE001BB0EE418BF21911B21D
:10BD300008EB0B0210B2B0EE480B109AF7F7DEF8E2
:10BD4000B9F1000F0DD0C8EB4900401E584400B2B5
:10BD50000490F01901B2B0EE480B109A0498F7F76E
:10BD6000CDF8BAF1000F0CD0C6EB4A00401E3844A3
:10BD700000B20390B0EE480B4046109A0399F7F7D3
:10BD8000BDF8B9F1000F09D0BAF1000F06D0B0EE3E
:10BD9000480B109ADDE90310F7F7B0F80298401C41
:10BDA00080B202900799029888429EDB079800EBC8
:10BDB0004000284485B20020029059E00EF0C8F8F7
:10BDC000029800EB4000284414F80080029800EB31
:10BDD00040002844401C265C029800EB40002844A8
:10BDE000801C205C09900020019039E0F21911B20A
:10BDF000019A42445A4410B2109AF7F773F8B9F115
:10BE0000000F0DD0C8EB4900401E0199401A58445C
:10BE100000B20490F01901B2109A0498F7F762F892
:10BE2000BAF1000F0DD0C6EB4A00401E384400B2F4
:10BE3000039001994144594408B2109A0399F7F7C5
:10BE400051F8B9F1000F07D0BAF1000F04D0109AE1
:10BE5000DDE90310F7F746F80198401C80B2019025
:10BE6000099901988842C1DB0298401C80B2029077
:10BE7000069902988842A1DB069800EB400028440E
:10BE800085B20020029070E00EF062F8029805EB97
:10BE9000800014F80080029805EB8000401C265CAE
:10BEA000029805EB8000801C205C0A909DED0A0A38
:10BEB000B8EE400BB0EE408B9FED300B88EE001BD0
:10BEC000B0EE418B029805EB8000C01C205C09900D
:10BED0000020019041E0F21911B2019A42445A4403
:10BEE00010B2B0EE480B109AF7F708F8B9F1000F4E
:10BEF0000FD0C8EB4900401E0199401A584400B2C7
:10BF00000490F01901B2B0EE480B109A0498F6F7BD
:10BF1000F5FFBAF1000F0FD0C6EB4A00401E3844BF
:10BF200000B2039001994144594408B2B0EE480B65
:10BF3000109A0399F6F7E2FFB9F1000F09D0BAF1B0
:10BF4000000F06D0B0EE480B109ADDE90310F6F7AB
:10BF5000D5FF0198401C80B2019009990198884250
:10BF6000B9DB0298401C80B2029005990298884281
:10BF70008ADB0BB0BDEC028BBDE8FF8F0000000038
:10BF800000E06F402DE9FF4104460D4616461F466E
:10BF9000102C71D2DFE804F0081018202830384047
:10BFA0004850586068717981684601F063FDDDE9A9
:10BFB0000001CDE902017AE0684601F067FDDDE9A4
:10BFC0000001CDE9020172E0684601F06BFDDDE998
:10BFD0000001CDE902016AE0684601F06FFDDDE98C
:10BFE0000001CDE9020162E0684601F073FDDDE980
:10BFF0000001CDE902015AE0684601F077FDDDE974
:10C000000001CDE9020152E0684601F07BFDDDE967
:10C010000001CDE902014AE0684601F07FFDDDE95B
:10C020000001CDE9020142E0684601F083FDDDE94F
:10C030000001CDE902013AE0684601F087FDDDE943
:10C040000001CDE9020132E0684601F08BFDDDE937
:10C050000001CDE902012AE0684601F08FFDDDE92B
:10C060000001CDE9020122E0684601F093FDDDE91F
:10C070000001CDE902011AE017E0684601F096FDE3
:10C08000DDE90001CDE9020111E0684601F09AFD09
:10C09000DDE90001CDE9020109E0684601F09EFDFD
:10C0A000DDE90001CDE9020101E0BDE8FF8100BF4B
:10C0B0009DF90D00304401B23B462846029AFFF735
:10C0C000A1FD00BFF1E72DE9FC4706460C461746E7
:10C0D00098463046F4F7DCF81FFA80F9002513E0A3
:10C0E000715D684601F0EAFB9DF90500384401B234
:10C0F00043462046009AFFF785FD9DF80400401C4A
:10C10000204404B2681C85B24D45E9DBBDE8FC87DC
:10C110002DE9FC4705460C4690469A4600262846DF
:10C12000F4F7B6F81FFA80F9002709E0E95D6846E0
:10C1300001F0C4FB9DF80400304486B2781C87B23D
:10C140004F45F3DB304606EBD071A4EB61010CB236
:10C15000002713E0E95D684601F0B0FB9DF905009A
:10C16000404401B253462046009AFFF74BFD9DF82C
:10C170000400401C204404B2781C87B24F45E9DB20
:10C18000BDE8FC872DE9FF4F87B005460C46904679
:10C19000DDE914AB00262846F4F77AF81FFA80F997
:10C1A000002709E0E95D05A801F088FB9DF818006B
:10C1B000304486B2781C87B24F45F3DB304606EB3D
:10C1C000D071A4EB61010CB2002719E0E95D05A86C
:10C1D00001F074FBDDE91610CDE900ABCDE90210EA
:10C1E0009DF91900404401B220460A9B059A00F0CF
:10C1F0000DF89DF81800401C204404B2781C87B24A
:10C200004F45E3DB0BB0BDE8F08F00002DE9FF4F99
:10C210002DED028B8BB080460E46144694F800A09C
:10C2200094F801B0E178A07801EB002080B208908A
:10C230006179207901EB002080B20790E179A07943
:10C2400001EB002080B20690617A207A01EB002099
:10C2500080B205904FF00A09002002904FE00DF0E7
:10C2600077FE029809EB4000275C029809EB40003A
:10C27000401C255C07EB08011A9881423BDB07EB69
:10C2800008011C98814236DCA9191B98814232DBD7
:10C29000A9191D9881422EDCAA1911B207EB0802D8
:10C2A00010B2109AF6F71EFEBAF1000F0AD0C7EBD3
:10C2B0004A00401E404400B204902946109A049857
:10C2C000F6F710FEBBF1000F0AD0C5EB4B00401E85
:10C2D000304400B203903846109A0399F6F702FEF4
:10C2E000BAF1000F07D0BBF1000F04D0109ADDE9BE
:10C2F0000310F6F7F7FD0298401C80B202900899EF
:10C3000002988842ABDB0221089801FB00901FFADB
:10C3100080F9002002906DE00DF01AFE029800EB0B
:10C3200040004844275C029800EB40004844401C11
:10C33000255C029800EB40004844801C205C0A9079
:10C340009DED0A0AB8EE400BB0EE408B9FEDB20BAC
:10C3500088EE001BB0EE418B07EB08011A98814272
:10C3600044DB07EB08011C9881423FDCA9191B98AC
:10C3700081423BDBA9191D98814237DCAA1911B211
:10C3800007EB080210B2B0EE480B109AF6F7B6FDB4
:10C39000BAF1000F0DD0C7EB4A00401E404400B276
:10C3A0000490A81901B2B0EE480B109A0498F6F761
:10C3B000A5FDBBF1000F0CD0C5EB4B00401E304477
:10C3C00000B20390B0EE480B3846109A0399F6F786
:10C3D00095FDBAF1000F09D0BBF1000F06D0B0EE09
:10C3E000480B109ADDE90310F6F788FD0298401C0F
:10C3F00080B202900799029888428DDB079800EB83
:10C40000400048441FFA80F9002002906AE00DF0D5
:10C410009FFD029800EB40004844275C029800EB27
:10C4200040004844401C255C029800EB4000484412
:10C43000801C205C0990002001904BE007EB080174
:10C440001A98814242DB07EB08011C9881423DDCCF
:10C45000A9191B98814239DBA9191D98814235DC45
:10C46000AA1911B2019A3A44424410B2109AF6F74E
:10C4700039FDBAF1000F0DD0C7EB4A00401E0199FB
:10C48000401A404400B20490A81901B2109A0498CE
:10C49000F6F728FDBBF1000F0DD0C5EB4B00401E99
:10C4A000304400B2039001993944414408B2109AD3
:10C4B0000399F6F717FDBAF1000F07D0BBF1000F93
:10C4C00004D0109ADDE90310F6F70CFD0198401C2A
:10C4D00080B20190099901988842AFDB0298401C14
:10C4E00080B2029006990298884290DB069800EB91
:10C4F000400048441FFA80F90020029081E00DF0CE
:10C5000027FD029809EB8000275C029809EB800068
:10C51000401C255C029809EB8000801C205C0A907E
:10C520009DED0A0AB8EE400BB0EE408B9FED3A0B42
:10C5300088EE001BB0EE418B029809EB8000C01C16
:10C54000205C09900020019053E007EB08011A9845
:10C5500081424ADB07EB08011C98814245DCA9199E
:10C560001B98814241DBA9191D9881423DDCAA1923
:10C5700011B2019A3A44424410B2B0EE480B109AFC
:10C58000F6F7BCFCBAF1000F0FD0C7EB4A00401E13
:10C590000199401A404400B20490A81901B2B0EECB
:10C5A000480B109A0498F6F7A9FCBBF1000F0FD0C6
:10C5B000C5EB4B00401E304400B203900199394452
:10C5C000414408B2B0EE480B109A0399F6F796FC76
:10C5D000BAF1000F09D0BBF1000F06D0B0EE480B46
:10C5E000109ADDE90310F6F789FC0198401C80B22F
:10C5F0000190099901988842A7DB0298401C80B2FB
:10C600000290059902988842FFF679AF0BB0BDEC15
:10C61000028BBDE8FF8F00000000000000E06F40CB
:10C620002DE9F04F8BB082468B46144694F800807B
:10C6300094F80190E178A07801EB002080B2099095
:10C640006179207901EB002080B20890E179A0792E
:10C6500001EB002080B20790617A207A01EB002084
:10C6600080B206900A270020039052E00DF070FC83
:10C67000039807EB4000255C039807EB4000401C43
:10C68000265C0020009006EB0B0291B205EB0A023B
:10C69000019090B200231A4600F0F8FBB8F1000FA9
:10C6A0000FD0C5EB4800401E504402B20592002056
:10C6B0000090B1B20190059A90B200231A4600F0A2
:10C6C000E5FBB9F1000F0FD0C6EB4900401E5844FE
:10C6D00002B20492002000900190049A91B2A8B294
:10C6E00000231A4600F0D2FBB8F1000F0DD0B9F1CB
:10C6F000000F0AD0002000900190049A91B2059A90
:10C7000090B200231A4600F0C1FB0398401C80B28F
:10C710000390099903988842A8DB0221099801FB3C
:10C72000007087B20020039054E00DF011FC0398D4
:10C7300000EB40003844255C039800EB400038448F
:10C74000401C265C0020009006EB0B0291B205EB2A
:10C750000A02019090B200231A4600F097FBB8F14C
:10C76000000F0FD0C5EB4800401E504400B20590AA
:10C7700000200090B1B20190059A90B200231A46B1
:10C7800000F084FBB9F1000F0FD0C6EB4900401E4A
:10C79000584400B20490002000900190049A91B295
:10C7A000A8B200231A4600F071FBB8F1000F0DD0BB
:10C7B000B9F1000F0AD0002000900190049A91B2C4
:10C7C000059A90B200231A4600F060FB0398401CC3
:10C7D00080B20390089903988842A6DB089800EB82
:10C7E0004000384487B2002003906EE00DF0B0FBAB
:10C7F000039800EB40003844255C039800EB4000B0
:10C800003844401C265C039800EB40003844801CF0
:10C81000205C0A90002002904FE00020009006EB80
:10C820000B0291B20190029A2A44524490B2002322
:10C830001A4600F02BFBB8F1000F13D0C5EB4800EF
:10C84000401E0299401A504400B20590002000900A
:10C8500006EB0B0291B20190059A90B200231A46A2
:10C8600000F014FBB9F1000F12D0C6EB4900401ED6
:10C87000584400B20490002000900190049A91B2B4
:10C88000029A2A44524490B200231A4600F0FEFA5B
:10C89000B8F1000F0DD0B9F1000F0AD000200090C0
:10C8A0000190049A91B2059A90B200231A4600F0C2
:10C8B000EDFA0298401C80B202900A9902988842D0
:10C8C000ABDB0398401C80B2039007990398884221
:10C8D0008CDB079800EB4000384487B200200390BF
:10C8E0006BE00DF035FB039807EB8000255C0398A7
:10C8F00007EB8000401C265C039807EB8000C01CFF
:10C90000205C0A90002002904FE00020009006EB8F
:10C910000B0291B20190029A2A44524490B2002331
:10C920001A4600F0B3FAB8F1000F13D0C5EB480077
:10C93000401E0299401A504400B205900020009019
:10C9400006EB0B0291B20190059A90B200231A46B1
:10C9500000F09CFAB9F1000F12D0C6EB4900401E5E
:10C96000584400B20490002000900190049A91B2C3
:10C97000029A2A44524490B200231A4600F086FAE2
:10C98000B8F1000F0DD0B9F1000F0AD000200090CF
:10C990000190049A91B2059A90B200231A4600F0D1
:10C9A00075FA0298401C80B202900A990298884257
:10C9B000ABDB0398401C80B2039006990398884231
:10C9C0008FDB0BB0BDE8F08F2DE9FF4F82B00E4634
:10C9D000174698460025C8F100047800C0F1020906
:10C9E000DFED361AB0EE610ADFED341AF0EE610ABF
:10C9F000DFED321AB0EE611A01EE907AF8EE611AAC
:10CA0000F0EE610A01EE908AF8EE611AB0EE611A5A
:10CA1000C1EE201AB0EE610A00BF01EE905AF8EEA6
:10CA2000E11A81EE802AFCEEC21A11EE900A400053
:10CA3000401C80B2019001EE905AF8EEE11A81EEAE
:10CA4000802AFCEEC21A11EE900A0299081A1FFA07
:10CA500080FB01985844401E80B20090301903B208
:10CA6000301901B2009802B20FFA8BF0FEF76CF8A1
:10CA7000301B03B2301B01B2009802B20FFA8BF0E8
:10CA8000FEF762F8CA46AA450BDC681C0546012180
:10CA900001EB40008144EC4203D1A24501DC4FF0A0
:10CAA000000AA24505DD601C0446012101EB40009F
:10CAB0008144002CB1DD06B0BDE8F08F000000001D
:10CAC0002DE9F04F04460D4616461F4621480078D2
:10CAD00008B9BDE8F08FA019401E1FFA80FAE819C6
:10CAE000401E1FFA80FB1C480068824504D31A4888
:10CAF0000088401E1FFA80FA18480068834504D356
:10CB000016480088401E1FFA80FB06B9E1E707B906
:10CB1000DFE711480068844200D3DAE70F48006875
:10CB2000854200D3D5E7A8460FE0A14607E041467D
:10CB3000484600F007F909F101001FFA80F9D145D4
:10CB4000F5DD08F101001FFA80F8D845EDDD00BFE2
:10CB500000BFBEE7D8130020E0130020E41300203C
:10CB60002DE9F0431148007808B9BDE8F0830026AC
:10CB700000270F480088401E1FFA80F80D480088E3
:10CB8000401E1FFA80F93C460BE0354605E0214681
:10CB9000284600F0D7F8681C85B24545F7DD601CD3
:10CBA00084B24C45F1DD00BF00BFDEE7D8130020A2
:10CBB000E0130020E413002070B503460C462C4817
:10CBC0000078002852D02B48006883424ED22A4871
:10CBD000006884424AD22948008890B928480168F0
:10CBE00024480068800000FB041101EB8301C87831
:10CBF000107088785070487890700878D070012054
:10CC000070BD1E480088012814D11D4801681948CC
:10CC1000006800EB400000FB041103EB43000144FB
:10CC2000FF20107088785070487890700878D07025
:10CC30000120E5E711480088042816D11048016852
:10CC40000C480068400000FB041101EB43014D78E3
:10CC50000E782809107005F00F00507030099070A0
:10CC600006F00F00D0700120CAE700BF0020C7E720
:10CC7000D8130020E0130020E4130020E813002064
:10CC8000DC1300200148008880B27047E4130020C4
:10CC90000148008880B27047E01300200149086015
:10CCA00070470000F013002030B50A4C20700A4C89
:10CCB00021700A4C22700A4C237000F0F00404EB3F
:10CCC0002114084D2C7002F0F00404EB2314064DDF
:10CCD0002C7030BDEA130020EB130020EC13002071
:10CCE000ED130020EE130020EF13002010B586B0E6
:10CCF000044600200E49087021466846F5F7D8FA28
:10CD0000009808B1012000E0002009490870094995
:10CD100000980860BDF8080007490860BDF80A00DF
:10CD20000649086006490398088006B010BD000057
:10CD3000D8130020DC130020E0130020E4130020AF
:10CD4000E81300200A462B49097801B970472A499F
:10CD50000968884200D3F9E7284909688A4200D364
:10CD6000F4E727490988A9B9264B1968224B1B68A3
:10CD70009B0003FB021101EB8001234B1B78CB705E
:10CD8000224B1B788B70224B1B784B70214B1B78EE
:10CD90000B702CE01A490988012914D1194B196824
:10CDA000154B1B6803EB430303FB021100EB40032D
:10CDB0001944164B1B788B70154B1B784B70154B19
:10CDC0001B780B7013E00E49098804290FD10D4B15
:10CDD0001968094B1B685B0003FB021101EB400162
:10CDE0000D4B1B784B700D4B1B780B7000BF00BFB9
:10CDF000ACE70000D8130020E0130020E41300206B
:10CE0000E8130020DC130020EA130020EB130020BD
:10CE1000EC130020ED130020EE130020EF13002090
:10CE200000B5B5EEC01BF1EE10FA09DBB6EE002B33
:10CE300031EE022BBDEEC22B12EE102A12B208E028
:10CE4000B6EE002B31EE422BBDEEC22B12EE102AB5
:10CE500012B291B2B5EEC00BF1EE10FA09DBB6EEEC
:10CE6000002B30EE022BBDEEC22B12EE102A12B2B6
:10CE700008E0B6EE002B30EE422BBDEEC22B12EED8
:10CE8000102A12B290B2FFF75DFF00BDF0B50C465C
:10CE9000DDE905562549097801B9F0BD244909683D
:10CEA000884200D3F9E7234909688C4200D3F4E7AC
:10CEB0002149098869B9214F39681D4F3F68BF0072
:10CEC00007FB041101EB8001CA708B704D700E706E
:10CED0002AE01949098801290ED1184F3968144FE1
:10CEE0003F6807EB470707FB041100EB4007394495
:10CEF0008B704D700E7017E00F490988042913D10B
:10CF00000E4F39680A4F3F687F0007FB041101EBA1
:10CF1000400102F0F00707EB23174F7005F0F00710
:10CF200007EB26170F7000BF00BFB6E7D81300202D
:10CF3000E0130020E4130020E8130020DC1300209D
:10CF40002DE9F0470D46DDE9087C0A9C0126002109
:10CF50009CE006EA0508B8F1000F75D0D0F8008013
:10CF60004FEA410A4FF0030909FA0AF928EA0908C9
:10CF7000C0F8008002F003084FEA410908FA09F8F6
:10CF8000D0F8009048EA0908C0F80080D0F8048082
:10CF90004FF0010909FA01F928EA0908C0F80480EC
:10CFA00003F0010808FA01F8D0F8049048EA0908EB
:10CFB000C0F80480D0F808804FEA410A4FF0030916
:10CFC00009FA0AF928EA0908C0F8088007F00308F6
:10CFD0004FEA410908FA09F8D0F8089048EA090828
:10CFE000C0F80880D0F80C804FEA410A4FF00309DE
:10CFF00009FA0AF928EA0908C0F80C800CF00308BD
:10D000004FEA410908FA09F8D0F80C9048EA0908F3
:10D01000C0F80C80082918DAD0F820804FEA810A7D
:10D020004FF00F0909FA0AF928EA0908C0F8208028
:10D0300004F00F084FEA810908FA09F8D0F82090A7
:10D0400048EA0908C0F820801BE0D0F82480A1F14C
:10D0500008094FEA890A4FF00F0909FA0AF928EA84
:10D060000908C0F8248004F00F08A1F108094FEA6C
:10D07000890908FA09F8D0F8249048EA0908C0F8A4
:10D080002480760001F1010808F0FF011029FFF665
:10D0900060AFBDE8F08700002DE9F34F2DED048B64
:10D0A000A1B025980F90BDF89800ADF84000FE485B
:10D0B000006813F05FF90E90FC4800788DF842008C
:10D0C000FB480088ADF844004FF0FF30ADF8460053
:10D0D000ADF84800ADF84A0000201390401EADF8AE
:10D0E000500000201590401EADF858009FEDF10B48
:10D0F0008DED180BADF858009FEDEE0B8DED1C0B70
:10D10000ADF878009DF89800002837D0E7480078FF
:10D1100038B90020E9490880E5490880E84813F05B
:10D1200061F9E748006813F025F9E649E34A1288F7
:10D1300041F83200BDF89400E04A128801EBC201C8
:10D140008880BDF89600DF49DC4A128801EBC201F5
:10D15000C880DA480088401CD84908800846008802
:10D160000A2801DB00200880D14800880A2804DA58
:10D17000CF480088401CCE4908808EE100200D90E9
:10D18000CB480088042874DB0120ADF84800CB4868
:10D19000008804B2002007900120059000207DE067
:10D1A000059921B101B2ADF8461000210591611E2B
:10D1B0000CB2002C00DA092498B9C24901EBC40171
:10D1C000B1F80490BF4951F834100991BD4901EB01
:10D1D000C401C9880C91BB4901EBC401C9880B91FA
:10D1E00056E0B84901EBC401CA880C998A4204DDB3
:10D1F000B44901EBC401C9880C91B24901EBC401E7
:10D20000CA880B998A4204DAAE4901EBC401C98885
:10D210000B91AC4901EBC401B1F80480A94901EBC1
:10D22000C401C9880A91A74951F83410089101280E
:10D2300014D1A44901EBC4018988B94202DD01215E
:10D24000069125E09F4901EBC4018988B94202DAC1
:10D25000002106911CE00121079122E0994901EB90
:10D26000C4018988B94205DD069989B90121079170
:10D2700017E0C4E0934901EBC4018988B94204DA9C
:10D28000069929B1012107910BE00121079108E0DE
:10D290008C4901EBC4018F88411C88B20428FFF639
:10D2A0007FAF00BF079800287ED10120ADF84A006B
:10D2B000DDE90810461A1396002E76DD40F6C410FC
:10D2C000864272DA0120ADF85000A8EB090005B2E1
:10D2D000002D01DA684205B20020ADF850000A2D99
:10D2E00072DD0120ADF85800DDE90B10401A0FFA8D
:10D2F00080FA00EE10AAB8EEC00B8DED180B554564
:10D3000058DD0120ADF8680000EE105AB8EEC00BF1
:10D31000B0EE408B00EE106AB8EEC00B88EE001B3A
:10D32000B0EE418B8DED1C8B9FED670BB4EEC08B87
:10D33000F1EE10FA25DDADF87800C84503DDB1EE59
:10D34000480BB0EE408B02208DF80000ADF8028053
:10D350000A98ADF804008DED028B9FED5D0B28EE71
:10D36000009BBDEEC90B10EE10BA5A4601210720F2
:10D3700005F002FA01200D909DE80F00F6F78AFAF9
:10D3800017E00020ADF878004FF47A7B00EE10BA79
:10D39000B8EEC00B20EE080BBDEEC00B10EE10BABD
:10D3A0005A460221072001E020E016E005F0E4F9EA
:10D3B00000BF07E00020ADF868000022062107202A
:10D3C00005F0DAF908E0FFE70020ADF858002A463A
:10D3D0000321072005F0D0F907E00020ADF8500048
:10D3E00032460421072005F0C7F907E00020ADF818
:10D3F0004A0000220521072005F0BEF902E00020C6
:10D40000ADF848000D98E0BB29480088002843DDAE
:10D41000274800880A283FDA2848008800283BDD92
:10D42000284903C9CDE90B0124480088401E25493D
:10D4300001EBC00103C9CDE90901BDF82800BDF821
:10D440003010401A04B2BDF82A00BDF83210401A5C
:10D4500005B2002C01DA604204B2002D01DA684204
:10D4600005B20A2C17DA0A2D15DA01208DF8100002
:10D4700014488088ADF812001248C088ADF8140036
:10D4800000E009E09FED0B0B8DED060B04A80FC823
:10D49000F6F700FA00BF00BF00BF9DF898000349EF
:10D4A00008700D48007819E0CC130020C01300204C
:10D4B000BC1300200000000000000000BE1300208C
:10D4C000C4130020D8060120B81E85EB51B89E3F3A
:10D4D0000000000000408F40D0130020F0B9124936
:10D4E000098801EBC101114A02EBC10048220EA9D3
:10D4F000F2F79EFE0C480088401C0B490880084645
:10D500000088642801DB002008800948008864281E
:10D5100004DA07480088401C0549088021B0BDECAA
:10D52000048BBDE8FC8F0000C813002028070120F1
:10D53000CA13002010B5024812F054FF10BD0000BD
:10D54000CC13002010B503211DA01CF0E7FE1D48E0
:10D55000008800B21CF010FF05211BA01CF0DEFEAD
:10D560001B48008800B21CF007FF5D201CF0C0FEC5
:10D57000002421E05B201CF0BBFE164931F834107A
:10D5800008B21CF0F9FE2C201CF0B2FE114901EB90
:10D59000C401898808B21CF0EFFE2C201CF0A8FE04
:10D5A0000C4901EBC401C98808B21CF0E5FE5D20FE
:10D5B0001CF09EFE601C84B20A2CDBDB10BD000058
:10D5C0005B633D00BC1300202C6964783D000000C3
:10D5D000BE130020D8060120014609480078032820
:10D5E0000BDA0848064A127840F8221004480078FE
:10D5F000401C034A1070012070470020FCE7000027
:10D60000D11300204823012000200349088003494A
:10D610000880012070470000CA130020C8130020B2
:10D6200010B51548007828BB1448008800B214498A
:10D6300008801248008800B2124908800F4800880C
:10D64000642805DB1048008800B21049088002E019
:10D6500000200E4908800120074908700948B0F9E8
:10D6600000200BA10F4825F0ADFC0E481CF086FFF2
:10D67000012010BD0020FCE7D0130020CA130020B9
:10D68000D4130020D6130020C8130020D21300208A
:10D690005B4C6F6744756D705374617274696E672B
:10D6A00025645D005423012010B50648007838B188
:10D6B00000200449087004A01CF060FF012010BD88
:10D6C0000020FCE7D01300205B4C6F6744756D7041
:10D6D000436F6D706C6574655D00000000B5A9B0A6
:10D6E0003848007800286AD03748B0F90000002890
:10D6F00002DCFFF7D9FF62E03448B0F9000000EB2C
:10D70000C000334A02EBC001482216A8F2F790FD90
:10D71000BDF9980014909DED240B8DED120BBDF911
:10D72000880010909DED200B8DED0E0BBDF978005B
:10D73000BDF970201B9B1D99CDE90932CDE90B1075
:10D74000BDF96A00BDF96810BDF96620BDF8643006
:10D75000CDE90532CDE907109DF8620016A9CA8807
:10D76000BDF85C1016AB1B7ACDE90131CDE9032081
:10D77000169800901748B0F900001349B1F900104D
:10D78000421A1448B0F900301349144825F01AFC25
:10D7900012481CF0F3FE0D480088401C00B20B49F3
:10D7A00008800846B0F90000642801DB00200880EA
:10D7B00005480088401E00B20349088000BF29B018
:10D7C00000BD0000D0130020D6130020D21300208B
:10D7D00028070120D4130020609B0D08542301204A
:10D7E00010B5FFF77BFF10BDBF207047F0B5ADF55A
:10D7F000017D06460C461546ADF8F8412046E11776
:10D8000004EB9161C1F38F11ADF8FA112046E117D5
:10D8100004EB91618911A4EB811189B2ADF8FC117F
:10D820000020ADF8FE01BDF8FA017C9015480068B3
:10D8300000F5C06000EB452000F110014FF4F872D4
:10D840006846F2F7F5FC0F48006800F5C06000EB91
:10D85000452797E80F00F3F7F1FA10B10120ADF872
:10D86000FE01BDF8FE01C0F1010080B2ADF800027A
:10D870007E9830607F987060BDF8000230810DF5B1
:10D88000017DF0BD9C14002008B50B48006890F89D
:10D89000000430B100208DF8000001208DF8010057
:10D8A00005E001208DF8000000208DF80100BDF892
:10D8B0000010084608BD00009C1400203CB504463A
:10D8C0000D46A5F120003B286FD2DFE800F0BBC772
:10D8D000C7C7C7C3C7C7C7C7C7C7B7C7AFB31E2266
:10D8E000262A2E32363A3E42BFC7C7C7C7C7C746E9
:10D8F0004A4E52565A5E62666A6F73777B7F8387A1
:10D900008B8F93979B9FA3A7AB00204600F0B2F8A4
:10D910003CBD204600F0BAF8FAE7204600F0C2F815
:10D92000F6E7204600F0CAF8F2E7204600F0D2F809
:10D93000EEE7204600F0DAF8EAE7204600F0E2F8E9
:10D94000E6E7204600F0EAF8E2E7204600F0F2F8C9
:10D95000DEE7204600F0FAF8DAE7204600F002F9A8
:10D96000D6E7204600F00AF9D2E7204600F012F987
:10D97000CEE7204600F01AF9CAE7204600F022F967
:10D98000C6E7204600F02AF9C2E7204600F032F947
:10D99000BEE7204600F03AF9BAE7204600F042F927
:10D9A000B6E7204600F04AF9B2E757E0204600F01B
:10D9B00051F9ADE7204600F059F9A9E7204600F0FB
:10D9C00061F9A5E7204600F069F9A1E7204600F0DB
:10D9D00071F99DE7204600F079F999E7204600F0BB
:10D9E00081F995E7204600F089F991E7204600F09B
:10D9F00091F98DE7204600F099F989E7204600F07B
:10DA0000A1F985E7204600F0A9F981E7204600F05A
:10DA1000B1F97DE7204600F0B9F979E7204600F03A
:10DA2000C1F975E7204600F0C9F971E7204600F01A
:10DA300001FA6DE7204600F0E5F969E7204600F0BD
:10DA4000D5F965E7204600F001FA61E7204600F0CD
:10DA5000C1F95DE7204600F0E1F959E7044903C93F
:10DA6000CDE90001DDE90001C4E9000100BF4FE795
:10DA70004C990D080CB5044A06CACDE90012DDE93F
:10DA80000012C0E900120CBD04980D080CB5044A40
:10DA900006CACDE90012DDE90012C0E900120CBD92
:10DAA0000C980D080CB5044A06CACDE90012DDE950
:10DAB0000012C0E900120CBD14980D080CB5044A00
:10DAC00006CACDE90012DDE90012C0E900120CBD62
:10DAD0001C980D080CB5044A06CACDE90012DDE910
:10DAE0000012C0E900120CBD24980D080CB5044AC0
:10DAF00006CACDE90012DDE90012C0E900120CBD32
:10DB00002C980D080CB5044A06CACDE90012DDE9CF
:10DB10000012C0E900120CBD34980D080CB5044A7F
:10DB200006CACDE90012DDE90012C0E900120CBD01
:10DB30003C980D080CB5044A06CACDE90012DDE98F
:10DB40000012C0E900120CBD44980D080CB5044A3F
:10DB500006CACDE90012DDE90012C0E900120CBDD1
:10DB60004C980D080CB5044A06CACDE90012DDE94F
:10DB70000012C0E900120CBD54980D080CB5044AFF
:10DB800006CACDE90012DDE90012C0E900120CBDA1
:10DB90005C980D080CB5044A06CACDE90012DDE90F
:10DBA0000012C0E900120CBD64980D080CB5044ABF
:10DBB00006CACDE90012DDE90012C0E900120CBD71
:10DBC0006C980D080CB5044A06CACDE90012DDE9CF
:10DBD0000012C0E900120CBD74980D080CB5044A7F
:10DBE00006CACDE90012DDE90012C0E900120CBD41
:10DBF0007C980D080CB5044A06CACDE90012DDE98F
:10DC00000012C0E900120CBD84980D080CB5044A3E
:10DC100006CACDE90012DDE90012C0E900120CBD10
:10DC20008C980D080CB5044A06CACDE90012DDE94E
:10DC30000012C0E900120CBD94980D080CB5044AFE
:10DC400006CACDE90012DDE90012C0E900120CBDE0
:10DC50009C980D080CB5044A06CACDE90012DDE90E
:10DC60000012C0E900120CBDA4980D080CB5044ABE
:10DC700006CACDE90012DDE90012C0E900120CBDB0
:10DC8000AC980D080CB5044A06CACDE90012DDE9CE
:10DC90000012C0E900120CBDB4980D080CB5044A7E
:10DCA00006CACDE90012DDE90012C0E900120CBD80
:10DCB000BC980D080CB5044A06CACDE90012DDE98E
:10DCC0000012C0E900120CBDC4980D080CB5044A3E
:10DCD00006CACDE90012DDE90012C0E900120CBD50
:10DCE000CC980D080CB5044A06CACDE90012DDE94E
:10DCF0000012C0E900120CBDD4980D080CB5044AFE
:10DD000006CACDE90012DDE90012C0E900120CBD1F
:10DD1000DC980D080CB5044A06CACDE90012DDE90D
:10DD20000012C0E900120CBDE4980D080CB5044ABD
:10DD300006CACDE90012DDE90012C0E900120CBDEF
:10DD4000EC980D080CB5044A06CACDE90012DDE9CD
:10DD50000012C0E900120CBDF4980D080CB5044A7D
:10DD600006CACDE90012DDE90012C0E900120CBDBF
:10DD7000FC980D080CB5044A06CACDE90012DDE98D
:10DD80000012C0E900120CBD04990D080CB5044A3C
:10DD900006CACDE90012DDE90012C0E900120CBD8F
:10DDA0000C990D080CB5044A06CACDE90012DDE94C
:10DDB0000012C0E900120CBD14990D080CB5044AFC
:10DDC00006CACDE90012DDE90012C0E900120CBD5F
:10DDD0001C990D080CB5044A06CACDE90012DDE90C
:10DDE0000012C0E900120CBD3C990D080CB5044AA4
:10DDF00006CACDE90012DDE90012C0E900120CBD2F
:10DE000034990D080CB5044A06CACDE90012DDE9C3
:10DE10000012C0E900120CBD2C990D080CB5044A83
:10DE200006CACDE90012DDE90012C0E900120CBDFE
:10DE300044990D080CB5044A06CACDE90012DDE983
:10DE40000012C0E900120CBD24990D08024A06CA4E
:10DE5000C0E9001270470000901C00200048704785
:10DE60009BC70C0800487047775E0D080048704754
:10DE700002E00C080048704756D90C08004870476B
:10DE8000C6E60C080048704716500D080048704759
:10DE9000E1D10C080048704791490D0800487047CF
:10DEA000F64C0D08004870479F350D080048704734
:10DEB000FB360D080048704744380D08004870478D
:10DEC000D3390D08004870479F3C0D080048704743
:10DED000A33D0D080048704742140D0800487047E4
:10DEE000EFEF0C080048704701400D0800487047EC
:10DEF00080180D080048704740540D0800487047CE
:10DF0000F6BD0C080048704737C10C080048704740
:10DF1000951D0D0800487047D81D0D080048704732
:10DF2000D9B00C080048704743B10C08004870474E
:10DF300083B10C0800487047CFB10C080048704707
:10DF400021B20C080048704770B20C0800487047B6
:10DF5000BFB20C080048704719B30C08004870475E
:10DF600059B30C0800487047BAB30C080048704712
:10DF70005AB00C0800487047C1B00C080048704700
:10DF8000F7D70C08004870476CC90C080048704768
:10DF90004FC00C080048704787F30C0800487047D2
:10DFA000B5F70C08004870475EFB0C080048704746
:10DFB00025FE0C08004870476C000D0800487047AB
:10DFC000CD010D0800487047A8030D0800487047B0
:10DFD0001E060D08004870474A090D0800487047A2
:10DFE000590D0D080048704774430D08F0B5ADF5A4
:10DFF000037D05460E4614462246314680A8FFF7AB
:10E00000F5FB0027BDF802027C901A48006800F575
:10E01000C06000EB442000F110014FF4F872684634
:10E02000F2F706F91348006800F5C06000EB442CD5
:10E030009CE80F00F2F702FF00B1012740F2D51073
:10E0400078430C49096801F5206101EB8020BDF897
:10E05000021200EB4120BDF8041200EBC100016880
:10E060007E9140687F907E9828607F9868600DF56B
:10E07000037DF0BD9C14002018B5024600200090DE
:10E0800000BF92F83C00012801D1022018BD0120F8
:10E0900082F83C0000BF0868092822D91068C068CF
:10E0A0000B780A3B03EB43040723A3409843136810
:10E0B000D8604F4B0868984207D11068C0680B7A47
:10E0C00040EA03601368D8601FE00B780A3B03EB5B
:10E0D0004303886898401368DB6818431368D86066
:10E0E00013E0106800690B7803EB43040723A34097
:10E0F0009843136818610B7803EB430388689840D2
:10E1000013681B691843136818614868072817D2F9
:10E110001068406B0B795B1E03EB83041F23A34045
:10E12000984313685863088880B20B795B1E03EB31
:10E130008303984013685B6B18431368586331E09E
:10E1400048680D2817D21068006B0B79DB1F03EBB2
:10E1500083041F23A340984313681863088880B280
:10E160000B79DB1F03EB8303984013681B6B184389
:10E170001368186316E01068C06A0B790D3B03EB57
:10E1800083041F23A34098431368D862088880B291
:10E190000B790D3B03EB830398401368DB6A18434C
:10E1A0001368D862134B1068984208D10868122887
:10E1B00005D11148006840F48000C3F804030D4BFA
:10E1C000106898420DD10A4B0868984202D008683E
:10E1D000112806D10848006840F40000054BC3F838
:10E1E000040300BF002082F83C0000BF00BF4DE7E1
:10E1F0001200001000200140042301402DE9FE4FD1
:10E2000004460026206C00283ED1606484F83C005F
:10E210002D492068084450B3B0F5007F32D12B4817
:10E22000006840F48060294908600846006800F4EE
:10E23000806526481438006840F0200023491439CE
:10E2400008600846006800F0200503274FF000082A
:10E250004FF003094FF0000A4FF0000B43463A46D7
:10E2600009151B488DE8000EFEF76AFE0BE0174803
:10E27000006840F48070154908600846006800F4A2
:10E28000807500E000BF00BF206C00F0100088B96E
:10E29000206C20F4885040F0020020642046F2F701
:10E2A000C5FB00206064206C20F0020040F00100FB
:10E2B000206400E0012600BF002084F83C0000BF7D
:10E2C0003046BDE8FE8F000000E0FEBF443802404B
:10E2D00000140240014600BF91F83C00012801D122
:10E2E00002207047012081F83C0000BF0868806868
:10E2F00000F0010028B90868806840F001000A6851
:10E30000906000BF002081F83C0000BF6FF0220049
:10E310000A6810600020E4E7014691F83500022801
:10E3200003D08020486501207047052081F8350022
:10E330000868006820F001000A6810600020F3E718
:10E3400070B504460CB9012070BD94F83500022860
:10E3500000D1F9E72068006820F00100216808601A
:10E360000020216808602168486021688860216871
:10E37000C860216808612120216848612046F3F7C0
:10E3800085FE054694F85C103F208840A860002078
:10E39000606584F8350000BF84F8340000BF00BF1A
:10E3A000D2E7000070B5044600250CB9012070BD0D
:10E3B00000BF002084F8340000BF022084F835003C
:10E3C0002068006820F001002168086000BF206814
:10E3D000006800F001000028F9D120680568224893
:10E3E0000540D4E901010843E16808432169084375
:10E3F00061690843A1690843E1690843216A084348
:10E400000543606A042803D1D4E90B01084305439E
:10E41000206805602068456925F00705606A0543A6
:10E42000606A04280DD1A06A0543E06A48B120461D
:10E43000F3F746FE28B140206065012084F83500DE
:10E44000B5E7206845612046F3F720FE064694F8BC
:10E450005C103F208840B06000206065012084F897
:10E4600035000020A3E700003F8010E010B504460F
:10E47000D4F894021CF02BFD10BD10B504460CB965
:10E48000012010BD032084F89102204600F011FB0A
:10E4900020681EF0DFF9002084F8910200BFF0E749
:10E4A00010B50446D4F894021CF030FD10BD10B530
:10E4B000044620681EF0E0FA10BD10B5044620683E
:10E4C0001EF0E0FA10BD024601EB810302F13800B4
:10E4D00000EBC30090F824007047024601EB810373
:10E4E00002F1380000EBC3004069704770B5044684
:10E4F0000D46002600BF94F89002012801D10220A9
:10E5000070BD012084F8900200BF294620681EF0EB
:10E51000C7FA00BF002084F8900200BF3046EFE742
:10E520002DE9FE4F04460D4616461F46DDE90D9ABD
:10E53000DDF830804FF0000B00BF94F89002012806
:10E5400002D10220BDE8FE8F012084F8900200BFB6
:10E5500005EB850104F1380000F8317005EB850109
:10E5600000EBC100A0F808A005EB850104F138001C
:10E5700000EBC100457005EB850104F1380000EBAC
:10E58000C10080F8079006F07F0105EB850204F1D9
:10E59000380000EBC2008170C6F3C01105EB8502A4
:10E5A00004F1380000EBC200C17005EB850104F1F5
:10E5B000380000EBC10080F804808DE800073B467E
:10E5C0003246294620681EF028FB834600BF002003
:10E5D00084F8900200BF5846B4E770472DE9F05F19
:10E5E00004460D4616461F46DDE90BB9DDF834A09A
:10E5F000DDF8288005EB850104F1380000EBC1004F
:10E60000C67005EB850104F1380000EBC100C7714D
:10E61000B8F1000F08D1032105EB850204F13800A1
:10E6200000EBC200817207E0022105EB850204F1D4
:10E63000380000EBC200817237B1012F7DD0022F6C
:10E640003DD0032F3AD182E0B8F1010F36D1AEBBF5
:10E65000B9F1000F07D1012105EB850204F1380063
:10E6600000EBC200417605EB850104F1380000EBB8
:10E67000C100407E40B9002105EB850204F138005D
:10E6800000EBC200817207E0022105EB850204F174
:10E69000380000EBC200817205EB850104F13800FF
:10E6A00000EBC10090F82400022807D005EB85019B
:10E6B00004F1380000EBC10080F805A085E05EBBE6
:10E6C00005EB850104F1380000EBC100407E40B944
:10E6D000002105EB850204F1380000EBC2008172D5
:10E6E00007E0022105EB850204F1380000EBC200CF
:10E6F000817205EB850104F1380000EBC10090F850
:10E700002400022822D005EB850104F1380000EB3B
:10E71000C10080F805A019E005EB850104F138007F
:10E7200000EBC100007E48B9002105EB850204F131
:10E73000380000EBC200817208E03DE0022105EBE9
:10E74000850204F1380000EBC20081723DE0CEB9D1
:10E7500005EB850104F1380000EBC100407E40B9B3
:10E76000002105EB850204F1380000EBC200817244
:10E7700021E0022105EB850204F1380000EBC20024
:10E78000817218E005EB850104F1380000EBC1004F
:10E79000007E40B9002105EB850204F1380000EB52
:10E7A000C200817207E0022105EB850204F1380006
:10E7B00000EBC200817208E0002105EB850204F144
:10E7C000380000EBC200817200BF00BF05EB85017D
:10E7D00004F1380000EBC100C0F80CB005EB850176
:10E7E00004F1380000EBC100C0F81090002105EBE7
:10E7F000850204F1380000EBC20080F8241005EB1C
:10E80000850204F1380000EBC200416105EB85018F
:10E8100004F1380000EBC1004570002105EB8502D2
:10E8200004F1380000EBC20080F82510227C05EBD3
:10E83000850C04F1380303EBCC0120681EF0B8FA14
:10E84000BDE8F09F2DE9F041044626680025002729
:10E8500020681EF020F901287ED172480088401CF3
:10E860007049088020681EF0C1FC08B9BDE8F0813D
:10E870006D4840696D49884202D063206C49088028
:10E8800020681EF0B3FC00F40010B0F5001F08D1A2
:10E8900068480088401C674908804FF400102168D0
:10E8A000486120681EF0A2FC00F48010B0F5801FC3
:10E8B00008D161480088401C5F4908804FF48010EF
:10E8C0002168486120681EF091FC00F08060B0F182
:10E8D000806F08D159480088401C584908804FF083
:10E8E00080602168486120681EF080FC00F0020012
:10E8F000022807D152480088401C51490880022054
:10E900002168486120681EF071FC00F00050B0F1F1
:10E91000005F15D14B480088401C4A490880D6F852
:10E92000400420F02E00C6F840042046FFF7B8FD52
:10E93000012120681EF0A9FB4FF0005021684861BA
:10E9400020681EF053FC00F08070B0F1807F09D188
:10E950003D480088401C00E061E03B4908802046BB
:10E9600001F04AF820681EF041FC00F00800082879
:10E970000AD136480088401C34490880204600F0FF
:10E98000D3F808202168486120681EF02FFC00F0B1
:10E990000070B0F1007F27D12D480088401C2C4921
:10E9A000088020681EF0FDF90746002515E00120CB
:10E9B000A840384080B106F5A06000EB4510006823
:10E9C00000F4004020B1E9B2204600F022FB03E051
:10E9D000E9B2204600F097FD6D1CA068A842E6D879
:10E9E0004FF000702168486120681EF0FFFB00F0C6
:10E9F0001000102813D117480088401C15490880C2
:10EA00002068806920F0100021688861204601F0AC
:10EA1000A3F82068806940F010002168886100BF79
:10EA200024E70000CC17002000000440330000045D
:10EA3000E2170020D0170020D2170020D4170020A2
:10EA4000D6170020D8170020DA170020DC17002086
:10EA5000DE170020E017002010B58AB0044614B974
:10EA600001200AB010BD032084F89102204600F076
:10EA700021F820681DF0EEFE282204F110016846FE
:10EA8000F1F7D6FB94E80F001DF086FE0121206807
:10EA90001EF0FDFB282204F110016846F1F7C8FBC7
:10EAA00094E80F001EF076FA012084F8910200200D
:10EAB000D7E770472DE9FE4F82464FF00009144812
:10EAC000006840F00200124908600846006800F043
:10EAD000020902240025032600274FF00C082B46CC
:10EAE00022464FF470410B488DE8C001FEF728FA2A
:10EAF0000748006840F00050054908600846006873
:10EB000000F00059200304490860BDE8FE8F0000B2
:10EB1000303802400004024008E100E010B504462D
:10EB200020681EF099FB10BD10B50446D4F894027D
:10EB30001CF057FA10BD10B5044600BF94F89002BF
:10EB4000012801D1022010BD012084F8900200BFED
:10EB500020681DF0DBFE012120681DF0B5FE00BF1E
:10EB6000002084F8900200BF00BFECE710B5044617
:10EB700000BF94F89002012801D1022010BD0120AD
:10EB800084F8900200BF20681EF099FB00BF0020AF
:10EB900084F8900200BF00BFF0E701460846002855
:10EBA00009DB00F01F0301229A4043099B0003F197
:10EBB000E023C3F8002100BF704700002DE9F04FAB
:10EBC00005460E461746002000BF24490968C1F3D8
:10EBD0000221084629460346B446B8461C46C4F1FD
:10EBE000070BBBF1040F02D94FF0040B01E0C4F195
:10EBF000070BDA4604F1040BBBF1070F02D24FF00A
:10EC0000000B01E0A4F1030BD9464FF0010B0BFA06
:10EC10000AFBABF1010B0BEA0C0B0BFA09FB4FF0F3
:10EC2000010E0EFA09FEAEF1010E0EEA080E4BEAD5
:10EC30000E0200BF002904DB13071C0E084B5C54B6
:10EC400009E013074FEA136C044B0C3301F00F0477
:10EC5000241F03F804C000BFBDE8F08F0CED00E0F6
:10EC600000E400E000BFFEE7816B014A11607047DD
:10EC7000E8160020F8B504460D46042700260020BB
:10EC800000902A466946204617F026FB064616B134
:10EC9000A06B3043A0630098C0F343273846F8BD0B
:10ECA0002DE9F04190B006460D469046002400271D
:10ECB00042466946304617F085FA074667B140F28A
:10ECC000FF502C490860B06B3843B063012086F8D0
:10ECD000340010B0BDE8F0810098C0F381142C70AE
:10ECE0000098C0F340146C700098C0F307444FF6CE
:10ECF000FF7000EA042068800098040E68882043B2
:10ED000068800198C4B2200668600198C0F30724A7
:10ED1000686840EA044068600198C0F30744686886
:10ED200040EA042068600198040E68682043686027
:10ED30000298C4B22C720298C0F307246C72029835
:10ED4000C0F30354AC720298040E4FF6FF7000EA51
:10ED50000420A8810398C4B2A8892043A8810398FD
:10ED6000C0F38524AC730398C0F30124EC73002036
:10ED7000AFE70000381C01402DE9F04387B004469E
:10ED8000884616461D46DDF838900027B8F1000F7A
:10ED900007D1A06B40F00060A063012007B0BDE880
:10EDA000F08394F83400012865D10020A063711924
:10EDB000E06D814205D9A06B40F00070A063012096
:10EDC000ECE7032084F8340000202168C862C4F80E
:10EDD00028806802E0622068C06B48F22A1108436C
:10EDE0002168C863606C012800D076024FF0FF30C4
:10EDF000019068020290902003900220049000206D
:10EE000005900120069001A9206816F01FFE4A46D1
:10EE10004FF40071206816F06DFC074657B140F2C0
:10EE2000FF5021688863A06B3843A063012084F8F9
:10EE30003400B3E7012D08D90A2020634A46314641
:10EE4000206816F095FC074607E0092020634A4633
:10EE50003146206816F0ABFC074657B140F2FF5030
:10EE600021688863A06B3843A063012084F83400D4
:10EE700094E7002092E7022090E7000038B50446AE
:10EE80000C4800780A2814D10B48007830B10F20C4
:10EE9000084908700020084908700AE0002003466D
:10EEA0000246042100908020F4F7F4FE102001496E
:10EEB000087038BDE01600200917002038B5044658
:10EEC0000C480078032814D10B48007830B1042096
:10EED000084908700020084908700AE0002003462D
:10EEE0000322092100908020F4F7D4FE0520014977
:10EEF000087038BDE0160020081700202DE9F04307
:10EF000087B00446894616461D460E9F4FF00008FE
:10EF1000B9F1000F08D1A06B40F00060A0630120A0
:10EF2000387007B0BDE8F08394F8340001286CD144
:10EF30000020A0637119E06D814207D9A06B40F0F9
:10EF40000070A063072038700120EAE7032084F8EE
:10EF5000340000202168C862C4F820906802606212
:10EF60002068C06B44F21A1108432168C863606CC2
:10EF7000012800D076023A464FF40071206816F05E
:10EF8000B9FB8046B8F1000F0BD040F2FF5021686A
:10EF90008863A06B40EA0800A063012084F8340075
:10EFA000BFE7012D08D9282020633A463146206862
:10EFB00016F00EFD804607E0182020633A463146E1
:10EFC000206816F024FD8046B8F1000F0BD040F207
:10EFD000FF5021688863A06B40EA0800A06301200D
:10EFE00084F834009DE74FF0FF30019068020290F2
:10EFF000902003900020049005900120069001A924
:10F00000206816F023FD00208BE70220387000BF37
:10F0100087E72DE9F04106460C463568002705F5DF
:10F02000A06000EB4410806800F0040090B104215F
:10F0300005F5A06000EB4410816005F5A06000EBD1
:10F040004410C06840F0020105F5A06000EB4410D8
:10F05000C16069E005F5A06000EB4410806800F035
:10F06000200030B1202105F5A06000EB4410816044
:10F070005AE005F5A06000EB4410806800F008003D
:10F0800028B305F5A06000EB4410C06840F0020111
:10F0900005F5A06000EB4410C160052104EB84027B
:10F0A00006F1380000EBC20080F82510102105F5AC
:10F0B000A06000EB44108160082105F5A06000EB22
:10F0C00044108160214630681DF0EAFC2CE005F513
:10F0D000A06000EB4410806800F4806020B305F568
:10F0E000A06000EB4410C06840F0020105F5A0608C
:10F0F00000EB4410C160214630681DF0D1FC1021A6
:10F1000005F5A06000EB44108160082104EB840247
:10F1100006F1380000EBC20080F82510C90105F5A2
:10F12000A06000EB4410816005F5A06000EB441086
:10F13000806800F40070B8B105F5A06000EB4410E1
:10F14000C06840F0020105F5A06000EB4410C1600A
:10F15000214630681DF0A4FC4FF4007105F5A06055
:10F1600000EB44108160CCE105F5A06000EB441099
:10F17000806800F0010000287DD03069A8B104EB60
:10F18000840106F1380000EBC100016905F5A060BB
:10F1900000EB44100069C0F31200091A04EB84026A
:10F1A00006F1380000EBC2004161012104EB84024A
:10F1B00006F1380000EBC20080F82510002104EBB6
:10F1C000840206F1380000EBC2000162012105F55E
:10F1D000A06000EB4410816004EB840106F138006C
:10F1E00000EBC100C07940B104EB840106F13800A6
:10F1F00000EBC100C079022816D105F5A06000EB34
:10F200004410C06840F0020105F5A06000EB441016
:10F21000C160214630681DF043FC102105F5A06057
:10F2200000EB441081602BE004EB840106F1380010
:10F2300000EBC100C079032822D105F5A06000EBE6
:10F240004410006840F0005105F5A06000EB441048
:10F250000160012104EB840206F1380000EBC200DA
:10F2600080F8241004EB840106F1380000EBC100A3
:10F2700090F8242000E014E021463046FFF7ADF975
:10F2800004EB840106F1380000EBC100007E80F041
:10F29000010104EB840206F1380000EBC2000176A4
:10F2A0002FE105F5A06000EB4410806800F002003B
:10F2B000002871D005F5A06000EB4410C06820F074
:10F2C000020105F5A06000EB4410C16004EB84016D
:10F2D00006F1380000EBC10090F82500012809D1A3
:10F2E000012104EB840206F1380000EBC20080F833
:10F2F000241069E004EB840106F1380000EBC10042
:10F3000090F82500052809D1052104EB840206F1B7
:10F31000380000EBC20080F8241055E004EB8401B3
:10F3200006F1380000EBC10090F82500062809D04E
:10F3300004EB840106F1380000EBC10090F82500D1
:10F34000082841D104EB840106F1380000EBC1002C
:10F3500004EB8401026A06F1380000EBC100006A88
:10F36000401C04EB840306F1380101EBC301086281
:10F37000032A12D9002104EB840206F1380000EBC5
:10F38000C2000162042104EB840206F1380000EBA4
:10F39000C20080F8241009E029E0022104EB840275
:10F3A00006F1380000EBC20080F8241005F5A060DB
:10F3B00000EB4410076827F0804747F0004705F549
:10F3C000A06000EB44100760022105F5A06000EB8F
:10F3D0004410816004EB840106F1380000EBC100A9
:10F3E00090F8242021463046FFF7F7F889E005F52C
:10F3F000A06000EB4410806800F0800070B305F559
:10F40000A06000EB4410C06840F0020105F5A06068
:10F4100000EB4410C16004EB840106F1380000EBFE
:10F42000C100006A401C04EB840206F1380101EBC4
:10F43000C2010862062104EB840206F1380000EBE9
:10F44000C20080F82510214630681DF029FB80217C
:10F4500005F5A06000EB4410816052E0FFE705F580
:10F46000A06000EB4410806800F01000E0B304EBF3
:10F47000840106F1380000EBC100C079032810D1E7
:10F4800005F5A06000EB4410C06840F0020105F5EE
:10F49000A06000EB4410C160214630681DF000FB05
:10F4A0001EE004EB840106F1380000EBC100C079D6
:10F4B00040B104EB840106F1380000EBC100C079D3
:10F4C00002280DD105F5A06000EB4410076827F075
:10F4D000804747F0004705F5A06000EB4410076047
:10F4E000032104EB840200E00BE006F1380000EB9E
:10F4F000C20080F82510102105F5A06000EB441033
:10F500008160BDE8F0812DE9F04105460C462E688A
:10F51000002706F5A06000EB4410806800F00400AE
:10F5200090B1042106F5A06000EB4410816006F55F
:10F53000A06000EB4410C06840F0020106F5A06036
:10F5400000EB4410C16054E206F5A06000EB4410EB
:10F55000806800F0200088B3202106F5A06000EB51
:10F560004410816004EB840105F1380000EBC10018
:10F5700040790128E7D1042104EB840205F1380029
:10F5800000EBC20080F8251006F5A06000EB4410E7
:10F59000C06840F0020106F5A06000EB4410C160B5
:10F5A000214628681DF07CFA022104EB840205F153
:10F5B000380000EBC20080F824101AE2FFE706F5DD
:10F5C000A06000EB4410806800F0400038B30421D4
:10F5D00004EB840205F1380000EBC20080F825102E
:10F5E000002104EB840205F1380000EBC200016247
:10F5F00006F5A06000EB4410C06840F0020106F57B
:10F60000A06000EB4410C160214628681DF048FA54
:10F61000402106F5A06000EB44108160E9E106F5A9
:10F62000A06000EB4410806800F40070B8B106F5EB
:10F63000A06000EB4410C06840F0020106F5A06035
:10F6400000EB4410C160214628681DF029FA4FF4F0
:10F65000007106F5A06000EB44108160C9E106F579
:10F66000A06000EB4410806800F0010030B300217E
:10F6700004EB840205F1380000EBC200016206F5DC
:10F68000A06000EB4410C06840F0020106F5A060E5
:10F6900000EB4410C160214628681DF001FA0121E9
:10F6A00006F5A06000EB4410816004EB840205F1D4
:10F6B000380000EBC20080F825109AE106F5A06042
:10F6C00000EB4410806800F00800F8B1082106F54E
:10F6D000A06000EB4410816006F5A06000EB4410D0
:10F6E000C06840F0020106F5A06000EB4410C16064
:10F6F000214628681DF0D4F9052104EB840205F1A8
:10F70000380000EBC20080F8251072E106F5A06019
:10F7100000EB4410806800F0100038B3002104EBC7
:10F72000840205F1380000EBC200016206F5A0601A
:10F7300000EB4410C06840F0020106F5A06000EB49
:10F740004410C160214628681DF0AAF9032104EB8A
:10F75000840205F1380000EBC20080F8251010216A
:10F7600006F5A06000EB4410816042E106F5A06060
:10F7700000EB4410806800F08000F8B106F5A0604E
:10F7800000EB4410C06840F0020106F5A06000EBF9
:10F790004410C160214628681DF082F9062104EB5F
:10F7A000840205F1380000EBC20080F825108021AA
:10F7B00006F5A06000EB441081601AE106F5A06038
:10F7C00000EB4410806800F4806028B306F5A06068
:10F7D00000EB4410C06840F0020106F5A06000EBA9
:10F7E0004410C160214628681DF05AF9102106F521
:10F7F000A06000EB44108160890106F5A06000EB79
:10F8000044108160082104EB840205F1380000EB0C
:10F81000C20080F82510ECE006F5A06000EB441073
:10F82000806800F0020000289FD006F5A06000EB81
:10F830004410C06820F0020106F5A06000EB4410FF
:10F84000C16004EB840105F1380000EBC10090F8C1
:10F850002500012822D1012104EB840205F13800A2
:10F8600000EBC20080F8241004EB840105F138009D
:10F8700000EBC100C07902280FD104EB840105F12F
:10F88000380000EBC100407E80F0010104EB8402EF
:10F8900005F1380000EBC200417698E004EB8401EA
:10F8A00005F1380000EBC10090F82500032809D1CC
:10F8B000022104EB840205F1380000EBC20080F85D
:10F8C000241084E004EB840105F1380000EBC10052
:10F8D00090F82500042811D1022104EB840205F1DF
:10F8E000380000EBC20080F82410002104EB8402F1
:10F8F00005F1380000EBC200417168E004EB8401BF
:10F9000005F1380000EBC10090F82500052809D169
:10F91000052104EB840205F1380000EBC20080F8F9
:10F92000241054E004EB840105F1380000EBC10021
:10F9300090F82500062809D004EB840105F1380071
:10F9400000EBC10090F82500082840D104EB8401A9
:10F9500005F1380000EBC10004EB8401026A05F1F7
:10F96000380000EBC100006A401C04EB840305F181
:10F97000380101EBC3010862032A11D9002104EB0D
:10F98000840205F1380000EBC2000162042104EB9F
:10F99000840205F1380000EBC20080F8241008E072
:10F9A000022104EB840205F1380000EBC20080F86C
:10F9B000241006F5A06000EB4410076827F080478C
:10F9C00047F0004706F5A06000EB441007600221F5
:10F9D00006F5A06000EB4410816004EB840105F1A2
:10F9E000380000EBC10090F8242021462846FEF79D
:10F9F000F4FDBDE8F08100007CB504464C48008869
:10FA0000401C4B4908802568D5F840040190D5F882
:10FA100040040090009820F02E000090019800F023
:10FA2000020002281AD143480088401C414908803E
:10FA3000019800F0010068B13F480088401C3E4931
:10FA400008802068806920F0005021688861204685
:10FA5000FEF70CFD009840F002000090019800F0C5
:10FA60000800082851D135480088401C33490880D7
:10FA7000009840F008000090019800F0040004286D
:10FA800037D12F480088401C2D490880A0690228E2
:10FA90001ED12C480088401C2A490880019800F497
:10FAA000C020B0F5802F09D127480088401C264986
:10FAB0000880022120681DF0E8FA16E0234800883B
:10FAC000401C22490880012120681DF0DEFA0CE06C
:10FAD000E068032809D11E480088401C1C490880A2
:10FAE0004EF6602140F2044041512046FEF7BEFC34
:10FAF0000BE0D5F8400420F02E00C5F84004206843
:10FB0000806940F0005021688861019800F0200071
:10FB1000202808D10F480088401C0E490880009812
:10FB200040F0200000900098C5F840047CBD000023
:10FB3000E4170020E6170020E8170020EA1700204D
:10FB4000EC170020EE170020F0170020F21700201D
:10FB5000F4170020F61700202DE9F04705462F681E
:10FB60000024A046A1462868D0F8208008F00F04A1
:10FB7000C8F3434AC8F30A16BAF1020F09D0BAF122
:10FB8000030F66D0BAF1050F61D0BAF1070F5FD14C
:10FB900060E0002E5AD004EB840105F1380000EB40
:10FBA000C100C068E8B3B2B204EB840C05F13803BD
:10FBB00003EBCC03D96828681DF01EFB04EB84011D
:10FBC00005F1380000EBC100C068811904EB840224
:10FBD00005F1380000EBC200C16004EB840105F1BF
:10FBE000380000EBC1004069811904EB840205F183
:10FBF000380000EBC200416107F5A06000EB441043
:10FC000000691649084060B107F5A06000EB441098
:10FC1000D0F8009029F0804949F0004907F5A0602C
:10FC200000E013E000EB4410C0F8009004EB840106
:10FC300005F1380000EBC100007E80F0010104EB0B
:10FC4000840205F1380000EBC200017603E002E017
:10FC500000BF00BF00BF00BFBDE8F0870000F81F75
:10FC600010B50DF041FC04461CB918F0B9F901209B
:10FC700010BD0020FCE7000010B5104991F82200EB
:10FC80000DF052FD28B90D4991F822000DF03DFD0F
:10FC900010B10DF051FE10E0084991F822000DF06E
:10FCA0004DFD50B10548408E4FF6FF71884202D19C
:10FCB0000CF008FE01E00DF023FC10BD080D022041
:10FCC00000B58BB000200A900521EEA009F028FEB7
:10FCD00038B102F047FD12F069FD01200A9002F0F0
:10FCE00051BB0921E9A009F01BFE30B118F0A2FBBD
:10FCF00012F046FD01200A90F1E70B21E6A009F081
:10FD00000FFE30B1F1F760FE12F01AFD01200A90EB
:10FD1000E5E70D21E3A009F003FE20B112F010FD8C
:10FD200001200A90DBE70C21E2A009F0F9FD30B1D7
:10FD3000F1F756FE12F046FD01200A90CFE70E21A2
:10FD4000E0A009F0EDFD20B112F03CFD01200A9089
:10FD5000C5E70C21DFA009F0E3FD30B112F066FD2C
:10FD600012F0B6FC01200A90B9E70B21DCA009F0E3
:10FD7000D7FD20B112F0C2FC01200A90AFE70421A8
:10FD8000DAA009F0B1FD98B104200190002209A980
:10FD900001A809F02BFF0028A1D0BDF82400C0B2B3
:10FDA000009002F0FDFB002899D001200A9096E710
:10FDB0000821D0A009F098FDD0B1082001900022C0
:10FDC00009A901A809F012FF002888D0BDF9240074
:10FDD000002884DBBDF924000E288DDA0020C849F4
:10FDE000BDF92420885412F0CBFC01200A9076E75C
:10FDF0000721C4A009F078FD70B30720019001220B
:10FE000009A901A809F0F2FE00288BD0BDF9240051
:10FE1000002887DBBDF924000E288FDA002208A90C
:10FE200001A809F0E3FE002888D00120B449BDF9FB
:10FE3000242088540020B549BDF9242021F812005F
:10FE4000BDF82000B249BDF9242021F8120012F0BB
:10FE500097FC01200A9042E70921AEA009F044FD79
:10FE6000A8B30020009009200190012209A901A84F
:10FE700009F0BCFE50B3BDF9240010B101281AD11D
:10FE80000CE00022694601A809F0B0FE28B1BDF9D6
:10FE90000000A349088001200A900DE00022694675
:10FEA00001A809F0A3FE28B1BDF900009D49088012
:10FEB00001200A9000E000BF00BF0A9830B1012085
:10FEC0009949BDF92420885412F03AFC07E7FFE76E
:10FED0000A2196A009F008FDD0B10A200190002265
:10FEE00009A901A809F082FE0028B4D0BDF92400B8
:10FEF0000028B0DBBDF924000228ACDA00208A49D2
:10FF0000BDF92420885412F01BFC01200A90E6E67B
:10FF1000092189A009F0E8FCD0B109200190002254
:10FF200009A901A809F062FE002894D0BDF92400B7
:10FF3000002890DBBDF924000B288CDA01208149D0
:10FF4000BDF92420885412F03DFC01200A90C6E639
:10FF50000A217DA009F0C8FCD0B10A20019000223E
:10FF600009A901A809F042FE0028AFD0BDF924007C
:10FF70000028ABDBBDF924000B28A7DA002071496B
:10FF8000BDF92420885412F01DFC01200A90A6E639
:10FF9000082170A009F0A8FCD0B10820019000222F
:10FFA00009A901A809F022FE00288FD0BDF924007C
:10FFB00000288BDBBDF924000D2887DA0120684971
:10FFC000BDF92420885412F083FB01200A9086E6B4
:10FFD000092164A009F088FCD0B109200190002219
:10FFE00009A901A809F002FE002890D0BDF924005B
:10FFF00000288CDBBDF924000D2888DA0020584940
:020000040802F0
:10000000BDF92420885412F063FB01200A9066E6B3
:10001000092157A009F068FCC8B10920019000220D
:1000200009A901A809F0E2FD002890D0BDF924003B
:1000300000288CDBBDF924000D2888DABDF82400E7
:1000400080B2009012F00AFB01200A9047E60421DA
:100050004AA009F049FC002899D00420019002220E
:1000600009A901A809F0C2FD002890D0BDF924001B
:10007000AA2801F09C8203DCAA2882F0828181E018
:10008000DAE100005245534554000000504F4C4CFB
:10009000535F4F4646000000494E4A454354535F64
:1000A0004F464600494E4A454354535F51554552C9
:1000B0005900000053574954434845535F4F464643
:1000C0000000000053574954434845535F5155457C
:1000D000525900004556454E54535F4F4646000066
:1000E00046494E4745525052494E540052454144AC
:1000F00000000000504F4C4C5F4F4646000000008F
:10010000BE270120504F4C4C5F4F4E0086270120E8
:10011000A2270120494E4A4543545F4F4E0000003C
:10012000061400200814002004140020494E4A45FB
:1001300043545F4F464600005357495443485F4F6E
:100140004E000000CC2701205357495443485F4FCD
:10015000464600004556454E545F4F4E0000000095
:10016000742801204556454E545F4F464600000016
:100170004556454E545F47455400000043414C4CA2
:1001800000000000810000BF794449688F440000EE
:1001900060050000760500008A0500009E0500004D
:1001A000AE050000BE050000CE050000DE05000023
:1001B000EE050000FE0500000E0600001E06000011
:1001C0002E0600003E0600005E0600006E060000DF
:1001D0007E0600008E0600009E060000AE060000AF
:1001E000C2060000E6060000FA0600001E07000036
:1001F00032070000460700005A0700006A070000A7
:100200008E070000A2070000B6070000C607000026
:10021000D6070000FA070000300800005008000070
:100220006008000092080000A6080000D80800003E
:10023000EC0800000009000010090000240900007B
:10024000380900005C090000700900008409000002
:1002500094090000A4090000B4090000C4090000CA
:10026000D8090000E8090000F8090000080A0000A9
:10027000260A00003A0A00004E0A0000620A000046
:10028000760A00008A0A00009E0A0000B20A0000F6
:10029000C60A0000DA0A0000EE0A0000020B0000A5
:1002A000120B0000260B00003A0B00004E0B000062
:1002B0005E0B00006E0B0000820B0000960B00002E
:1002C000AA0B0000CE0B0000E20B0000120C000095
:1002D000420C0000560C00006A0C00007E0C00006E
:1002E000920C0000A60C0000BA0C0000CA0C000022
:1002F000EE0C0000220D0000360D00004A0D00003B
:100300005E0D0000720D0000860D00009A0D0000C9
:10031000AE0D0000C20D0000D60D0000EA0D000079
:10032000FE0D0000120E0000260E00003A0E000026
:100330004E0E0000620E0000760E00008A0E0000D5
:100340009E0E0000B20E0000C60E0000DA0E000085
:10035000EE0E0000120F0000360F00005A0F0000D2
:100360007E0F0000B20F0000C60F0000DA0F000081
:10037000EE0F000002100000161000002A1000000E
:100380003E10000052100000661000007A100000BD
:100390008E100000A2100000B6100000CA1000006D
:1003A0000E1100003E110000521100006611000005
:1003B0007A1100008E110000A2110000B611000099
:1003C000CA110000DE110000F21100000612000048
:1003D0001A1200002E1200004212000056120000F5
:1003E0006A1200007E12000092120000A6120000A5
:1003F000BA120000CE120000E2120000F612000055
:10040000061300001A1300003A1300004E130000F8
:10041000621300007613000086130000961300009C
:10042000A6130000BA130000CE130000E213000070
:10043000F61300000A140000AB38A92881F0A18748
:10044000810000BF794449688F44000076110000A4
:100450008A1100009E110000B2110000C6110000B8
:10046000DA110000EE110000021200001612000066
:100470002A1200003E120000521200006612000014
:100480007A1200008E120000A2120000B6120000C4
:10049000CA120000DE120000F21200000613000073
:1004A0001A1300002E130000421300005613000020
:1004B0006A1300007E13000092130000A6130000D0
:1004C000BA130000CE130000E2130000F613000080
:1004D0000A1400001E14000032140000461400002C
:1004E0005A1400006E1400008214000096140000DC
:1004F000AA140000BE140000D2140000E61400008C
:10050000FA1400000E150000221500003615000038
:100510004A1500005E1500007215000086150000E7
:100520009A150000AE150000C2150000D615000097
:10053000EA150000FE150000121600002616000045
:100540003A1600004E1600006216000076160000F3
:100550008A1600009E160000B2160000C6160000A3
:10056000DA160000EE160000021700001617000051
:100570002A1700003E1700005217000066170000FF
:100580007A1700008E170000A2170000B2170000B3
:10059000C2170000D6170000EA170000FE1700007F
:1005A0000E1800002418000036180000481800003B
:1005B0005A1800006C1800008218000098180000FB
:1005C000AA180000C0180000D6180000EC1800009F
:1005D00002190000181900002E190000441900002B
:1005E0005A19000070190000861900009C190000BB
:1005F000B2190000C8190000DE190000F41900004B
:100600000A1A0000201A0000361A00004C1A0000D6
:10061000621A0000781A00008E1A0000A41A000066
:10062000BA1A0000CC1A0000DE1A0000F41A00000A
:100630000A1B00003C1B00005E1B0000701B00003A
:10064000821B0000941B0000AA1B0000C01B0000BE
:10065000D61B0000EC1B0000FE1B0000101C00005D
:10066000261C00003C1C0000521C0000681C0000FE
:100670007E1C0000901C0000A61C0000BC1C00009A
:10068000D21C0000E81C0000FE1C0000141D00002D
:100690002A1D0000401D0000561D00006C1D0000BA
:1006A000821D0000981D0000AE1D0000C41D00004A
:1006B000DA1D0000EC1D0000021E0000181E0000E4
:1006C0002E1E0000441E00005A1E0000701E000076
:1006D000861E00009C1E0000B21E0000C81E000006
:1006E000DE1E0000F41E00000A1F0000201F000094
:1006F000FDF77AF801460090002011F073FF012009
:100700000A9001F03EBEF6F777F80146009001200E
:1007100011F00EFF01200A90F3E7F6F767F80146A3
:100720000090022011F05EFF01200A90E9E7F6F741
:1007300007F9032011F0E8FE01200A90E1E7F6F73F
:10074000ACF8042011F0E0FE01200A90D9E7F6F79A
:1007500095F8052011F0D8FE01200A90D1E7F6F7B0
:10076000A1F8062011F0D0FE01200A90C9E7F6F7A3
:100770008FF8072011F0C8FE01200A90C1E7F6F7B4
:1007800082F8082011F0C0FE01200A90B9E7F4F7C2
:1007900078FD092011F0B8FE01200A90B1E7F4F7C6
:1007A00075FD0A2011F0B0FE01200A90A9E7F4F7C8
:1007B00081FD0B2011F0A8FE01200A90A1E7F4F7BB
:1007C0006AFD0C2011F0A0FE01200A9099E700229A
:1007D00006A901A809F0B2FA40B1BDF81800F4F773
:1007E0005FFD0D2011F090FE01200A9089E7F4F7DB
:1007F00039FD0E2011F088FE01200A9081E7F4F700
:100800003BFD0F2011F080FE01200A9079E7F4F7FC
:100810002EFD102011F078FE01200A9071E7F6F706
:1008200099F8112011F070FE01200A9069E703F099
:10083000CDFC122011F068FE01200A9061E703F060
:100840009FFC01460090132011F072FE01200A90D7
:1008500057E7002204A901A809F0C8F950B1BDF872
:100860001000C0B2009003F095FC142011F04CFE73
:1008700001200A9045E703F043FC01460090152053
:1008800011F056FE01200A903BE7002204A901A8BE
:1008900009F0ACF950B1BDF81000C0B2009003F0FF
:1008A00039FC162011F030FE01200A9029E703F0F0
:1008B00037FC01460090172011F03AFE01200A9003
:1008C0001FE703F06DFC01460090182011F030FE88
:1008D00001200A9015E703F06FFC014600901920F3
:1008E00011F026FE01200A900BE71FF03FFC1A20B2
:1008F00011F00AFE01200A9003E7002204A901A8D2
:1009000009F074F950B1BDF81000C0B200901FF0AA
:1009100019FC1B2011F0F8FD01200A90F1E61FF0F0
:100920006FF9014600901C2011F07AFE01200A9018
:10093000E7E61FF07FF9014600901D2011F070FEE0
:1009400001200A90DDE620F007FB1E2011F0DCFDFF
:1009500001200A90D5E618F0D3FA1F2011F0D4FD3B
:1009600001200A90CDE6002204A901A809F03EF971
:1009700050B1BDF81000C0B2009018F019FB202053
:1009800011F0C2FD01200A90BBE6012206A901A8D0
:1009900009F0D4F998B1002204A901A809F026F9B8
:1009A00068B1BDF81000C0B201460090BDF8180053
:1009B00018F00CFB212011F0A7FD01200A90A0E601
:1009C000002206A901A809F0B9F940B1BDF8180044
:1009D00018F0ACFA222011F097FD01200A9090E661
:1009E00018F0A0FA232011F08FFD01200A9088E66C
:1009F000012207A901A809F027FA88B1002206A957
:100A000001A809F09BF958B1BDF81810079818F023
:100A1000F9FA01460090242011F08AFD01200A9085
:100A20006FE618F0E9FA01460090252011F080FDEC
:100A300001200A9065E6012207A901A809F004FA3D
:100A400088B1002206A901A809F078F958B1BDF8CB
:100A50001810079818F09AFA01460090262011F015
:100A600067FD01200A904CE618F08AFA01460090D2
:100A7000272011F05DFD01200A9042E618F04EFAA1
:100A800001460090282011F053FD01200A9038E61D
:100A90000FF074F9292011F037FD01200A9030E69B
:100AA0000FF06EF8014600902A2011F07DFD012024
:100AB0000A9026E60FF0C0F8014600902B2011F0B6
:100AC00055FD01200A901CE6002202A901A808F0A9
:100AD00045FF50B19DED020B0FF030F9014600903B
:100AE0002C2011F061FD01200A900AE6FCF798FD28
:100AF000014600902D2011F093FD01200A9000E6A0
:100B0000FCF7D2FD014600902E2011F089FD012056
:100B10000A90F6E5FCF778FD2F2011F0F5FC012096
:100B20000A90EEE5FCF70EFD302011F0EDFC0120FF
:100B30000A90E6E50CF0DCFD312011F0E5FC012027
:100B40000A90DEE50CF02EFF322011F0DDFC0120D2
:100B50000A90D6E5F3F72CF901460090332011F006
:100B600023FD01200A90CCE5F3F762FB342011F05D
:100B7000CBFC01200A90C4E5F3F760FB352011F0AF
:100B8000C3FC01200A90BCE5F3F7F2F8362011F01F
:100B9000BBFC01200A90B4E5002207A901A809F0D6
:100BA00053F938B10798F3F73DFB372011F0ACFC4F
:100BB00001200A90A5E5F3F727FA014600903820B6
:100BC00011F02EFD01200A909BE5F3F725FA01466E
:100BD0000090392011F024FD01200A9091E5F3F7EF
:100BE00020FA014600903A2011F01AFD01200A90E7
:100BF00087E5F3F7BBF8014600903B2011F010FDAC
:100C000001200A907DE5F3F783FA014600903C202D
:100C100011F006FD01200A9073E5EFF7AFFE0146E3
:100C200000903D2011F0DEFC01200A9069E5EFF70D
:100C3000D1FE014600903E2011F0D4FC01200A9024
:100C40005FE51BF013FF014600903F2011F070FCA0
:100C500001200A9055E51BF08BFE014600904020D4
:100C600011F066FC01200A904BE51BF08BFE01465B
:100C70000090412011F05CFC01200A9041E51BF03E
:100C800065FE01460090422011F052FC01200A90BE
:100C900037E51BF049FE432011F036FC01200A9095
:100CA0002FE51BF03BFE01460090442011F040FC74
:100CB00001200A9025E51CF073FA014600904520BA
:100CC00011F036FC01200A901BE51CF075FA014674
:100CD0000090462011F02CFC01200A9011E51CF038
:100CE0007DFA472011F010FC01200A9009E51CF064
:100CF0006FFA482011F008FC01200A9001E516F077
:100D00004BFA01460090492011F012FC01200A9094
:100D1000F7E416F0F7F9014600904A2011F062FC62
:100D200001200A90EDE416F023FA014600904B20D2
:100D300011F03AFC01200A90E3E4002206A901A880
:100D400008F0FCFF50B1BDF8180016F06DFA01462E
:100D500000904C2011F0ECFB01200A90D1E418F037
:100D6000B7FE014600904D2011F0E2FB01200A90F1
:100D7000C7E4012206A901A808F0E0FF80B1002223
:100D800005A901A808F0DAFF50B1BDF81410BDF8AC
:100D9000180018F0C3FF4E2011F0B6FB01200A9096
:100DA000AFE4012206A901A808F0C8FF80B1002223
:100DB00005A901A808F0C2FF50B1BDF81410BDF894
:100DC000180018F0C1FF4F2011F09EFB01200A907F
:100DD00097E40BF061FA01460090502011F0A8FB57
:100DE00001200A908DE40BF051FA01460090512049
:100DF00011F0F8FB01200A9083E417F099FE0146F8
:100E00000090522011F094FB01200A9079E417F031
:100E100083FE01460090532011F08AFB01200A90C6
:100E20006FE417F07FFE01460090542011F080FB24
:100E300001200A9065E417F059FD01460090552005
:100E400011F0EEFB01200A905BE417F027FF56201B
:100E500011F05AFB01200A9053E4002206A901A8D0
:100E600008F06CFF50B1BDF8180017F0CDFC01463A
:100E70000090572011F0D4FB01200A9041E4012298
:100E800006A901A808F05AFF90B1002205A901A8FF
:100E900008F054FF60B1BDF81410BDF8180017F049
:100EA000DBFC01460090582011F0BAFB01200A90AB
:100EB00027E417F069FD01460090592011F0B0FBBE
:100EC00001200A901DE417F067FD014600905A20AA
:100ED00011F0A6FB01200A9013E417F04DFD014626
:100EE00000905B2011F09CFB01200A9009E417F0B0
:100EF0005BFD014600905C2011F092FB01200A90FE
:100F00000AE417F059FD014600905D2011F088FBBE
:100F100001200A900AE417F083FD014600905E204C
:100F200011F07EFB01200A9008E417F05FFD0146F6
:100F300000905F2011F074FB01200A9006E417F086
:100F400089FD01460090602011F06AFB01200A90A3
:100F500004E417F0F3FD01460090612011F024FB3A
:100F600001200A900AE417F067FE01460090622013
:100F700011F056FB01200A9008E417F067FE0146C5
:100F80000090632011F04CFB01200A9006E417F05A
:100F9000A7FE01460090642011F0CAFA01200A90D1
:100FA00004E417F08FFE01460090652011F0C0FAAE
:100FB00001200A900AE417F0F7FD01460090662030
:100FC00011F02EFB01200A9010E417F0CDFD014630
:100FD0000090672011F024FB01200A9006E417F02E
:100FE0001BFE01460090682011F01AFB01200A90B8
:100FF00004E417F001FE01460090692011F010FB97
:1010000001200A900AE417F0BFFD014600906A2013
:1010100011F006FB01200A9008E417F0D5FD014607
:1010200000906B2011F0FCFA01200A9006E417F002
:1010300043FF014600906C2011F0F2FA01200A9063
:1010400006E417F071FC014600906D2011F070FA73
:1010500001200A900EE417F017FD014600906E2063
:1010600011F066FA01200A9004E417F031FD014600
:1010700000906F2011F05CFA01200A9004E4002235
:1010800006A901A808F05AFE50B1BDF8180017F0E3
:101090009BFC01460090702011F0C2FA01200A90DA
:1010A00004E4002206A901A808F048FE50B1BDF8EA
:1010B000180017F0BDFC01460090712011F0B0FA45
:1010C00001200A9006E4002206A901A808F036FED5
:1010D00050B1BDF8180017F091FC01460090722045
:1010E00011F09EFA01200A9006E4002206A901A848
:1010F00008F024FE50B1BDF8180017F0B3FC01460B
:101100000090732011F08CFA01200A9006E401226D
:1011100006A901A808F012FE90B1002205A901A8B5
:1011200008F00CFE60B1BDF81410BDF8180017F0FF
:1011300039FB01460090742011F072FA01200A90E8
:1011400008E418F02DF801460090752011F0F0F930
:1011500001200A9006E418F00BF801460090762072
:1011600011F0E6F901200A900EE418F007F80146A4
:101170000090772011F0DCF901200A9004E418F0C7
:1011800003F801460090782011F0D2F901200A906E
:1011900015E417F0FFFF01460090792011F0C8F91F
:1011A00001200A900BE417F06DFF014600907A20B1
:1011B00011F0BEF901200A9011E417F0B1FF0146C9
:1011C00000907B2011F0B4F901200A9007E417F099
:1011D00099FF014600907C2011F0AAF901200A90A5
:1011E00005E417F05CFF014600907D2011F0A0F9A6
:1011F00001200A9014E417F05EFF014600907E2063
:1012000011F096F901200A900AE417F06EFF0146EA
:1012100000907F2011F08CF901200A900AE417F069
:1012200057FF01460090802011F082F901200A90BA
:1012300019E417F081FF01460090812011F078F940
:1012400001200A900FE417F085FF014600908220EC
:1012500011F06EF901200A9005E4012204A901A809
:1012600008F0C4FCD0B1012206A901A808F066FD6F
:10127000A0B1002205A901A808F060FD70B1BDF879
:101280001000C0B20090BDF81420BDF8181018F07E
:1012900077F8832011F038F901200A9009E401223F
:1012A00006A901A808F04AFD80B1002205A901A8FD
:1012B00008F044FD50B1BDF81410BDF8180018F046
:1012C00072F8842011F020F901200A900DE403F057
:1012D0007BFB01460090852011F02AF901200A903D
:1012E0000DE403F0C9FE01460090862011F098F944
:1012F00001200A900DE403F0C7FA01460090872010
:1013000011F070F901200A900BE403F0DBFE0146B6
:101310000090882011F084F901200A9009E404F07B
:10132000C1FC01460090892011F07AF901200A9051
:1013300007E404F0A5FA014600908A2011F070F944
:1013400001200A9005E404F0C7FA014600908B20C2
:1013500011F066F901200A9005E403F0F5FA014660
:1013600000908C2011F0E4F801200A900BE403F0C7
:1013700091FA014600908D2011F016F901200A9093
:1013800009E403F0EDFA014600908E2011F00CF90B
:1013900001200A900EE403F0EFFA014600908F203E
:1013A00011F002F901200A9004E403F0D3FA014697
:1013B0000090902011F0F8F801200A9004E403F066
:1013C00049FE01460090912011F02AF901200A906F
:1013D00004E403F0CBFA01460090922011F0E4F807
:1013E00001200A9004E403F0CDFA01460090932016
:1013F00011F0DAF801200A9004E402F00FFF014630
:101400000090942011F0D0F801200A9004E402F03A
:101410006BFE01460090952011F0C6F801200A905D
:1014200004E404F021FA01460090962011F0BCF883
:1014300001200A9004E402F03FFE0146009097204C
:1014400011F0B2F801200A9004E402F041FE0146D6
:101450000090982011F0A8F801200A9004E403F00D
:1014600007FA01460090992011F09EF801200A9099
:1014700004E403F003FA014600909A2011F094F876
:1014800001200A9004E404F057F89B2011F03CF886
:1014900001200A9004E403F0A7FA014600909C2082
:1014A00011F046F801200A9004E4002206A901A8E0
:1014B00008F044FC40B1BDF8180004F0FDFB9D208D
:1014C00011F022F801200A9008E404F07BF90146AB
:1014D00000909E2011F02CF801200A9006E404F000
:1014E000B7F9014600909F2011F022F801200A90E0
:1014F00004E415F0E7FE01460090A02011F054F836
:1015000001200A9004E415F0CFFEA12010F0FCFFAA
:1015100001200A9006E415F0BDFEA22010F0F4FFB1
:1015200001200A9008E415F0ABFEA32010F0ECFFB8
:1015300001200A9012E411F087FD01460090A420DA
:1015400011F032F801200A9008E411F0E7FC01469E
:101550000090A52010F0ECFF01200A9008E411F0A3
:10156000EFFC01460090A62011F01EF801200A9021
:1015700016E411F0EBFC01460090A72011F014F8DE
:1015800001200A900CE411F04DFD01460090A820C6
:1015900011F00AF801200A901AE411F037FD014613
:1015A0000090A92011F000F801200A9010E411F039
:1015B0003FFD01460090AA2010F0F6FF01200A909E
:1015C00006E411F03BFD01460090AB2010F0ECFF6B
:1015D00001200A9006E411F01FFD01460090AC20A6
:1015E00010F0E2FF01200A9006E411F009FD014627
:1015F0000090AD2010F0D8FF01200A9006E411F011
:10160000ABFC01460090AE2010F0CEFF01200A9006
:1016100006E411F0BFFC01460090AF2010F0C4FFBB
:1016200001200A9006E411F0A3FC01460090B020CE
:1016300010F0BAFF01200A9006E411F093FC014675
:101640000090B12010F0B0FF01200A9004E411F0E6
:1016500095FC01460090B22010F0A6FF01200A90F0
:101660000CE411F091FC01460090B32010F09CFFB7
:1016700001200A901CE411F093FC01460090B42074
:1016800010F092FF01200A9012E411F08FFC014645
:101690000090B52010F088FF01200A9008E411F0B6
:1016A000A3FC01460090B62010F07EFF01200A90B6
:1016B00008E411F087FC01460090B72010F074FF99
:1016C00001200A9008E411F077FC01460090B82050
:1016D00010F06AFF01200A9008E411F079FC01463D
:1016E0000090B92010F060FF01200A9008E411F08A
:1016F00075FC01460090BA2010F056FF01200A90B8
:1017000008E411F077FC01460090BB2010F04CFF7C
:1017100001200A9008E411F007FC01460090BC206B
:1017200010F042FF01200A9008E411F003FC01468A
:101730000090BD2010F056FF01200A9008E412F03E
:10174000D3FC01460090BE2010F0F2FE01200A906A
:1017500008E411F0B3FB01460090BF2010F060FFD9
:1017600001200A9008E411F0CDFB01460090C02052
:1017700010F056FF01200A9008E411F099FB014691
:101780000090C12010F010FF01200A9008E411F031
:10179000B3FB01460090C22010F024FF01200A9004
:1017A00008E411F0B5FB01460090C32010F038FFAB
:1017B00001200A9008E411F099FB01460090C42032
:1017C00010F02EFF01200A9008E411F06BFB014697
:1017D0000090C52010F024FF01200A9008E411F0C9
:1017E00079FB01460090C62010F0DEFE01200A9031
:1017F00008E411F075FB01460090C72010F010FFBF
:1018000001200A9008E411F05FFB01460090C82017
:1018100010F006FF01200A9008E411F041FA014699
:101820000090C92010F0FCFE01200A9008E411F09D
:10183000CDFA01460090CA2010F0F2FE01200A9075
:1018400008E411F0C9FA01460090CB2010F0E8FE40
:1018500001200A9008E411F09BFA01460090CC2088
:1018600010F0DEFE01200A9008E411F06DFA014646
:101870000090CD2010F0D4FE01200A9010E411F069
:101880001BFA01460090CE2010F08EFE01200A9037
:1018900006E411F08FFA01460090CF2010F0C0FE50
:1018A00001200A900EE411F079FA01460090D02050
:1018B00010F0B6FE01200A9004E411F099FA0146F6
:1018C0000090D12010F0ACFE01200A900CE411F041
:1018D00077FA01460090D22010F0A2FE01200A9073
:1018E00014E411F0FBF901460090D32010F098FEAB
:1018F00001200A900AE411F0F7F901460090D42083
:1019000010F070FE01200A901AE411F029FA014645
:101910000090D52010F084FE01200A9010E411F010
:1019200019FA01460090D62010F07AFE01200A90A4
:1019300006E411F027FA01460090D72010F070FE5F
:1019400001200A9006E411F017FA01460090D82011
:1019500010F066FE01200A9006E411F0CBF9014672
:101960000090D92010F05CFE01200A9006E411F0EE
:10197000D3F901460090DA2010F052FE01200A90BF
:1019800006E411F0C3F901460090DB2010F048FE98
:1019900001200A9006E411F037FA01460090DC209D
:1019A00010F03EFE01200A9006E411F027FA0146ED
:1019B0000090DD2010F034FE01200A9006E411F0C2
:1019C000BDF901460090DE2010F02AFE01200A90A9
:1019D00006E411F01FFA01460090DF2010F020FE0F
:1019E00001200A9006E411F0C1F901460090E020C0
:1019F00010F016FE01200A9006E411F011FA0146DB
:101A00000090E12010F00CFE01200A9006E411F095
:101A100059F901460090E22010F002FE01200A90E0
:101A200006E411F085F901460090E32010F0F8FD7E
:101A300001200A9006E411F04BF901460090E420E1
:101A400010F0EEFD01200A9006E411F0ADF9014618
:101A50000090E52010F0E4FD01200A901EE411F052
:101A6000C1F901460090E62010F0DAFD01200A904D
:101A700014E411F057F901460090E72010F0D0FD72
:101A800001200A900AE411F03BF901460090E82099
:101A900010F0C6FD01200A9018E411F007F9014684
:101AA0000090E92010F0BCFD01200A900EE411F036
:101AB000C9F901460090EA2010F094FD01200A9037
:101AC00004E411F0C5F901460090EB2010F08AFD06
:101AD00001200A9000E211F0C1F901460090EC20CB
:101AE00010F080FD01200A90F6E111F0C9F90146DD
:101AF0000090ED2010F076FD01200A90ECE111F04D
:101B000095F901460090EE2010F06CFD01200A903E
:101B1000E2E111F091F901460090EF2010F062FD32
:101B200001200A90D8E111F09FF901460090F020C1
:101B300010F058FD01200A90CEE111F09BF901460A
:101B40000090F12010F04EFD01200A90C4E111F048
:101B500083F801460090F22010F062FD01200A9007
:101B6000BAE111F07FF801460090F32010F01CFD5F
:101B700001200A90B0E111F07BF801460090F420BA
:101B800010F030FD01200A90FBE311F077F80146D8
:101B90000090F52010F044FD01200A90F1E311F0CF
:101BA00073F801460090F62010F03AFD01200A90EB
:101BB000E7E311F06FF801460090F72010F012FDF6
:101BC00001200A90DDE311F041F801460090F82071
:101BD00010F0EAFC01200A90D3E311F031F801463D
:101BE0000090F92010F01CFD01200A90C9E30EF0CE
:101BF000FFFBFA2010F088FC01200A90C1E30EF0F0
:101C000001FCFB2010F080FC01200A90B9E30EF0EB
